:020000024000BC
:100000006FD0C2500000000000180118002801281D
:100010000228032800290129022903290429052986
:10002000062907290829002A012A022A032A042A64
:10003000052AA62A2CE10600D64104006804002007
:10004000EA040020EA030020B80300205003002047
:10005000BA2900206E4204009043040026460400A2
:10006000404704002E410400DC400400B40200209C
:1000700054020020FC4B04006408002044420400A9
:10008000024904001E7B0600047D06006A7D06000E
:10009000245706005E570600AA860500787B0500F7
:1000A000F475060030490400FC5E0600F8FA04000E
:1000B00086FB0400E4FB0400005404003E540400EA
:1000C000B452040006BD0400ECB70400DC2A002092
:1000D0002AC904007CCC04008EAA040030AA0400C3
:1000E000FCAD0400DAAA04000EAA040086AA0400EB
:1000F000C4A904005CAB0400B4AB040064AB04000E
:1001000068AB0400F6AB0400BCAB0400ECAB04002D
:10011000CEB00400D2B0040058AB040060AB0400C1
:10012000F4AB0400D0B00400A2AC04002EB2040072
:100130002ADA04009CDA0400D6DA04004CBF04007A
:1001400062BF04009CBF0400A69F0400ACA1040091
:1001500074A20400A0710400EA6B0400A4950400DA
:10016000666C04005A9104006ABA0600A0B2060048
:10017000A6B70600E2CE0600ACCD060004D206000B
:10018000C0D10600FCD1060050D306005CA10600D9
:10019000E0D206003EC5060064C5060084C5060020
:1001A000C0D30600A0CB060038CB060030D4060032
:1001B000E0A3060078A4060098A406004AA406005E
:1001C000B25E05003C490500B84C0500784A0500C0
:1001D000CA540500923C00208C75060090A10600D0
:1001E0008A4D040074580600DC5E0600D45F0600E9
:1001F000E26D06006A6E0600C86F060006C30400C2
:10020000B45D0500725505000C4705002058050037
:10021000EC4805002A0A00204C5906002AD20600A4
:10022000C4D10600F8D10600F4D10600A6450400AA
:1002300084C0040032D20600586206001E63060025
:10024000866306000EB806002ED2060078D206009D
:10025000FA7A05007CD20600422000200820002007
:10026000EEB7060084B9060080D20600D4D206009C
:10027000D8D2060036D2060070D2060074D206002C
:10028000DCD206006A5E05000000000000000000ED
:10029000000000000000000000000000000000005E
:1002A000000000000000000000000000000000004E
:1002B000000000000000000000000000000000003E
:1002C00097470000938707E117470000130707646B
:1002D0006373F700828023A007009107D5BF97477B
:1002E0000000938767D117E706E01307674C97462E
:1002F0000000938626DE63F3F60082801043110728
:0603000090C39107CDBF80
:100308004111B7E700E022C480433707200006C642
:10031800798C23A0E7180F10000011C199E5B7E701
:1003280000E023A08710014579A80D05334505088D
:10033800130740037199B34705086366A702174579
:100348000000032525D99746000083A626D8639187
:10035800A60217470000032767FA71D3C207DD8D8D
:10036800054502976DBF17450000032565D6E1BF17
:100378007A2131EF5A21636CF704B306F74021481C
:1003880017460000130606F26375D8028328050095
:1003980003586600938687001D8FAA966117DAA214
:1003A80023A016012393060014C15EA1130788FF3A
:1003B8007AA27A226EA12105B307F7407EA2B7E799
:1003C80000E023A08710B240224441018280084106
:1003D800BDBFB7E700E08C433707200023A0E7182C
:1003E800F98D0F10000001E523A0B7108280174394
:1003F8000000032323CE9748000083A828CD9A87BE
:10040800814663FE170903A80700636DF508636B4F
:10041800A808138787006364E508F22321670507A6
:100428006319E60017460000130636D91822050797
:1004380018A2174500001305E5E6D2237A21239375
:1004480007003297334707087AA163856702174385
:1004580000000323E3C7630FF30003D36600631BA5
:100468000300DE2223A0060121073E962106D2A220
:100478007AA1B6879843630417039746000083A6BA
:1004880026C5630ED700762399EAD623522318434C
:10049800A106B296D6A398C37E21A1077EA1B7E78D
:1004A80000E099B7BE86C287A9BFAA871747000090
:1004B800032747C217460000032646C1B305B540C7
:1004C8006314E6003E8529A8930687001843E3E9EC
:1004D800D7FEE3F7E7FE2E85E3E4D5FEE3F2E5FE7B
:1004E800828023AC05FE1C4199E30CC182803E87C3
:1004F80083A787FFEDFF232CB7FE8280411126C218
:10050800B7E400E04AC003A90400B707200006C604
:1005180022C43379F90023A0F4180F10000009E56C
:1005280023A0241101452DA09565938505D0C98D7B
:100538002A842105B3C5050833450508D1336DD193
:10054800FD572320050042A17CA123A024112105E9
:10055800B240224492440249410182804111B7E7E6
:1005680000E04AC003A9070026C23707200006C6D4
:1005780022C4AA843379E90023A0E7180F100000E9
:100588009747000083A747B50144014695E311C882
:10059800A28517450000130525B4974004E0E780BD
:1005A800C0DCA1652685974004E0E78080321DA065
:1005B80003C7E7FF631B970215CCA2851745000008
:1005C800130585B1974004E0E78020DAA165268508
:1005D800EF202069B24022852244B7E700E023A03B
:1005E8002711924402494101828011E03E8683A787
:1005F80087FF69BF3E84E5BF37E700E01C43B706C5
:1006080020002320D718F58F0F10000019C191C1C1
:1006180011E637E700E02320F71082802E960F704E
:10062800B650D5BF37E700E01C43B70620002320AB
:10063800D718F58F0F10000019C1014785E137E77A
:1006480000E02320F7108280B386E50003A80600A7
:10065800B306E5007D1623A00601110775F6C5B798
:1006680037E700E01C43B70620002320D718F58F92
:100678000F10000001C53307C50011E637E700E099
:100688002320F71082800505A30FB5FEE31DE5FEC4
:10069800F5B7B7E600E09C42370620002A87F18FBD
:1006A80023A0C6180F1000000145B306A7008386D3
:1006B800060091E637E700E02320F7108280050561
:1006C800EDB70111B7E700E026CA84434AC83707E7
:1006D800200006CE22CC2A892E86F98C23A0E71882
:1006E8000F1000009305F00432C633450608093997
:1006F8002A8401C53246CA850137F2402285624400
:10070800B7E700E023A097104249D24405618280F0
:1007180037E700E01C43B70620002320D718F58FE1
:100728000F10000001C599C1014711EA37E700E041
:100738002320F710054582800507E309E6FE330804
:10074800E500B386E500034808009422E306D8FED6
:1007580037E700E02320F7100145828037E700E003
:100768001C43B70620002320D718F58F0F10000070
:100778001307F6FFBA952A966317C50037E700E016
:100788002320F71082809821FD150505A30FE5FEAB
:10079800E5B737E700E01C43B70620002320D71849
:1007A800F58F0F10000001C53307C50019E637E7BC
:1007B80000E02320F7100145828014210505E39805
:1007C800B6FEE31CE5FE37E700E02320F7100545F9
:1007D8008280797126D2974400009384649122D450
:1007E800804006D64AD04ECE52CC56CA5AC85EC6AB
:1007F80062C455C437C9C901814B174B0000130B9C
:10080800AB8E1309F937174A0000130A2AAC974A26
:100818000000938A2AA997490000938929B03E20AD
:1008280091EF5C4463990B009CC0032CC4002285A3
:100838004D36628489A823A6FB00C5BF83270B0019
:1008480082971C443307F5406376F50003A78900B7
:100858001D8F2A976368E9062E200820EF20604044
:100868005C405844A9CB0C4417460000032686ABCD
:10087800AE97BE8663E4B70063E4C700B386C7409B
:1008880014C4A28B3A8441FC17470000032787A2AF
:10089800894763E6E7009747000023AD07A0B250F9
:1008A800225492540259F249624AD24A424BB24BFC
:1008B800224C4561828063940B0098C0BDB723A683
:1008C800EB00A5B703274A021DCB63EDA7023385CA
:1008D800A7401C2099EF03479A0183A68900611756
:1008E800B307A7003E8563E4E70063E4D7003385D8
:1008F800D74083A70A016374F50023A8AA00A28B36
:10090800404451B703A78900BA97D1B7011126CA45
:1009180006CE97440000938464A022CC4AC84EC6F1
:1009280052C49C288844DDC3B7E700E003A9070048
:100938003707200023A0E7183379E9000F100000DB
:10094800173700000347C77919CB23A02711F240B6
:100958006244D2444249B249224A0561828017471B
:100968000000130727CD8357C70AB1CB9C44032443
:10097800870A6306F404974900009389A99203A79C
:1009880009012285630DF702173A0000130ACA7598
:1009980083270A008297636EA40C83270A00098CB8
:1009A800829783A7090198443354F40AB307A40033
:1009B8003E8563E4870063E4E7003385E740B7E7F3
:1009C80000E023A027119C44639DA7021744000060
:1009D8001304448D18489737000083A7E770631DF8
:1009E800A70882979444374736FE130707C83697F7
:1009F800B307A7003E8563E4E70063E4D7003385C7
:100A0800D740174400001304E4E55C5C99CB974693
:100A1800000083A626809C463707CDFF7D17F98FF7
:100A28009CC611E1884485475CD09747000083A79E
:100A3800278C829715E15C5C99CF5C5089CF9760D1
:100A480006E0E780009E975006E0E780800E974713
:100A5800000023AB07E2B53B5C5CE38A07EE17377F
:100A680000000327277B1C47B7063300D58F1CC718
:100A7800F9BD9C443E9415B7829714489844B387AF
:100A8800A6003E8563E4D700E3EDE7F63385E7404B
:100A98008DBF9737000023A3A76411C58547173773
:100AA8000000230FF7628280AA8799E517470000A4
:100AB8000347C78709C7F1BF11476369B7001747DD
:100AC800000013076784B3C5E5209CC1828097376F
:100AD800000083A7A76085C3411106C68297973790
:100AE800000083C7E75F89E79737000023A8075E00
:100AF800B240410182809737000083C7675E91E763
:100B08009737000023AC075C82808280411122C4A1
:100B180026C206C64AC0974400009384A4D483C75B
:100B28003402173400001304247EB9C717340000B8
:100B380013044477173900001309C95B0327090018
:100B48001C2014300146B3A5E7208E21A5CD11C283
:100B58001CA00820636FD50697370000238407740C
:100B68009737000083A74758C5EFB2402244924404
:100B780002494101828082971C40F5FF97370000A7
:100B880083C7C77A85E3DC48858B89CFD84C9947DA
:100B9800631EF7009747000023A007CEEF10F01858
:100BA8005C4482971C44D9D3829749B7D84C9D4757
:100BB800E31AF7FE9747000023A007CCEF10F016C2
:100BC8001C48C5B7850793F7F70F0546E3EDD7F639
:100BD80041B73327E5200E2323100700973700007D
:100BE800239107509737000083A74750B347F52054
:100BF8009C4382971C20832609001737000003575F
:100C0800474E3377E540B3A6D7209222518F9AA258
:100C180099C385071CA018201C30E368F7F42DBF82
:100C28009737000083A707701CC8653683C734024E
:100C38008DFF83C7140299CBDC4C89EB97470000E2
:100C4800A38207C4975006E0E780801B973700000F
:100C580083A7076A99DB1C4889DB183083260900BB
:100C6800814763C9E702D84C9147E3E0E7F097472B
:100C7800000083C7A79A918BE39907EE9737000086
:100C880083C70746E39307EE2244B24092440249E1
:100C98004101ADB933A6D7201222E31806EC850727
:100CA800C9B7B7C700401387C7201443139626490E
:100CB80010C301000100938787261735000003251C
:100CC80025609C436A0514C393C7F7FF99835D8D1C
:100CD80082809737000083A7674291C382871305F4
:100CE800F00F82809737000023AAA740828017461A
:100CF80000001306E68F9746000093866691DC365F
:100D0800383E4C4ABA97FD8B33D7F5001CB2DCB697
:100D1800058B0DE7943A13050002B3F7D702814615
:100D280033D8E548630908006394D70018B2828075
:100D3800850693F6F60F0507E314A7FE828097470A
:100D4800000083A767B3C1E741114AC09737000085
:100D580083A7873906C622C426C28297174900008E
:100D68001309098B83278900638DA7046363F5043E
:100D78001D8D974400009384A487BC2C1354550000
:100D88006361F404AD37BC2C0327890093965700A0
:100D980036971D8C2324E900E376F4FE224488303C
:100DA800B2409244024981454101173305E067008A
:100DB8000357173700000327E756B307F7403E9558
:100DC8004DBFB24022449244024941018280828050
:100DD800011126CA9737000083A7073106CE22CC17
:100DE8004AC84EC652C482979744000093844482EE
:100DF8009844AA870145630DF70463E3E706998FD2
:100E0800173900001309C97E93F9F70113D4570065
:100E18008347A901636AF402173A0000130A0A50CB
:100E2800F9350347A9018C4403268A009317570014
:100E3800AE97198CBE8663E4B70063E4C700B38637
:100E4800C74094C4E37EE4FC1315540033653501B0
:100E5800F2406244D2444249B249224A0561828042
:100E68009736000083A6064C3387E640BA9749BFF9
:100E7800411122C4174400001304C49E1C4426C216
:100E880006C6858B9744000083A4048191EBEF206C
:100E9800F0742244B2402685924441016F10907A42
:100EA80098289747000023A3079C8947E301F7FE8A
:100EB8000146930550020145EF103017814517751B
:100EC80005E01305C5D2CD36014681450545EF102D
:100ED800607B5C44858BC5DFB2402244924441016B
:100EE80082809737000083A7E77E63930718011174
:100EF80022CC2A84094506CE26CA4AC84EC6EF2007
:100F08001076973900009389E92F03A60900930703
:100F18008007173900001309292E7CD29737000063
:100F28002380071C83270900973400009384842EAC
:100F3800B7053300D8572285719B13671700D8D798
:100F480098431377F7CF98C398431377F7CF13676E
:100F5800072098C398401447CD8E14C7B7060300DE
:100F68009386862534CA5457F59A54D7984334241F
:100F7800137707F893F6F607558F98C3EF20E00329
:100F880083A60900370500827D15DC4293E7170028
:100F9800DCC203260900030784065C569375F70331
:100FA800E605E98FCD8F5CD69305A0039C4063D5F9
:100FB800E508F84FB70500074D8FF8CFB7C7898EFA
:100FC800938767ED1CC6B7575500938757555CC282
:100FD8008347A40683444406DD8C894717470000ED
:100FE8002320F78A9747000023A407887C44BCDEA7
:100FF8009737000083C7873399C7FC52FDFF97478F
:10100800000023A5078618289D478145172500005D
:101018001305E53A6306F70017050000130585E593
:10102800613410386244F2404249B249A685D2443C
:10103800014505616F1000659305200263DAE5003C
:10104800F84FB70500F9FD156D8FB7050005ADB769
:10105800B70500F96945FD156357E500F84F6D8F31
:10106800B705000391BFF84F6D8F13178729B1B7E4
:101078008280973700009387E75BE853054754253C
:101088006390E60203C747079147631AF700011107
:1010980006CE2AC6EF10D0563245F240056191B50A
:1010A800828083278511E5CB411122C406C65825C5
:1010B8008345E5049437D2272A841377C70F1395FD
:1010C800466063F7C50663510506882793F6F60759
:1010D80094B70546936627006314C5009366170006
:1010E80054A4D8430907D8C3032504114CB82E8645
:1010F800CC430905EFF04FD0832784115438D843E7
:101108003697D8C3DA27158FDAA789473CBC034737
:1011180064039737000083C7871C6369F706B240EA
:1011280022440145410182801367170058A46DBF0E
:101138009376F60F635505028827854513662700C1
:101148006314B5001366170050A454B8A3840700AD
:1011580085473CBC832784119C43D5FBC9B71367DB
:10116800170058A454B8A384070003250411CC43DE
:101178000905EFF06FC8832784115438D843369790
:10118800D8C3DA27158FDAA78D47E1B75C2493E730
:1011980007015CA469B705458280411197370000B3
:1011A80083A7C70322C406C6858B2A84C5E7416581
:1011B800130525F5978005E0E780607141CD3C2552
:1011C8003EA583270412ADE32320A4122322A412F0
:1011D80085472311F404232005007C2854415EA58B
:1011E800583418A5054718B5138517021737000096
:1011F8000327076B15811C437D151375F50F9CC2DA
:101208005C43DCC21C479CC65C47DCC61C4B9CCAC2
:101218005C4BDCCA1C4F9CCE5C4FDCCE0DC1938668
:10122800060213070702C1BF8327441288C38357E6
:1012380024042322A4128507B3C7070859BF173708
:1012480000001307273F1E2785071EA7B240224428
:10125800410182805C2423090400054593C74700A7
:101268005CA4EDB7142D854763EED70A1C3D2A8789
:101278000145DDEB5C2713F507013C2B99CB834631
:1012880067039737000083C7970563ECF60001E50D
:10129800828059E582808357271E0357671EBA97B5
:1012A80021A08357271E75F90145BDCF9387C71223
:1012B8001735000003554507B3B5A70237460F0099
:1012C800411113060624814622C426C206C67D544F
:1012D8003385A70297C006E0E78080569734000060
:1012E80083C45400AA949737000083A7E73D03A757
:1012F80007099C433354E40AFDFB9737000083A792
:10130800A7DE829781476364A400B307A440B24074
:10131800224433B597001345150092444101828059
:101328008147A5BF014582808280173700000327C7
:1013380067ED3C5BFDFF01000100828039C90111A6
:101348006C0022CC06CE2A84EF20D00315C9FD57A5
:10135800630DF502B2479735000083C5B5F863EB16
:10136800B700034594026244F240B385B740056173
:101378006F10D013173700000327C7FABA97D5B7ED
:101388006244F24005616F202043F24062440561E7
:1013980082808280797152CC173A0000130A8A2918
:1013A80026D283244A0906D622D44AD04ECED5C89E
:1013B800973700009387074BD44F15476386E60499
:1013C800DC532A8989CF975006E0E780800597404B
:1013D80006E0E78000769737000023A7074AFD5903
:1013E8006C002685EF20007A0DE91725000013050B
:1013F800E53CEFF00FEA9737000083A7A7E037072F
:10140800100098C70547B8DB0D45B25022549254D6
:101418000259F249624A4561828063743501324457
:10142800AA898440D5FCFD571305F00FE38FF9FC1A
:10143800914763F187029307B4FF2320F90023241F
:10144800FA0A99E79737000083A7C7ED2320F90028
:10145800014565BF9737000083A7C7ECED17A29732
:10146800E9BF09455DB7797126D206D622D44AD09C
:101478004ECE52CC56CA5AC85EC68347550303445B
:101488007513AA843E941374F40F9307400263F60D
:1014980087001304B4FD1374F40F03A9841383A9FC
:1014A800C413A38B841222864A85CE8597C006E092
:1014B800E7804034058915E503CBD412014A814AF7
:1014C800337B6403930B500252864A85CE8597C0BE
:1014D80006E0E780203205890DC563916A0313741D
:1014E800FA0F238B8412B250225492540259F249B3
:1014F800624AD24A424BB24B45618280850A939A2E
:101508004A60050AE3127AFDE9BF83278509035675
:101518000504797193D60701BD8EB3C60608358ECA
:1015280093575640898B135776485D8F93573640AB
:10153800918B5D8F93571640A18B5D8F9317160083
:10154800C18B5D8F9317360093F707025D8F931752
:10155800560093F707045D8F9317760093F7F70FFC
:1015680022D45D8F2A849357D6001355B60011896B
:10157800898B93558600C98F1355F6002582C98F2C
:10158800218AD18F13961500418AD18F1396350081
:1015980013760602D18F1396550013760604D18F61
:1015A800139675001376F60FD18FA207C5455D8F88
:1015B8003307B70226D24AD04ECE03298413832993
:1015C800C4135AC806D652CC56CA369733470708AA
:1015D80013565740098A93577748D18F1356374087
:1015E800118AD18F13561740218AD18F13161700ED
:1015F800418AD18F1316370013760602D18F13163E
:10160800570013760604D18F131677001376F60F5A
:10161800D18F1358B7001356D70013784800098A9A
:1016280013558700336606011358F7002583336680
:101638000601218B518F13161500418A518F1316FD
:10164800350013760602518F1316550013760604DB
:10165800518F131675001376F60F518F2207D98F05
:10166800B387B7025EC6B697B3C7070813D5574006
:10167800098913D77748498F13D537401189498F7E
:1016880013D517402189498F139517004189498F30
:101698001395370013750502498F13955700137575
:1016A8000504498F139577001375F50F598D13D8D5
:1016B800B70013D7D70013784800098B13D68700D3
:1016C8003367070113D8F700A58333670701A18B98
:1016D800D98F13171600418BD98F1317360013773C
:1016E8000702D98F13175600137707041E06D98FE0
:1016F8001376F60FD18FA2073367F5003307B702C9
:10170800130650024A85CE853697B98EB3C40608AB
:1017180033F6C402137BF60F97C006E0E780800D0E
:10172800058905E9834AD412014A930B5002B38A0A
:101738009A02814493DA0A0126864A85CE8597C0A3
:1017480006E0E780200B05890DC563914A0313FB6A
:10175800F40F230B6413B250225492540259F249E5
:10176800624AD24A424BB24B45618280050A137ADB
:10177800FA0F8504E39274FDE9BF8327C508035671
:101788008508797193D60701BD8EB3C60608358ED4
:1017980093575640898B135776485D8F9357364039
:1017A800918B5D8F93571640A18B5D8F9317160011
:1017B800C18B5D8F9317360093F707025D8F9317E0
:1017C800560093F707045D8F9317760093F7F70F8A
:1017D80022D45D8F2A849357D6001355B6001189F9
:1017E800898B93558600C98F1355F6002582C98FBA
:1017F800218AD18F13961500418AD18F139635000F
:1018080013760602D18F1396550013760604D18FEE
:10181800139675001376F60FD18FA207C5455D8F15
:101828003307B70226D24AD04ECE0329040A8329A9
:10183800440A5AC806D652CC56CA369733470708C0
:1018480013565740098A93577748D18F1356374014
:10185800118AD18F13561740218AD18F131617007A
:10186800418AD18F1316370013760602D18F1316CB
:10187800570013760604D18F131677001376F60FE8
:10188800D18F1358B7001356D70013784800098A28
:1018980013558700336606011358F700258333660E
:1018A8000601218B518F13161500418A518F13168B
:1018B800350013760602518F131655001376060469
:1018C800518F131675001376F60F518F2207D98F93
:1018D800B387B7025EC6B697B3C7070813D5574094
:1018E800098913D77748498F13D537401189498F0C
:1018F80013D517402189498F139517004189498FBE
:101908001395370013750502498F13955700137502
:101918000504498F139577001375F50F598D13D862
:10192800B70013D7D70013784800098B13D6870060
:101938003367070113D8F700A58333670701A18B25
:10194800D98F13171600418BD98F131736001377C9
:101958000702D98F13175600137707041E06D98F6D
:101968001376F60FD18FA2073367F5003307B70256
:10197800130650024A85CE853697B98EB3C4060839
:1019880033F6C402137BF60F97C006E0E78080E6C3
:10199800058905E9834A1408014A930B5002B38A62
:1019A8009A02814493DA0A0126864A85CE8597C031
:1019B80006E0E78020E405890DC563914A0313FB1F
:1019C800F40F230F6407B250225492540259F2497B
:1019D800624AD24A424BB24B45618280050A137A69
:1019E800FA0F8504E39274FDE9BF8327450903567E
:1019F8008508797193D60701BD8EB3C60608358E62
:101A080093575640898B135776485D8F93573640C6
:101A1800918B5D8F93571640A18B5D8F931716009E
:101A2800C18B5D8F9317360093F707025D8F93176D
:101A3800560093F707045D8F9317760093F7F70F17
:101A480022D45D8F2A849357D6001355B600118986
:101A5800898B93558600C98F1355F6002582C98F47
:101A6800218AD18F13961500418AD18F139635009C
:101A780013760602D18F1396550013760604D18F7C
:101A8800139675001376F60FD18FA207C5455D8FA3
:101A98003307B70226D24AD04ECE0329040B832936
:101AA800440B5AC806D652CC56CA3697334707084D
:101AB80013565740098A93577748D18F13563740A2
:101AC800118AD18F13561740218AD18F1316170008
:101AD800418AD18F1316370013760602D18F131659
:101AE800570013760604D18F131677001376F60F76
:101AF800D18F1358B7001356D70013784800098AB6
:101B080013558700336606011358F700258333669B
:101B18000601218B518F13161500418A518F131618
:101B2800350013760602518F1316550013760604F6
:101B3800518F131675001376F60F518F2207D98F20
:101B4800B387B7025EC6B697B3C7070813D5574021
:101B5800098913D77748498F13D537401189498F99
:101B680013D517402189498F139517004189498F4B
:101B78001395370013750502498F13955700137590
:101B88000504498F139577001375F50F598D13D8F0
:101B9800B70013D7D70013784800098B13D68700EE
:101BA8003367070113D8F700A58333670701A18BB3
:101BB800D98F13171600418BD98F13173600137757
:101BC8000702D98F13175600137707041E06D98FFB
:101BD8001376F60FD18FA2073367F5003307B702E4
:101BE800130650024A85CE853697B98EB3C40608C7
:101BF80033F6C402137BF60F97C006E0E78080BF78
:101C0800058905E9834AF408014A930B5002B38A0F
:101C18009A02814493DA0A0126864A85CE8597C0BE
:101C280006E0E78020BD05890DC563914A0313FBD3
:101C3800F40F230F6407B250225492540259F24908
:101C4800624AD24A424BB24B45618280050A137AF6
:101C5800FA0F8504E39274FDE9BF411126C206C656
:101C680022C44AC09734000083A444A263890410A4
:101C780003A4C40AAA86054525C43C241307700A90
:101C88006392E70858301C341729000013090969C2
:101C980003268900B387E7020357C900B387E70221
:101CA8001307003293870719B3D7E70203A744093C
:101CB8003E97BA846364F7006364C700B304C740FF
:101CC8009727000083A7474284C28297B387A4401E
:101CD80063F5A40003278900BA9789EB1305F00F71
:101CE800B24022449244024941018280583093060E
:101CF800204E3307D702E3F3E7FE930780FA3CA4AC
:101D08000145F9BF1307800AE39AE7FC972700000B
:101D180083A7873D82972A893545EF204014AD4730
:101D280017370000232EF7B458301C34172600004C
:101D38001306C65EB387E7025A261046B387E70242
:101D48001307003293870719B3D7E70203A744099B
:101D58003E97BA866364F7006364C700B306C7405A
:101D6800E31ED9F617D505E0130565C3EFE07FD26A
:101D78009727000083A707490947F8D785B705457E
:101D880085B7397156D2973A0000938AAAAD83A7CE
:101D98000A033707080026DA06DE22DC4AD84ED6C0
:101DA80052D45AD05ECE62CC66CA6AC86EC6F98F63
:101DB8009734000083A4848D638A071C83A9C40A0E
:101DC80083C7990003A4C90092073E942820B1470D
:101DD80005053305F5025E203E9533450508EFE01D
:101DE800EFF1AA8C630F051A130DC5002324A50172
:101DF80034203146370B0300B386C6022313040090
:101E08000149172A0000130AEA3F972B0000938B19
:101E1800AB3E972D0000938DED3F130B8B15054CB2
:101E2800EA9654C483C679009307D00783250A002D
:101E3800B386F602C1679CC5370833008606B4D15D
:101E480083A60B0090421376F6CF90C29042137689
:101E5800F6CF1366062090C203A50D001045336621
:101E6800060110C503A6090023A8650593055002BD
:101E780090C672205444B2962324DD0014300146E3
:101E8800CA96A301DD0003C504089736000023ADF8
:101E9800069CEF00901983260A00CC461396154934
:101EA800D0C60F10000083260A003706020090C62D
:101EB8001306000823A8CA0003A60B0010421356F5
:101EC8007648631E860B1306E018F0D2CCC6173688
:101ED80000002323069A173600002327069823A01C
:101EE8008601A125EF10906F83A64A00858AD9CA7A
:101EF800EA85268597E005E0E78080B40DE903468A
:101F08005D0049C276204E20B29663DDB606B4283D
:101F1800AC4803258D00918E8906B695EFE0CFED8C
:101F280023020D0003465D007620B29676A00326B4
:101F38000A00310D3452FDFE342005091379F90FDA
:101F4800E362D9EE9C246685A381FC001C20A38251
:101F58000C002383DC002382FC006254F250D2542C
:101F68004259B259225A925A025BF24B624CD24CF5
:101F7800424DB24D2161172305E0670043C61306A1
:101F8800E01AA1B7FD562302DD0055B797270000D8
:101F980083A74727FC5791C78547172700002301C8
:101FA800F714F2506254D2544259B259225A925AF2
:101FB800025BF24B624CD24C424DB24D21618280A1
:101FC800797122D426D22E84AA84414697C506E088
:101FD8009385C5C20A8506D6972004E0E780402C81
:101FE800414697C506E0938565C10808972004E037
:101FF800E780002B3C3010088A85DC875C2026852A
:102008005C875C30DC86973006E0E780A06C03478D
:10201800F1011C200145631EF7000347E1011C3054
:1020280001456318F7000345D1013C201D8D133588
:102038001500B2502254925445618280011122CC7D
:1020480026CA4AC84EC606CEAA841724000003240E
:10205800A46A13092500854905C09C303830858B52
:102068006304F700405CCDBF1946930544004A85D8
:10207800EFE00FEAE31835FFF24022856244D244CC
:102088004249B24905618280411122C426C24AC030
:1020980006C6172400000324246693042500054976
:1020A80001E8B240228522449244024941018280DB
:1020B800A6851305A4022937E30525FF405CCDB7A3
:1020C800411122C426C24AC006C6172400000324B0
:1020D800A46293042500054901E8B2402285224400
:1020E8009244024941018280A6851305A401C93D95
:1020F800E30525FF405CCDB7011126CA644122CC17
:102108004AC84EC652C406CE2A841D49930965059D
:10211800054A3C4463E4F4000545A1A05834DC209A
:1021280063192705034784026304F7008440D5B781
:10213800D83083475405E31BF7FE19469305640519
:1021480013856400EFE0CFDC8547E311F5FED82462
:1021580083479402E31CF7FCFA243E34E318F7FCA7
:102168000145F2406244D2444249B249224A0561DB
:102178008280E31DF7FAD83083475405E318F7FA4D
:102188001946CE8513856400EFE08FD8E31045FB30
:10219800C1BF411122C406C626C24AC01724000086
:1021A8000324C4505DC88347840B1307700A6393E4
:1021B800E7080347140E8347A40B172900001309E7
:1021C800E91583268900B387E7020357C900B38757
:1021D800E7021307003293870719B3D7E7020327EB
:1021E800440A3E97BA846364F7006364D700B30473
:1021F800D7409727000083A727EF04C18297B387AA
:10220800A44063F5A40003278900BA9785CB034748
:10221800140E9306204E3307D70263F1E7029307A3
:1022280080FA230CF40A0145B24022449244024940
:10223800410182801307800A639EE700172506E0A4
:102248001305C563EFE0FF849727000083A787FB8A
:102258000947F8D71305F00FC1BF0545F1B70111BC
:1022680022CC26CA06CE2AC42EC617240000032470
:102278002448854419E001450DA09C841830858BBD
:102288006304F7000044FDB719469305A100130540
:102298002400EFE0EFC7E31795FEF2406244D24412
:1022A80005618280EFE0BF8273000000000000003B
:1022B800972200009382C2E2038302002380020077
:1022C800630F0300F32510342EC097050000938593
:1022D800A5FD73901534EF00805D7300203086DC17
:1022E800EF00E05CE6508280000041114AC01729E7
:1022F8000000130969F00327090026C206C61C5FFF
:1023080022C4972400009384E4EE93D76748C1C79A
:10231800930700061CDF172400001304A454184C6C
:10232800930700086317F7009C409C4393F7070442
:102338001CCC1C4093F7070499CB9727000083A770
:10234800A7DA829748D81C4093F7F7FB1CC01C40BB
:1023580093F7070299CF1C4017270000032787EA45
:10236800B706080093F7F7FD1CC05C5414C786072E
:102378007CD71C4893F7070499EF85475CC8370753
:1023880002009727000083A7E7E798C71307000C08
:1023980018C81854F8D383270900985F135747487B
:1023A80005C3985F1367070198DF9727000083A785
:1023B80067E523A20706854717270000232CF74A5D
:1023C8009C40D8431357174819C7D843759BD8C39F
:1023D800D843799BD8C3B240224492440249410170
:1023E8008280213773002030972700009387874722
:1023F8003707040088DB698F11CF172700000327F0
:1024080067E0FD5634D7972600009386A6E9D84E94
:102418000507D8CE137785000DC398479726000087
:1024280083A686DD1367170098C71307000898CBA3
:10243800D856719B13671700D8D61377150011CF9C
:10244800D8439726000083A626DB13671700D8C356
:10245800D856719B13671700D8D6137765000DC33C
:102468001377450059C798431367170098C39726F1
:10247800000083A666D8D856719B13671700D8D674
:102488004167698F0DC39726000083C6E621C18A7C
:10249800172700001307071AB5C28346470793E6B4
:1024A8000602230AD70637070200698F11CF984B17
:1024B8001377070819C3054798CB9727000083A708
:1024C80067D43707020098C7B70708007D8D0DC18C
:1024D800172700000347571D058B97270000938790
:1024E80067151DCB03C7570713672700A38AE7069D
:1024F8008280D84713671700D8C795BF8346470718
:102508000946BD8A6388C600834647070D46BD8ACB
:10251800E39BC6F8914671B703C75707118B69DB70
:1025280003C7570713678700D1B79726000083A60C
:1025380066CD172700001307E7321C43858B91E708
:102548005C43858B99E3FC52EDFB9727000023A59C
:102558000732828097260000938606CA2A87884217
:102568001C5D93D75748C1EB81C51C59BD839CA1FD
:1025780015C69C42945BC60693D7660163D60600CF
:1025880093E707C0B3C707088316060093975760F9
:10259800A9CABE968947B3C6F60216A297270000B5
:1025A80083A747C6BC4B083393D757488DCF29C557
:1025B8009726000083A6862C93F6060493079500B9
:1025C80009459DCABA979C230547194593F6F7060E
:1025D8006394E60201459397476063DF0700394536
:1025E80082801EA265BF2A9748331375F5077D15AB
:1025F8003335A0008280054582809727000083A795
:10260800E7BF99CB944BD04B9842518F98C29443D3
:102618009C479842D98F9CC217260000130686BE95
:10262800054818429726000083A606BD9727000094
:1026380093874723631D050388421365050888C2ED
:1026480083C62702B3C5D5209385A50C5447139597
:10265800164948C70F1000001842370602008605C1
:1026680010C71306000890CB6CD354C782808842E9
:102678001375F5F788C283C62702B3E5D52093857D
:10268800E50EE9B7411122C4AA8706C626C22E85DF
:1026980017240000130404B7B285CDEB1C40F8538F
:1026A8007DFF3707020098C79727000023A0071C63
:1026B80097240000938484C1DC5085C7B7E700E005
:1026C8003707200023A0E728B7F700E0938707D053
:1026D800984B6D9B98CB984B1367870398CB7300E7
:1026E8005010213F9727000083A707B1984313177D
:1026F800772998C3D857719BD8D79727000023AD5F
:1027080007169727000023A107161C40094798C3FE
:10271800DC5099CB37F700E0832707D193E7870090
:102728002328F7D073005010144017270000130710
:1027380067131C47858B91E75C47858B99E3FC52AF
:10274800EDFBB24022449244410182800D476390E0
:10275800E7069727000023AB07109727000023A957
:10276800071097240000938464B6DC5085C7B7E748
:1027780000E03707200023A0E728B7F700E0938799
:1027880007D0984B6D9B98CB984B1367870398CBD2
:10279800730050109D359727000083A7E7A598433D
:1027A8001317772998C3D857719BD8D795B705477A
:1027B800E39CE7F697260000938646B1DC5285C76E
:1027C800B7E700E03707200023A0E728B7F700E0C5
:1027D800938707D0984B6D9B98CB984B13678703CB
:1027E80098CB730050101C40D04713171649D8C710
:1027F8000F1000001C403707020098C71307000895
:102808009725000023A8E506172700000327C79E81
:1028180018431357774819C71307E018F8D3D0C7D8
:10282800DC52C5BD1307E01AD5BF9727000083A760
:10283800E79C89CFD44303A88700984233670701F0
:1028480098C2D447DC4B9842D98F9CC2054797273A
:10285800000083A7679A9505631BE50298431367F1
:10286800070898C3984F137707C01367A71398CF23
:1028780013078007B8BB939735009387C70319C21E
:1028880093171600172700002322F7008280984329
:102898001377F7F798C3984F137707C01367271371
:1028A80098CF1307F007B8BB93974500F9B7972758
:1028B800000083A727958847D847798D01C988C71D
:1028C8009727000083A7C79391C38287828089676F
:1028D8001727000003270793938707F47CD39726CD
:1028E800000083A6269383A7060993D7A74991C713
:1028F80083A7060993D7974999E37C53EDF782801C
:10290800411106C622C426C24AC063030510AD475A
:102918002A8463EAA70C1304F5FF1374F40F1385D4
:10292800F5FF01469305F00F1375F50FFD3D97244C
:1029380000009384248E9840172900001309C98B3E
:10294800136404045C571374F40717050000130597
:10295800250DF59B5CD7032709001C4393F707F85F
:10296800C18F1CC3B7477671938797121CC7B75797
:10297800550093875755172400001304A4885CC397
:1029880018409727000023AF07EC5C43F99B5CC312
:10299800A547172700002325F7EEEFE08F8F144097
:1029A8009727000023AA07EC9727000023AE07EA21
:1029B8000327090085479CC21C433706330001459D
:1029C80093F7F7CF1CC31C4393F7F7CF93E7072080
:1029D8001CC398401C47D18F1CC7B70703009387B7
:1029E8008715BCCA05A0B1476307F50293076002C3
:1029F80063E5A7001304E5FF0DB793077002494587
:102A0800E30FF4F0B240224492440249410182802B
:102A18001304500229B71304600211B717270000E6
:102A2800032787E4058B972700009387A7C001CF6A
:102A3800171700000327477C185F1357574801E70B
:102A48009A2705079AA703C68703EC33C8234DBD09
:102A5800AA87171500000325A56911E182803A218C
:102A68006315B7001821E30BF7FE4845FDB7411180
:102A780022C406C626C24AC02E849DCD13F915006D
:102A88008147414763040904131745003E97B1463F
:102A98003307D7029714000083A40466B317F028FD
:102AA80033C90708BA949C40C840829723A0040001
:102AB80023A2040033448900B24022852244924470
:102AC800024941018280B356F448DDFE8507E39C44
:102AD800E7FECDB7011126CA06CE22CC4AC84EC69B
:102AE800AE84B1C593F7150001444147A1CF9317B0
:102AF8004500A2973147B387E702971900009389E9
:102B0800A95F03A909003E998327090081C7032506
:102B18004900829731473307E40283A70900BA972F
:102B28009C478DC733148028B3470408BD8CF240F6
:102B380062444249B2492685D24405618280B3D6AF
:102B48008448D5F60504E31CE4FECDB7232009002C
:102B580023220900C1BF7971B7E700E022D480437E
:102B680052CC06D626D24AD04ECE56CA5AC85EC6CF
:102B780062C43A8A37072000798C23A0E7180F101F
:102B8800000005E123A087100945B2502254925451
:102B98000259F249624AD24A424BB24B224C456131
:102BA80082809717000083A72754B6892A89AE8A9E
:102BB800328B971B0000938B2B54829703A70B0033
:102BC8008144B146C147338CD40233068701104291
:102BD80041E2C165938505F04145EFD06FF219EDEB
:102BE8009717000083A7877181C781451145829790
:102BF800B7E700E023A087102D4541BF1717000055
:102C08001307074F1C43A1E308C323000500B317AC
:102C180090283EA183A70B002326050023246501E5
:102C280023224501E29723A0270123A2570123A4C9
:102C380047016384090023809900B7E700E023A0D7
:102C48008710014599B73E87DC47F5FF48C775BF30
:102C58008504E39AF4F6B7E700E023A0871021453E
:102C68002DB7B7E700E09843B706200023A0D71890
:102C7800758F0F1000009716000083C6B662637345
:102C8800D5029716000083A6E6463325D5201621DF
:102C9800D58D0EA19716000023AE066023A0E7107D
:102CA8000145828023A0E7100D4582800111B7E716
:102CB80000E022CC80433707200006CE26CA4AC847
:102CC800798C23A0E7180F100000BD4763E9A7041B
:102CD80031473307E5029717000083A7E741BA9702
:102CE8009C4395CF3315A0282E89B3450508014587
:102CF8002EC6B93BAA8409C9B2450145972004E00C
:102D0800E780A08123A42401B7E700E023A087106F
:102D18000145F2406244D244424905618280B7E7E6
:102D280000E023A087100945EDB79726000083C669
:102D3800E68B9717000083A7A74401476394E60032
:102D4800014582808E23138687026394A5003E8501
:102D5800828005071377F70FB287CDB79727000052
:102D680083C7D788AA86850717150000032505425B
:102D7800014712216307D60005071905E36BF7FE23
:102D8800014582802A87171500000325A54011E117
:102D980082801C45B227636BC70003584500B30601
:102DA800C8006355D7008146639406010841C5B73A
:102DB80003D3A700938807016316E30091C192A18A
:102DC8003E8582808506C687B3C60608F1BF97266A
:102DD800000083C6A6819717000083A7673E0147B6
:102DE8006394E60001458280AE231386C70363948B
:102DF800A5003E85828005071377F70FB287CDB708
:102E0800411122C406C697270000238F078817148C
:102E180000000324E43B05C06C390145B315B02814
:102E2800B3C50508972004E0E78040BC9307102746
:102E38003305F50202942244B2408145014541011F
:102E48006FD09FC6411106C6383D19C73425631097
:102E5800D704B24041016DB73C2DE5DF3825E30AC0
:102E6800F7FE3CA5814517E5FFFF1305C520EFD008
:102E7800BFC39717000083C7674B99C79717000010
:102E880083A747385147F8D3B240410182803C2D8F
:102E980089C7E398F6FC38A5F1B7C5FEEDBF411127
:102EA8004AC0172900001309E99B8327890022C417
:102EB80026C206C6971400009384C477858BE05019
:102EC8009DCB9727000023A3079A83C74407C18B8C
:102ED80085CFEF00B07083C7440793F70702E5DF9B
:102EE80083C74407228593F7F70C238AF406974093
:102EF80005E0E78060EDEF00706E22852244B24065
:102F0800924402494101EDBD83C75407858B91CB9B
:102F1800EF00D06C8D47230EF406BC5822858297AB
:102F2800D9BF83C744071547BD8B6395E70483471B
:102F3800B406034534060146930550025D8DEFF053
:102F4800DF8E014681450545EFF0CFF38327C900A1
:102F5800858BD5D322859727000023AB0790974010
:102F680005E0E78020CE41F9B2402244924402496C
:102F78004101828083C744071947BD8BE39DE7F66B
:102F88008347B406034534060146930550025D8D18
:102F9800EFF0BF89014681450545EFF0AFEE832785
:102FA800C900858BA9DB22859727000023A2078CFF
:102FB800974005E0E78040A27DB7411122C426C2B0
:102FC80006C67C2578452A84BD8B1CA91CA31D47F1
:102FD8006445639BE7340547B8A08347F5058D46EC
:102FE8006395D7185E2DCDE37C491147B18B638D6E
:102FF800E70831476398E700034715068347F50755
:103008006304F7088547BCB0194693056403138524
:103018004400EFD06FDEBC20990793F7F70FBCA0F0
:10302800034704061377070401CFB8301367070472
:10303800B8B07844BA975838B8B3BC208507BCA054
:103048009717000023820766BC2013F7F7030507CC
:1030580018B80347E4051A07D98FBCA0834754035F
:10306800858B91E70347440389476317F700784442
:103078001C2393E707041CA37C44183898B3B24078
:103088002244924441018280A147BCB08357C406C0
:10309800971500009385055A171600001306861623
:1030A800DCA08357C406034714067444A18312079F
:1030B800BD8BD98FDCB2B4208547890693F6F60F0D
:1030C800B4A0171700000347275E631EF706183CD5
:1030D8009387E6008E07231AF4069387C708B387F9
:1030E800E702794510420948238A0507C1650CC6DD
:1030F800938707FBB3C7070893877716B3C7A70259
:1031080033C70708B387A70286073CD2BC3093E7CA
:103118000701BCB07C44B6978346240693E60604B0
:10312800B4B3B4207C44B697D8A3B4207C4421839C
:103138007D8BB697834634069606558FD8B3BC2048
:103148008D07BCA011B71042F94738520583335791
:10315800F7023C5268528583FD8BAA977CD28D4733
:10316800238AF5063347070855B71946639DC712E2
:103178005E2DC1E393056503B8B013854400EFD015
:10318800AFC7BC201385A4009907BCA0BC3093E747
:103198002700BCB083475403898B95CF0C58BC29B2
:1031A8009DCB1946D105EFD02FC578441C2393E752
:1031B80007F81CA3BC20990793F7F70FBCA0034797
:1031C800040613770704E30D07E6B430784493E662
:1031D8000604B4B085B58347D40391C778441C234B
:1031E80093E707F81CA319469305E403EFD0CFC073
:1031F800D1B7A147BCB08357C506DCA08357C50625
:10320800034615066C45A1831206BD8BD18FDCB130
:10321800B020171500001305E541971500009385A8
:1032280065FE09061376F60FB0A09717000083C74E
:10323800A7476398E704183C9307E6008E07231A0C
:10324800F4069387C708B387E70279488946230AB3
:10325800D5069441C1658CC6938707FBB3C7070899
:1032680093877716B3C7070333C70708B3870703DE
:103278008607BCD2BC3093E70701BCB07C44B29748
:1032880061BD8C41B851F94705833357F702BC51EA
:1032980003A845068583FD8BC297FCD1230AD50672
:1032A80033470708C1BFA147BCB08357C506DCA098
:1032B8008357C506034615066C45A1831206BD8BC8
:1032C800D18FDCB1B020171500001305A53609060B
:1032D8001376F60FB0A09717000083C7E73C971541
:1032E800000083A525F2E39FE7F8183C9307E60062
:1032F8008E07231AF4069387C708B387E702F946AF
:103308000948230A0507416588C5938707FBB3C7A2
:10331800070893877716B3C7D70233C70708B38759
:10332800D7028607BCD1B9B70547639EE706B14700
:103338001CB983475503898BA1CB0C59BC29A9C754
:103348001946D10513858400EFD00FAB78441C23B0
:1033580093E707F81CA36844194693056403090515
:10336800EFD08FA911679717000083A7A739F98FA6
:10337800E38607CE7C24B98BE39207CE78441C23DE
:1033880093E707021CA3D9B98347D40389C79C20B4
:1033980093E707F89CA0684419469305E4032105C0
:1033A800EFD08FA54DBF522D0C559307660093F7AC
:1033B800F7031CB913858400E5B7011126CA9714D1
:1033C80000009384244A9C4422CC06CE17140000A3
:1033D80013044426858B6850D9C32AC69717000062
:1033E80023A60748EF00901F034744078947324543
:1033F8006307F700034744078D47631EF7029716D4
:10340800000083A626E0BC520357450785831307AF
:10341800C71263F2E702BC528583B1C391470347E1
:103428004407E31EF7FE6244F240D24405611743A5
:1034380005E06700C3C2382D3C3D09CF3425630938
:10344800D7026388F60238A56244F240D244056187
:103458006FD03FA999CF382509EF3CA5F5B72AC603
:10346800EF00D01762443245F240D244056149BAB0
:10347800EDF7DC4CEDF70347440789476307F7008E
:10348800034744078D47E31CF7FC9147034744076C
:10349800E31EF7FE49BF63000532011122CC06CEB8
:1034A80026CA4AC84EC652C456C2582585472A84D9
:1034B8006318F72C971700009387C73AD44F15471E
:1034C800638AE600D44F0D476386E600D84FAD47C0
:1034D8006312F7026C386244F240D2444249B2495E
:1034E800224A924A01450561B315B028B3C50508BB
:1034F8006FF02FF7163113070064971400009384B8
:1035080064133347D7029C20E8D0850793F7F70F59
:103518009CA063CAE700972004E0E78020939717F0
:1035280000002389071078249D47631FF704834709
:103538009406B1C38356040763ECF6020C24930780
:1035480030041CAC1305300493F6F60F014697704F
:1035580006E0E78060B722856244F240D2444249DF
:10356800B249224A924A0561174305E06700235F82
:1035780085062318D406930530020545972004E0F4
:10358800E780A0852301A4060549238A2407183C5F
:103598008D47631CF70E971004E0E78080EE0D89D5
:1035A800630F051463162517930760023CA493075D
:1035B80050023CAC9307700278243CBC85476302F8
:1035C800F70889659385F57013051027171A000009
:1035D800130ACAD483497401972004E0E780608203
:1035E8000E30835ACA002A8913060064B38555032E
:1035F800814613850532B335B50097A006E0E7800C
:103608002024AA84B335590337460F00130606242D
:1036180081463305590397A006E0E7806022832797
:103628000A00AA948297B307950003278A00BE85EB
:1036380063E4A70063E4E700B385E7404E85EFF055
:10364800EFE683475403898BE9CB8347C403F1C76B
:103658000C58E1C5BC25F1C38947230AF402194671
:10366800B10513056403EFC03FF90347C407894751
:1036780063E9E70A22856244F240D2444249B249EA
:10368800224A924A05616FD0DF8589467C346315EA
:10369800D70213F7170019CB898B1307500291EB48
:1036A8009307700238A43CAC814739B7130760020E
:1036B800C5BF93076002FDB799CF93F617001307AC
:1036C800500291E6898B13B717001307670238A4D5
:1036D800230D0400D1BF3C2C130740026368F70098
:1036E800930750023CAC3C2C3CA47DBF850793F764
:1036F800F70F3CAC13077002E364F7FEEDB713074E
:103708007002930750023CAC38A4930760026DB571
:103718001307500293077002FDB78547230AF40286
:10372800A9B70327C40A9716000083A6E69B3C277F
:10373800ADC31C37583397140000938424BE9044BB
:10374800B387E702DA24B387E702130700329387C7
:103758000719B3D7E702032744093E973A896364F8
:10376800F7006364C7003309C7408296B307A940CE
:103778006374A9009844BA9703576407E3FCE7EE1B
:10378800F2406244D2444249B249224A924A05610F
:10379800828083248409829663E9A400835764079E
:1037A8003385A440E378F5ECE1BF9717000083A7C1
:1037B80067B7BE94E5B7828001114EC6971900001D
:1037C800938949E722CC03A4C9094AC817190000FC
:1037D8001309C9B40357C90026CA83546408832748
:1037E800040906CEB384E40237470F009306F72393
:1037F8001307072452C456C25AC0B694B3D4E4027D
:1038080063E09704171A0000130A0A8EB3849740DE
:1038180083270A00829763E9A4023385A440634999
:10382800050283570404A30F040085072310F4043A
:1038380083470414639E07102285EFD0DFC221AAB4
:1038480003278900BA977DBF83278900BE94F1B703
:1038580083270A008297032784086366E50A198D7F
:103868007E3C0357C9008E07B387E702130700326F
:1038780093870719B3D7E70263ECA708B74A0F0085
:10388800138BFA23938A0A24835704048507231089
:10389800F4048347041481E72285EFD0DFBC228536
:1038A800975005E0E78020156317052403260409CF
:1038B8000327C408832689003297BA876364C70040
:1038C8006364D700B307D740783C0356C900232860
:1038D800F408050778BC035764083307C7025A97EA
:1038E80033575703B384E74063F5E700998EB384F1
:1038F800F60083270A00829763E6A4043385A44070
:10390800E34405F839BF83278900998F3E9589BF1D
:10391800A1452285975005E0E7800006A305A4028B
:103928009717000083A7879D6387071C6244F240AE
:10393800D2444249B249224A924A024B8945154526
:103948000561828783278900A6973385A7404DBFE5
:103958002285EFD09FBB2285975005E0E780A0091C
:10396800631B05180355C90083576408B7460F0041
:103978001386F623B387A702938606240327040930
:10398800230B0402832A8900B297B3D7D702636E48
:10399800F716B307F7408326C4082324F408014B1D
:1039A800B387E600BE8463E4D70063E45701B384B9
:1039B80057411E3023289408A1CB835604045A305B
:1039C80037460F0056B03387E640B387E7023A30F0
:1039D8001306062481468145BA97B3C7070833857D
:1039E800A7023EB097A006E0E78080E511CD2695B6
:1039F800B3349500A695AA876314BB006364550188
:103A0800B30755412328F40883270A008297AA841C
:103A180083270A008297E30D95FE83270A008324F3
:103A28008408829763E8A40E3385A44063010510D7
:103A3800035AC90083576408B7440F001387F42357
:103A4800B387470393840424BA97B3D79702171709
:103A5800000003473789BA9763EBA70CB335950283
:103A6800835A2402528681463305950297A006E0C0
:103A7800E78000DD3389AA0033854A0337460F0003
:103A8800130606248146814597A006E0E78040DBBF
:103A980015C1B337950252868146B385B402338582
:103AA800A402BE9597A006E0E78080D9B38AAA4011
:103AB800231154033545652623AE890838348547D4
:103AC800631EF704930700FD7CA4814517050000D9
:103AD8000325C571EFC05FFD954717170000232127
:103AE800F7DA370710009707000083A7A77198C770
:103AF800060923A82707F2406244D2444249B24942
:103B0800224A924A024B05618280B3065701B38765
:103B1800F64051B583278900BE9439B7930710FC46
:103B28007CA48145170500000325C56B65B7971769
:103B3800000023AF07B8834709019DC3170500009C
:103B480003254569EFD00F9A624483274900F24064
:103B5800D2444249B249224A924A024B05618287BD
:103B6800834594026244F240D2444249B249224A0F
:103B7800924A024B01450561B315B028B3C5050843
:103B88006FF02F8E011122CC26CA4EC606CE4AC827
:103B980052C456C25AC038358547832405092A8439
:103BA800AE896314F70C83570508835AC503170AAF
:103BB8000000130AAA76035BCA0063FE571914298A
:103BC800639BE61803278511631707180327450A1F
:103BD8006313071874351D47639FE6162A3DB38A99
:103BE800FA409307204E3305550303294409374605
:103BF8000F001306062481463305F50297070000D7
:103C080083C7476E33592503B335AB023E99334911
:103C18000908231324093305AB0297A006E0E780BF
:103C280020C2B307950033B5A7002E9503278A0055
:103C3800BE8419E163E4E700B384E740B30769038E
:103C480037470F009306F7231307072423A099008B
:103C5800B697B3D7E702D69763E4F4009D8C31A0FA
:103C680003278A00B307F740BE9417090000130919
:103C7800A9478327090023A09900829763E2A4102B
:103C88003385A440635D050A83270900170B0000EC
:103C9800130BCB68829703A709006369E50E198D9A
:103CA8007E3C0357CB008E07B387E7021307003229
:103CB80093870719B3D7E70263EFA70C374A0F00BA
:103CC800930AFA23130A0A24835704048507231046
:103CD800F4048347041481E72285EFD0CFF82285C6
:103CE800975005E0E78020D161E583260409832702
:103CF800C40803278B00B697BE8463E4D70063E447
:103D0800E700B384E7407C3C8356CB002328940823
:103D180085077CBC83576408B387D702D697B3D787
:103D2800470363E6F40A9D8C8327090023A09900C2
:103D3800829763E1A40A3385A440E34705F897070F
:103D4800000083C7375A63E6A7069717000023A128
:103D580087980145B9A88357640837470F00930629
:103D6800F723B387670313070724B697B3D7E70288
:103D7800E3F6F4EE03278A002697B304F740F5B577
:103D88009707000083A7075ABE94DDBD83278B00E1
:103D9800998F3E9531B7A1452285975005E0E78078
:103DA800A0BDA305A4029707000083A7275581EFAC
:103DB8007D55F2406244D2444249B249224A924A6D
:103DC800024B05618280894515458297D5B71D8FBD
:103DD800BA9499BF83278B00BE94B1BF97060000A1
:103DE800938646429C42B84B1377F78FB8CB9843DB
:103DF8001367870098C39C4393D7374889C7010046
:103E0800010001000100170700000327E73E1C43DB
:103E180093F7F7CF93E707101CC317060000032694
:103E2800663F1C463707CEFF7D17F98F1CC69C429C
:103E380037070300B8CB9707000083A7273C99CB27
:103E4800D44390479842518F98C2944BDC4B984288
:103E5800D98F9CC29717000023A407A282809707D6
:103E6800000083A7273A9C438D8BF9C74111B7E718
:103E780000E04AC003A9070026C23707200006C68B
:103E880022C4AA843379E90023A0E7180F100000A0
:103E9800171400001304049D584C8D47631AF7004B
:103EA8009707000083A7C775014681454545829756
:103EB80019476393E4048347140289CB83470402B8
:103EC8006396970097170000A38E079A584CA1474E
:103ED8006315F700930780101EB097070000238131
:103EE8000720ED3DB2402244B7E700E023A02711A8
:103EF80092440249410182809D47639BF4008347B5
:103F08001402E9D7034704028D47E311F7FC5DBFAC
:103F1800544C6389E600584C6306F700584CA14797
:103F2800E31DF7FA83471402CDFB5C4C2300F4022F
:103F38008547A300F40255B78280411122C42A8420
:103F4800354506C6293F49CCAD4763E987067D1448
:103F58001374F40F9707000083A7C72B984BB70675
:103F680000C1FD161374F403758F6204418F98CB5A
:103F7800984B9706000083C6A636717693F6F6032B
:103F88001306F60FA206718F558F98CBF84FB70618
:103F9800F9FFFD1613674700F8CF984B0145758F59
:103FA8001317172998CB370702001307874F98C7AD
:103FB800B147171700002325F78C39A8B1476304C8
:103FC800F4029307600263E48700791451B79307FA
:103FD80070024945E300F4F8B2402244410182806E
:0C3FE8001304500285BF13046002ADB743
:103FF4002A8309CA83830500230073007D16050301
:1040040085056DFA82809707FC1F83A7E7E11707F0
:10401400FC1F0327E7E001456313F7008280F623C2
:1040240099E2D62336959C43C5BF1707FC1F130797
:1040340027FF1C435A23411193860711E117BA97AE
:1040440085651706FC1F2321D6DE1706FC1F2329CE
:10405400F6DC06C69D051356370063F4E500130627
:1040640000203387C6009705FC1F23ADE5DA6116EF
:1040740098C2D2A2239306001CC3998FE1175EA3B2
:10408400231307004937B2409707FC1F2399A7F66B
:10409400410182809707FC1F83A707D91707FC1FDC
:1040A400032707D801456313F7008280F62381E6CE
:1040B400D6233375D50A9C43FDB7184183A785FFE2
:1040C4006319B7001CC1FD5723AC05FE238FF5FE11
:1040D4008280232CF6FEC5BF411122C437E400E0E0
:1040E40026C204403707200006C6F98C2320E418B2
:1040F4000F10000009E9232094101545B240224412
:104104009244410182800347E5FF9307F00F630661
:10411400F700232094101145D5B797C0FB1FE78003
:10412400C000014523209410D1BF41114AC037E992
:1041340000E022C403240900B707200006C626C2F3
:104144007D8C2320F9180F10000089E523208910A5
:10415400154515A0AA849707FC1F83C7F7E92E8588
:1041640063F5F400894763EE9700BD37B7E700E0D5
:1041740023A087100D45B2402244924402494101D4
:10418400828083A785FF99E703C7E5FF9307F00FB4
:104194006308F7009137B7E700E023A087104DBF0D
:1041A400238F95FE1705FC1F130545C897C0FB1FF9
:1041B400E780A008A165268597E0FB1FE780E07FE4
:1041C40001452320891045BF9707FC1F23A007C67C
:1041D40082804111B7E700E026C2844337072000FC
:1041E40006C622C4F98C23A0E7180F100000970715
:1041F400FC1F83A7E7E41704FC1F130464BA91C7E8
:1042040082971C40AA971CC031A09707FC1F83A764
:10421400E7C2FDF70840B74703009387D73F33054C
:10422400F502B7A72600938737ECB2403E9508C045
:104234002244B7E700E023A0971092444101828012
:10424400411122C406C69707FC1F83A7E7BE1704C3
:10425400FC1F130464DA89C782975C48AA975CC878
:104264004848B240224441018280B7E700E09843C5
:10427400B706200023A0D718758F0F1000009706EB
:10428400FC1F83C676D76370D5029706FC1F83A6EE
:10429400A6BB3325D5201621B3F5B6400EA123A025
:1042A400E7100145828023A0E7100D4582807971D3
:1042B400B7E700E026D284433707200006D622D48D
:1042C4004AD04ECE52CCF98C23A0E7180F10000030
:1042D400930705FF93F7F70F7D476363F70A3147A9
:1042E4003307E5029707FC1F83A747B6BA979C4399
:1042F400C1CB135445003D893315A028AE89B3457D
:10430400050822852EC697E0FB1FE780E0492A892D
:1043140039C9B2452285170AFC1F130A6AD5B13779
:104324009707FC1F83A787B182978357CA002A8403
:1043340081463387370313060064B3B73703130585
:104344000732B335E500BE95EF908224B3078500AC
:1043540083268A003E8763E4A70063E4D70033879B
:10436400D7402324E900B7E700E023A097100145D4
:10437400B250225492540259F249624A45618280F1
:10438400B7E700E023A097100945DDB7797122D47F
:1043940037E400E04AD003290400B707200006D61A
:1043A40026D24ECE52CC56CA5AC85EC63379F900CC
:1043B4002320F4180F1000009707FC1F83C7D7C3EE
:1043C4006378F500970BFC1F83AB4BA763970B0037
:1043D400B7E700E023A0271199A0970AFC1F938A4E
:1043E4002AC903AB8A00B74736FE938707C83E9BAA
:1043F40083D7CA002E8AAA84B385C702B2898146AC
:10440400B3B7C70213850532B335B500130600648C
:10441400BE95EF90E2176370AB022320241101458F
:10442400B250225492540259F249624AD24A424B3F
:10443400B24B45618280829B83D7CA002A841306CB
:104444000064B38537038146B3B737031385053258
:10445400B335B500BE95EF90A213B307850003A74B
:104464008A003E8463E4A70063E4E7003384E74002
:10447400D285268597E0FB1FE780003301C900C57C
:10448400B7E700E023A02711054559BF93E504F0E1
:104494004145B3C5050897C0FB1FE780E0BB11E9A0
:1044A4009707FC1F83A7C7BA85D7A68511458297AE
:1044B40005B71707FC1F1307E7981C4389EF08C3C8
:1044C40085472326050000C52311450104A11CB11D
:1044D4002322050075B73E87DC47F5FF48C7CDB7F3
:1044E4007971B7E700E026D284433707200006D667
:1044F40022D44AD04ECE52CC56CA5AC85EC662C4E2
:1045040066C2F98C23A0E7180F10000035C12A8970
:104514002E8AB28AB6894144B14C170BFC1F130B87
:10452400EB92130C0003B30B940383270B00DE9769
:104534009C43B9EF135544409375F40056861375A4
:10454400F50FB315B028B3C50508893531C18327E4
:104554000B00DE9723A0270123A2470163840900EF
:1045640023808900B7E700E023A09710014521A02C
:1045740023A097100945B250225492540259F2498B
:10458400624AD24A424BB24B224C924C45618280E1
:104594000504E31A84F9B7E700E023A09710214546
:1045A400D9BF011122CC37E400E026CA04404AC82E
:1045B4004EC652C406CEB70720002A892E8AB28975
:1045C400FD8C2320F4180F100000C933D2854A85CE
:1045D40097E0FB1FE780401D01ED23209410214547
:1045E400F2406244D2444249B249224A056182807F
:1045F4009707FC1F83D787A8B38537032A89130637
:1046040000648146B3B7370313850532B335B5006B
:10461400BE95EF80F2772322A90023209410014550
:10462400C1B7011126CAB7E400E04AC803A90400CF
:1046340022CC4EC6B707200006CE52C4AA892E84C7
:104644003379F90023A0F4180F10000097E0FB1F42
:10465400E7808015170AFC1F130A0A9A1DE1A28538
:104664004E85213183470A006382370523A0241134
:104674001945F2406244D2444249B249224A056192
:10468400828023110500A2854E85C53683470A0022
:104694006386370123A024110145E1BF17F7FB1FEF
:1046A400130767791E23C18F1EA3EDB797F7FB1F6E
:1046B400938767789A23598C82A34DBF01114AC806
:1046C40037E900E022CC03240900B707200006CE16
:1046D40026CA4EC67D8C2320F9180F1000009307BC
:1046E400F00263E7A704B144B304950297F9FB1FF2
:1046F4009389C97583A70900A6979C4395CB9375A5
:10470400F5001181B315B028B3C50508193F83A777
:1047140009000145A69723A0070023A20700232030
:104724008910F2406244D2444249B2490561828010
:10473400B7E700E023A087100945E5B74111B7E7C3
:1047440000E026C2844306C622C437072000F98C41
:1047540023A0E7180F10000097E0FB1FE780C004B8
:1047640019E90145B2402244B7E700E023A09710BD
:10477400924441018280004597F7FB1F83A7076C91
:1047840082979707FC1F9387A78E6367A4029847B5
:10479400B74636FE938606C83305A4403697E372BF
:1047A400E5FC13070064B335E502D22781463305DF
:1047B400E502EF80F25D7DB798473A94C9BF411195
:1047C40006C697F7FB1F23A9A7660295B240970771
:1047D400FC1F23AFA782014541018280411151464C
:1047E40081451705FC1F1305658706C622C426C22A
:1047F40097F7FB1F23A8076497F7FB1F23AE0762F5
:1048040097F7FB1F23AC076297F7FB1F238407620C
:1048140097F7FB1F23AE076097C0FB1FE780C0B963
:1048240013068002814517F5FB1F1305E57C97C02D
:10483400FB1FE78060B8EFF04FFF97F7FB1F9387EC
:10484400277EE82BFC3B17F4FB1F1304E47A854511
:104854003E958D473305F502994797F4FB1F9384E2
:10486400E45E39051375F50F28A03305F502130529
:1048740005243345050897B0FB1FE780E07D88C019
:1048840035C93020994781453306F60213060624BC
:1048940097C0FB1FE78040B29C40382097F4FB1F71
:1048A4009384045A938707249CC0B347F72017F7CF
:1048B400FB1F232BF758093A25211C30944017E697
:1048C400FB1F1306A6F633C7D72010C313871700A0
:1048D4001377F70F17E6FB1F1306E6EE3347D720CF
:1048E40010C313873700890718B093F7F70FB3C7BE
:1048F400D72090C3B240224492444101828097F66B
:10490400FB1F9386666F2A87BC228832637DF5007D
:104914001306150097F7FB1F83A7875290B2B3477E
:10492400F52098C382801305F00F82801C41E5CBEB
:10493400370700F07D8FB706002089476312D70E32
:104944005A21411122C406C62A8469C7194693050F
:10495400F00F690597C0FB1FE78020B905478D4715
:10496400630AE50A1C4491C75858994745C7185C1F
:1049740055C31306C003814517F5FB1F1305456A8C
:1049840097C0FB1FE78040A31306C003A28517F559
:10499400FB1F1305E56897C0FB1FE780609B97F733
:1049A400FB1F9387E767DA2701E713070010DAA7ED
:1049B400F82719E30547F8A79A2B19E36D479AAB33
:1049C400F83719E31547F8B7B82B19E30547B8AB1F
:1049D400B83B19E3F837B8BBD83B11C79376370017
:1049E4000983F4ABF8BBD82B19E35547D8AB182C83
:1049F40001E71307C00398AF9C5791C7829797F7B5
:104A0400FB1F239FA75EFD5717F7FB1F2304F75EC9
:104A1400F1338147B24022443E8541018280894777
:104A24003E85828079714ECE97F9FB1F9389496444
:104A340083A7090006D622D426D24AD052CC829724
:104A440013090064B335250303D6C900814617FA58
:104A5400FB1F130A6A5A32C633052503EF8052330B
:104A640083248A012A8401456386840232463305FD
:104A7400944063EF840003A589008146B335A902FD
:104A84003305A902EF80D230B30795403385870000
:104A9400232C8A00B250225492540259F249624A99
:104AA40045618280011122CC0A852E844146979566
:104AB40002009385E5E706CEEFF08FD31808332480
:104AC400E420035704FFF240624497F7FB1F83D7A7
:104AD400075B37450F00BA97130505243355F502D4
:104AE4000561828097F7FB1F83D7675951471D459E
:104AF400637CF702794719456378F70213072003AB
:104B040015456373F7021307B0041145637EF7007C
:104B1400130740060D456379F7001307600909453B
:104B24006374F70013B5B70F8280411122C426C203
:104B34002E84AA8406C6058CEFF0AFE9B327A4023D
:104B4400B2402244338597001375F50F9244410116
:104B54008280411122C426C22E84AA8406C6058CF2
:104B6400EFF02FE7B327A402B24022443385970025
:104B740033450508924441018280411122C426C272
:104B84002E84AA8406C6058CEFF0AFE43335A40264
:104B9400B2402244269592444101828041114AC088
:104BA40017F9FB1F1309C9478327890206C622C4C4
:104BB40026C28DCF829797F4FB1F9384E4439E24EF
:104BC4002A848DC733F7A70A33470708B3D7A70A40
:104BD400B3C70708B307F74051476359F700832762
:104BE400C90291C38297EF10A23E82A4B24022442C
:104BF4009244024941018280011122CC97F7FB1FA4
:104C040023A8072417F4FB1F130484415C5406CE25
:104C1400AA8581C72AC68297B245D1C59C4105455C
:104C2400BDCF9C45ADCFDE25BDCBFE25ADCB9C29AC
:104C340081CB7C287838BA976343F506DC41A5C359
:104C44001306400217F5FB1F1305854297B0FB1F9F
:104C5400E780007097F7FB1F93878741984397F687
:104C6400FB1F23ADE61C183C19EFCA279307805796
:104C740037460F003305F5021306062481468145A5
:104C8400EF80121108BC183C9D4763E4E700A1477C
:104C94001CBC17050000130525D915360145F24043
:104CA40062440561828097F7FB1F23A5073697F7B7
:104CB400FB1F9387E73B17C7FB1F130707D498C352
:104CC40037873200FD56130727A194C7D8C797F733
:104CD400FB1F2387073AB7C7004023A4D7269DBFED
:104CE400011122CC17F4FB1F13048433084406CEAD
:104CF40026CA4AC801E90545F2406244D244424901
:104D0400056182805C58E5DB185C75D770008545C9
:104D140082971844B247E300F7FE4A249305E0045F
:104D240017F9FB1F1309492D97B0FB1FE780C03209
:104D34002320A90269D152249305F00F814497B02E
:104D4400FB1FE78060677C240326090263C1F40229
:104D5400328597B0FB1FE780403D014597F7FB1F65
:104D640023AC072A97F7FB1F23AA072A71B74E24FF
:104D74001844B3879502898185043385E7001C5C58
:104D840008C28297C9B7011122CC17F4FB1F130480
:104D940024291C4426CA4EC656C206CE4AC852C44A
:104DA4005AC0AA84AE89B28A6388071A585839CB84
:104DB4001307F01F6366A71017FAFB1F130ACA2311
:104DC40003290A02631209044A249565938515E0B0
:104DD40097B0FB1FE78040282320AA022A861DC122
:104DE4004E245C580844898182971C4403290A0292
:104DF4002322FA028947639EF402C1479305090CF2
:104E04006381F9042945BDA003274A02E384E7FE30
:104E14004A249565938525E097B0FB1FE780C0235E
:104E24002A896DD14E242A865C5808448981829748
:104E3400D1B78D47639AF404C1479305490DE393B1
:104E4400F9FCB8219307A0056312F7069E21639F1E
:104E540097044E869105568597B0FB1FE780404F17
:104E640083270A02638727014A8597B0FB1FE780DF
:104E7400C02B0145F2406244D2444249B249224A1D
:104E8400924A024B0561828091476397F40093052F
:104E9400890EE39999F675B793070010E394F4F635
:104EA400A147E3E137F79305090F61BF83270A029E
:104EB400E38A27F54A8597B0FB1FE780002799B757
:104EC4001D67637FE506130705E099463347D7025C
:104ED400562417FBFB1F130B2B123307D702330A7D
:104EE400F70083274B026396470103290B026311E2
:104EF40009024A249305E00497B0FB1FE780C0151C
:104F04002A8909D14E245C582A8689815285829740
:104F140091451307A00593F5C50FB307B900B42352
:104F24006399E60296236394960291054E86CA9588
:104F3400568597B0FB1FE780A04183270B021DB75E
:104F4400A166F916E3E0A6EC3307E54051B7AC33AC
:104F5400D9B783270B02A9BF97F5FB1F83A5C50B00
:104F6400E38205EA91479306A00593F7C70F3387B9
:104F7400F5003023E318D6E81223631B960091074B
:104F84004E86BE95568597B0FB1FE780603CD5B52D
:104F94003C33E1BF97F7FB1F93878708984721C7E6
:104FA400985F31C385466310D504411122C417F4B8
:104FB400FB1F13046404105006C615C2CE274850C4
:104FC40089810297085097B0FB1FE780001697F776
:104FD400FB1F23A3070497F7FB1F23A10704B24079
:104FE400224441018280828001114AC817F9FB1FC3
:104FF400130909034EC68329890022CC26CA52C448
:1050040006CE56C2AA842E84328A638D091A832757
:10501400890399EB2945F2406244D2444249B2499A
:10502400224A924A0561828083274903E5D7930780
:10503400F01F63E0A70C97F9FB1F9389E9FB83A793
:10504400090295CF0325890083A749026395A70424
:105054008947639FF404C147E31EF4FA03A50902D8
:105064001305050C9307A0053CA106A12286D28551
:10507400110597B0FB1FE780A02D014569BF0355BB
:10508400C9009305E00497B0FB1FE780E0FC23A070
:10509400A9024DF941B78355C9008327490303A6E3
:1050A4000902898182978327890023A2F9024DB7D7
:1050B4008D47639AF400C147E31EF4F403A5090283
:1050C4001305450D45B791476399F400E31494F42F
:1050D40003A509021305850E71B793070010E39B1E
:1050E400F4F2A147E3E887F203A509021305050FCB
:1050F40095BF9D676373F506930705E01947B3C72A
:10510400E7020357C90097FAFB1F938AEAEEB387B5
:10511400E702BE9983A70A02A1CB83A74A0263913F
:10512400370703A50A0291479305A0051308F00F5A
:1051340013F7C70FB306E500B0226313B60683D88E
:105144000600B032639C9804B307F64063C6870434
:1051540011072286D2853A9529BF21677917E36B17
:10516400A7EAB307F54071BF0355C9009305E004EE
:1051740097B0FB1FE78040EE23A0AA0259FD59BD5A
:105184008355C9008327490303A60A0289814E85F2
:10519400829723A23A0371B723900601B28749BFCD
:1051A4003386870011061308F00B6374C8002D457D
:1051B4009DB5ACA213063400719A1106B29786A26B
:1051C400BCB279B797F9FB1F938909E383A7090256
:1051D4009DCB03A5090291471308A0059305F00F81
:1051E40013F7C70FB306E500B0226310060583D892
:1051F4000600B03263979800B307F640E3DA87F409
:105204008EA2B287F1BF8347E9000355C900930515
:10521400E0043305F5023345050897B0FB1FE7802A
:10522400A0E323A0A90255F5F5B30356C9008345AD
:10523400E900B385C502338687001106E3E9C5F6A4
:105244002381060185BF014582809C211CA1BE21CA
:105254001CB1BE21A1833CA1DC213CB1114582805B
:1052640097F7FB1F23AA07BE97F7FB1F23A407BECC
:1052740082800DCD411122C426C206C6AA842E8482
:10528400014585C122854146978502009385456D78
:1052940097B0FB1FE780C00B9C2005455CA49C30A5
:1052A4005CB4B24022449244410182800145828030
:1052B400011122CC26CA06CE8947AA843284639E71
:1052C400F5006383B602414781476395E6048A8506
:1052D4004D3741468A8522850DA841476392E504EE
:1052E400638FF600639EB6022E86A2856244F24066
:1052F4002685D244056117B3FB1F6700E3168A8530
:105304003285853F41468A85268597B0FB1FE78015
:10531400A015AA87F2406244D2443E85056182808A
:105324008147CDBF97F7FB1F23A6A7B2828097F7CB
:10533400FB1F23A3A7B28280011122CC622106CED7
:1053440026CA4AC84EC63DC8832985002A88AE8429
:1053540003C9090081471317496063550702B14720
:10536400054563F6870403552800511433440408A3
:105374004E8633878900A2868545EFB0D003B337C4
:10538400A0008507135569487D141379F903334444
:1053940004089CA088B023812401C2A0014719C03D
:1053A4001387190098C409476383E7000145F24055
:1053B4006244D2444249B249056182800545C5BF71
:1053C400C167F917630AF502D94763F7B7020111F8
:1053D40022CC2EC606CE2A84EF90C007B24563685D
:1053E400B50022856244F24005616FA0A07CF240C2
:1053F400624405450561828005458280C167F917CD
:105404006314F5006F900005411106C6EFA02069F2
:1054140011E15D45B240410182809147639DF500F1
:105424001C211CA23C211831A207D98F3EA23C3179
:1054340001455CA28280114582804111814522C4CC
:1054440026C206C6AA849D232A8409E997F7FB1F6E
:1054540083A747A081C7F94526858297B240228554
:10546400224492444101828039714ED652D45AD09A
:105474005ECE06DE22DC26DA4AD856D22A8A2E8B63
:10548400B289B68B0DE79D3F9145EF90C00A2A84FF
:105494004D49854A19EDF2506254D254B259225AF8
:1054A400925A025BF24B4A854259216182803A84C6
:1054B400814A230034018544630A0B00DE85130509
:1054C4001400029B93041500B3C404089399496023
:1054D40063D30902C1455285EFA0A06A654915E569
:1054E40033069400A6852285EFB000322A8911ED97
:1054F400B104B3C4040891472C0052857C8422C6AD
:105504006485EF90D07F2A8959D5E3860AF82285ED
:1055140097B0FB1FE78060C1BDBF011122CC26CA32
:105524004AC84EC606CE2A893284B689353FAA8433
:105534000DE197F7FB1F83A7279281CF05476317D8
:10554400E40003C4090005041374F40FA2854A851A
:105554008297F24062444249B2492685D2440561A9
:105564008280AE860147054697050000938525CEC7
:105574006DB79E211CA19E21A1831CB10945828087
:105584009E211CA19E21A1831CB1BE213CA1BE2150
:10559400A1833CB1114582809E211CA19E21A1833F
:1055A4001CB1BE213CA1BE21A1833CB1DC315CA174
:1055B400FC215CB18A2519053345050882809E21AA
:1055C4001CA19E21A1831CB1094582809E211CA19E
:1055D4009E21A1831CB1BE213CA1BE21A1833CB16B
:1055E40011458280CA2106053345050882809E2123
:1055F4001CA19E21A1831CB1AA21090533450508DC
:1056040082809E211CA19E21A1831CB1BE213CA1AC
:10561400BE21A1833CB1CA2111053345050882800E
:105624009C211CA1054582809E21411122C406C6ED
:105634001CA19E212E841105A183A30EF5FEBE217B
:105644009505230FF5FE83D7D5FFA183A30FF5FEA0
:1056540003C6F5FF97B0FB1FE78080CF4820B24018
:10566400224411054101828089476399F5001C3168
:1056740018210145A207D98F1EA28280114582807C
:105684009A21011106CE22CC2EC6D94763F4E70233
:105694002A84EF80305CB2469E22636DF500228539
:1056A4006244F24001470946970500009385A5EC42
:1056B40005615DBBF2406244094505618280AA87A9
:1056C400A9C11421FD150547B3C505086398E60073
:1056D40013D725008D89114589CD8280094711454D
:1056E4006392E602494533D7A502B3F5A5021145F5
:1056F40091E9114501CB850734A21AA25CC2014588
:10570400828011458280AE860147114697050000CC
:10571400938545E791BB13F73500AA8701EB89818F
:10572400114591C50EA25CC201458280114582805B
:10573400D8218947631BF702011122CC2A84C8456A
:1057440006CEAE8601C92EC69D4597B0FB1FE780E5
:1057540040ABB2462A8722856244F2401946970537
:1057640000009385A5E3056101B30945828099E1B1
:10577400114582801C2105473EA2E37BF7FEFD15FF
:1057840093F5F50F33D7F502B387E702E392F5FEFD
:10579400050548C21AA201458280DC210947AE866C
:1057A4006385E70041476399E70001472146970570
:1057B40000009385A5E74DB9094582800EA291E1C9
:1057C400014548C201458280AE86014729469705B6
:1057D4000000938505DF49B90EA291E1014548C255
:1057E40001458280AE8601473146970500009385C6
:1057F40025DE9DB90EA291E1014548C20145828092
:10580400DA21854763FFE702011122CC2A8488410B
:1058140006CE2EC615C1854597B0FB1FE780609E56
:105824002A8722856244B246F24039469705000031
:10583400938585DB05610DB9F24062440945056134
:10584400828009458280AA878DC518218D4611451D
:1058540063F2E602FD15B3C50508B3C6E5023308D5
:10586400D70263990501850716A23AA25CC20145D5
:10587400828011458280DC210947AE866385E7007A
:1058840041476399E7000147414697050000938526
:10589400E5D9D9BE094582803335B0000A05828036
:1058A400011122CC26CA06CE98258547AA842E84C7
:1058B4004946631FF70099363E204915130620090F
:1058C40063C8A700F2406244D2440945056182805E
:1058D400183485476314F70013660604484001C969
:1058E4008D4532C697B0FB1FE780A0913246A28651
:1058F4006244F2402A872685D244970500009385A6
:1059040045CF056195B68D4763F7B7021C31182161
:10591400F115A207D98F1EA23C313821B3C5050861
:10592400A207D98F014799C1130745003EA24EA291
:1059340018C60145828011458280011122CC2A8437
:10594400884506CEAE8601C92EC6954597B0FB1F85
:10595400E780208BB2462A8722856244F24059466A
:1059640097050000938525CA0561FDBC3335B00059
:105974000A058280AE86014761469705000093853B
:1059840065CADDB48547114563F1D7021C320C2288
:105994000945A207CD8F81456384A600930526009F
:1059A400F9161EA336A34CC30145828001478146E4
:1059B4007946814555BC9E211CA19E21A1831CB121
:1059C40009458280BC2105471CA18A216397E70011
:1059D4000A050505334505088280C9473305F502E4
:1059E400CDBF8A210A05334505088280BE211CA14A
:1059F4008A21BE213305F502050533450508828059
:105A04008A2182808A2182808A218280BE211CA1EF
:105A14008A21BE213305F502050533450508828038
:105A24009E211CA19E21A1831CB1BE213CA1BE21AB
:105A3400A1833CB1CA2111053345050882809E210A
:105A44001CA19E21A1831CB1AA2109053345050887
:105A54008280894711456398F6001C32142201455F
:105A6400A207D58F1EA382809A21D947AE8663F9F7
:105A7400E70001470D4697050000938505F471BCC6
:105A8400094582801145639DA6001C3214220145FC
:105A9400A207D58F1EA33C323422A207D58F3EA382
:105AA4008280BC210547FD1793F7F70F6361F70464
:105AB4009E2195CF011122CC2A84C84106CE2EC640
:105AC40015C1894597A0FB1FE780A0732A8722850B
:105AD4006244B246F2401546970500009385C5EE30
:105AE400056125BCF240624409450561828009458F
:105AF4008280954763F0D706411122C426C24AC06A
:105B040006C61C323A841822A207B284D98F1EA07A
:105B14003C32382293854400A207D98F3EA089479E
:105B24005CA0094613055400368997B0FB1FE78033
:105B34002082194781476304E90093876400691947
:105B440023142401B2405CC4224492440249014516
:105B540041018280114582809E2195CF011122CC82
:105B64002A84C84106CE2EC615C1854597A0FB1FC1
:105B7400E78020692A8722856244B246F2401D46A6
:105B840097050000938525E6056141BAF240624419
:105B9400094505618280094582809947B2856388F9
:105BA400F600D147114541466384F60082800946D8
:105BB400411106C650A39C31942113055700A20736
:105BC400D58F1EA3BC31B4219105A207D58F3EA366
:105BD40097A0FB1FE780C077B24001454101828056
:105BE4009E219DCF011122CC2A84C84106CE2EC607
:105BF4001DC1894597A0FB1FE780A0602A872285E5
:105C04006244B246F240254697050000938545DE7E
:105C140005616FF09F90F2406244094505618280FE
:105C240009458280894711456398F6001C32142285
:105C34000145A207D58F1EA38280011122CC2A849C
:105C4400C84106CEAE8601C92EC6854597A0FB1F66
:105C5400E780205BB2462A8722856244F2402D46C3
:105C640097050000938505DA05616FF01F8B19BD58
:105C7400011122CC2A84C84106CEAE8601C92EC6A3
:105C8400854597A0FB1FE780C057B2462A87228527
:105C94006244F2403546970500009385E5D60561D8
:105CA4006FF0BF8793F71600114581EB8947638630
:105CB400F600858256A310C301458280011122CCCF
:105CC4002A84C84106CE2EC61DC1854597A0FB1F58
:105CD400E78020532A8722856244B246F2403D463B
:105CE40097050000938585D205616FF01F83F2400C
:105CF40062440945056182809E219DCF011122CC19
:105D04002A84C84106CE2EC61DC1894597A0FB1F13
:105D1400E780204F2A8722856244B246F2404546F6
:105D2400970500009385C5CE05616FF00FFFF24023
:105D3400624409450561828009458280854763F490
:105D4400D70208A70CB71C320C220945A207CD8F35
:105D540081456384A60093052600F9161EA336A385
:105D64004CC30145828011458280014781464D46DE
:105D740081456FF08FFA8D47114563F5D7021C32C8
:105D84000C22A207CD8F1EA33C322C22A207CD8F5A
:105D940081456384A60093054600F1163EA356A3ED
:105DA4000CC701458280011122CC2A84884506CE85
:105DB400AE8601C92EC6954597A0FB1FE7806044B7
:105DC400B2462A8722856244F2405D469705000068
:105DD400938545C505616FF04FF48547114563957B
:105DE400F6001C2201451CA38280014781466546BA
:105DF40081456FF08FF2011122CC2A84C84106CE6E
:105E0400AE8601C92EC68D4597A0FB1FE780603F73
:105E1400B2462A8722856244F2406D469705000007
:105E2400938525C205616FF02FE4011122CC2A84E9
:105E3400C84106CEAE8601C92EC68D4597A0FB1F6C
:105E4400E780203CB2462A8722856244F2407546A8
:105E5400970500009385E5BE05616FF0EFE0011141
:105E640006CE2EC6EF90D03F19C5B245F2402A2186
:105E740005616FE0C004F24049450561828097E7FF
:105E8400FB1FA381070097E7FB1F238D07FE97E7FE
:105E9400FB1F23A707FE97E7FB1F23A107FE97E736
:105EA400FB1F23AB07FC97E7FB1F23A507FC97E722
:105EB400FB1F23A707FA97E7FB1F23A107FA97E71E
:105EC400FB1F9387271D3706840390D33707B4003D
:105ED40037C6070098C3130606B83747A000D8C3CF
:105EE400D0D33707100041669306070AB705500060
:105EF4009308060194C723A4170393860501930806
:105F040016F8D4C723A61703B706D007B7087F002F
:105F14001308070513850601410723A81703B0C317
:105F2400930816009386060513861500D8CBF8C38C
:105F340023A8070188CF23AE070023AA170323ACA5
:105F4400070223AE070223A40704F0C7B4CB23AA95
:105F54000704ACCF23AE0705B8D33707A000F8D7A2
:105F64001307000AB8DB1307C01CF8DB370714005B
:105F7400B8DF0547F8DFE8D323A40706930710F832
:105F840017E7FB1F2328F7188280011152C42A8ABD
:105F9400214522CC26CA4AC84EC606CE2E84B289D2
:105FA4003689BA8497A0FB1FE780C02A05C99307E6
:105FB40000FD1CA19947A30045013CA12303250131
:105FC40064B123123501AA8522856244F240D24489
:105FD4004249B249224A05616FE02F95F24062447A
:105FE400D2444249B249224A0561828097E7FB1FA5
:105FF40023A8A7E8828097E7FB1F23A1A7E8828054
:1060040097E7FB1F23AAA7E6828097E7FB1F23A33A
:10601400A7E68280011122CC26CA4AC806CE4EC603
:106024002A89AE840144B309890063699400F2406B
:106034006244D2444249B24905618280EFE06F99DB
:10604400B3470508A1832380F9009307140093F74D
:10605400F70F850963F89700CA97090488A3137496
:10606400F40FD1B73E84D1B7411122C417E4FB1F0A
:106074001304840A6A20C16706C6FD17630EF5007F
:1060840017E6FB1F0346462B97E5FB1F938585DD2B
:10609400EF90007EFD577EA0B240224441018280F1
:1060A40009C925151375F50F1335850E134515000C
:1060B40082800145828023900500C9C2797122D46F
:1060C40026D252CC56CA5AC806D64AD04ECE5EC63E
:1060D4002A8B2E8AB28A3684814463FF5405B3071F
:1060E400940083C9070013891400334909086385A0
:1060F4000904B387290163C1FA04B307240183CBDC
:1061040007005E85713F0DC99387F9FF2310FA00DC
:1061140063906B03050933052401B2502254925451
:106124000259F249624AD24A424BB24B45618280DB
:10613400CE94B3C4040855B70145C5B70145828060
:10614400011122CC26CA4AC84EC606CE97E4FB1FCC
:10615400938484FC2E89D0C88CC8C8C42A84414640
:106164009305F00F4A8597A0FB1FE7800038854907
:10617400631935038848C145713D41469305F00FC5
:10618400228597A0FB1FE780403605496315250348
:106194006244C844F240D2444249B249C14505610F
:1061A40095BD414681454A8597A0FB1FE780E033B2
:1061B400E31535FDC1B741468145228597A0FB1FF4
:1061C400E780A032E30625FDF2406244D24442490E
:1061D400B24905618280411122C426C22E84AA8458
:1061E40013060002814517E5FB1F1305E5F206C6F9
:1061F4004AC097A0FB1FE780201C17E9FB1F130967
:10620400A9F197E7FB1F238B8712A3019900EFD015
:10621400504D854719C1814749452300F900B240D3
:10622400224492440249410182809DC91DC9854787
:106234006318F500DC3193E707FCDCB10545828087
:1062440089476316F500DC3193F7F703FDB78D47F3
:10625400E316F5FEDC3193F7F70393E70704F1BF88
:10626400014582808DC10DC1DC311307000C054549
:1062740093F7070C638AE700130700040945639545
:10628400E7000D45828001458280411122C4005DF2
:1062940006C626C21DC8AA84085009C597A0FB1FBC
:1062A400E780A0E8485009C597A0FB1FE780E0E716
:1062B400085409C597A0FB1FE78020E7228597A013
:1062C400FB1FE78080E623AC0402B24022449244E0
:1062D4004101828019ED97E7FB1F83C707E417E5A7
:1062E400FB1F1305E5E491CB17E5FB1F130505B868
:1062F400828017E5FB1F1305A5E3828017E5FB1FCA
:106304000345A5E1828017E5FB1F0325A5E18280F3
:1063140017E5FB1F032545E1828097E7FB1F83A751
:10632400E7E08843828017E7FB1F1307E7DE544B3F
:106334009C4285079CC228339307F00F6307F5003E
:10634400916517C3FB1F670043678280011122CC4C
:1063540006CE2E8432C6EF9030019147B245631EBB
:10636400F50097E7FB1F83A7E7B099CF9C4389CF3C
:1063740022856244F2400561828797E7FB1F83A769
:10638400E7AF99C3DC43E5B7F240624405450561D4
:106394008280797122D42A844A214ECE06D626D20E
:1063A4004AD097C0FB1FE780007897E9FB1F9389C9
:1063B40069AD29E983C409009307F00F639DF400D4
:1063C40097E5FB1F83C515AC2685513C09E597E786
:1063D400FB1F238907AA4A20EF9000799147631C89
:1063E400F50097E7FB1F938727D35620FA2363947E
:1063F400E6007D57FAA3B250225492540259F2494E
:1064040045618280582504212A893AC6BD3D4A85C2
:10641400EF9050344A20EF90607083C709003247F0
:1064240099C3E38F97F89307F00F5220E385F4FAAA
:1064340074202820A685913E79BF79715AC82A8B89
:106444002E854ECE52CC56CA06D622D426D24AD057
:106454005EC62E8AB28AB68997C0FB1FE780A06CFD
:1064640075C5045D2A89FDC09C501305400391E362
:1064740061459C5489C79307450133C50708638662
:1064840009009307C50133C50708DC5089C7930782
:10649400750133C5070897A0FB1FE780A0DB2A849A
:1064A40055C56146814597A0FB1FE780E0F097EB57
:1064B400FB1F83CB2BC163940B00834B0900930711
:1064C40000FD1CA0A947A30064013CA023035401C0
:1064D4008C50231244011305840191C908C47146E8
:1064E400130A440397A0FB1FE78080E652858C546F
:1064F40091C948C45146130A450197A0FB1FE78080
:1065040020E55285638C090008C87146CE85130ABC
:10651400C50197A0FB1FE780A0E35285CC5099C525
:1065240048C85D4697A0FB1FE78080E2A2855E8590
:10653400EFD0BFBF2254B2509254F249624AD24AB9
:10654400424BB24B4A850259456181B3B250225441
:1065540092540259F249624AD24A424BB24B4561C3
:10656400828001114EC6AA892E8526CA06CE22CC67
:106574004AC8AE8497C0FB1FE780E05A21C917E9D7
:10658400FB1F034929B46314090003490500194595
:1065940097A0FB1FE78000CC2A840DC981451946CA
:1065A40097A0FB1FE78040E1930700FD1CA0B947BB
:1065B400A30034013CA046A0A2856244F240D24428
:1065C400B2494A85424905616FD03FB6F240624400
:1065D400D2444249B24905618280797162C42A8CED
:1065E4002E8526D24ECE52CC56CA5AC85EC606D680
:1065F40022D44AD0AE84B28B368BBA8A3E8AC28900
:1066040097C0FB1FE780205235C52A89414597A0D2
:10661400FB1FE78020C42A8431CD4146814597A0E1
:10662400FB1FE78060D917E5FB1F0345A5A919E106
:1066340003450900930700FD1CA0BD47A300840186
:106644003CA023047401A304640123055401A3059D
:10665400440146A023263401A2852254B250925408
:106664000259F249624AD24A424BB24B224C45612A
:106674006FD0BFABB250225492540259F249624ACD
:10668400D24A424BB24B224C45618280011126CA48
:10669400AA8439454AC84EC652C406CE22CC2E8A94
:1066A400B289368997A0FB1FE780C0BA15CD93073E
:1066B400000D1EA1B1472A84231245013CA1CE85B9
:1066C4001905194697A0FB1FE78080C823062401FB
:1066D400A2856244F2404249B249224A13F5F40FBA
:1066E400D24405616FD07FA4F2406244D24442494F
:1066F400B249224A05618280411126C206C622C4DB
:106704004AC097E4FB1F938424A1B8309307F00F89
:106714006308F7042A89394597A0FB1FE78080B3F3
:106724002A841DCD930700FD1CA1A300250123018C
:10673400050097E5FB1F9385A59F0D05194697A0B6
:10674400FB1FE780E0C09E24A285A8303EA49C30B5
:106754005CA42244B2409244024941016FD0FF9CA0
:10676400B24022449244024941018280011156C23E
:10677400AA8A314526CA4AC84EC652C406CE22CC7D
:106784005AC0AE84328AB6893A8997A0FB1FE78043
:1067940060AC2DCD2A84268597C0FB1FE780A038E6
:1067A40009C55825A1476311F70417EBFB1F034BD9
:1067B400DB96930700FD1CA09D47A30054013CA059
:1067C40046A0231344012314340123152401A28574
:1067D4006244F240D2444249B249224A924A5A851A
:1067E400024B05616FD07F9417EBFB1F034B1BB566
:1067F400E3910AFC97D7FB1F83A7C77C9C47D5DB93
:10680400CA864E86D2852685829765B7F240624451
:10681400D2444249B249224A924A024B05618280DB
:10682400411126C2AA84214522C406C62E8497A0FB
:10683400FB1FE78020A215C5930700FD1CA1C547D7
:106844003CA13C30AA853CB15E205EA17C207CA1A9
:106854007C307CB12244B2402685924441016FD001
:10686400DF8CB240224492444101828041114AC0EB
:106874002A89714526C206C622C4AE8497A0FB1F8E
:10688400E780409D3DC5930700FD1CA1F5473CA151
:10689400BC302A849385C4003CB1DE2031051946FE
:1068A400231CF5FEFE20231DF5FE9E24231EF5FE6B
:1068B400BC24230FF5FEBC34A30FF5FE97A0FB1FE9
:1068C400E78000A9BC28A2854A853CA8DE285EA8EA
:1068D400FC287CA8FC387CB89C2C1CAC9C3C1CBCC4
:1068E400BC2C3CAC2244B2409244024941016FD0DA
:1068F400DF83B24022449244024941018280011163
:106904004AC82A89614526CA4EC606CE22CCAE891B
:10691400B28497A0FB1FE780E09325C1930700FD95
:106924001CA1BC302A84938584001CB195473CA1EA
:10693400FC3011051946A30FF5FE97A0FB1FE78055
:1069440020A1DE2023063401A2853EA4BE2C4A8564
:106954007EA4DE2C1EA8FE2C3EA883C704025CA8DD
:1069640083C714025CB8BE30F240D2447EA86244AD
:106974004249B24905616FD04FFBF2406244D244B0
:106984004249B24905618280411122C406C617D426
:10699400FB1F130464783C209DCBAA85194617D5A8
:1069A400FB1F1305A54C97A0FB1FE780609A2820C6
:1069B40097D5FB1F9385854BEFF03F872244B24068
:1069C40017D5FB1F1305854A41016FD04052B240D1
:1069D4002244014541018280411126C206C622C4D7
:1069E4004AC097D4FB1F93842473B8309307F00FE5
:1069F4006302F7042A89294597A0FB1FE780808555
:106A04002A840DC9930700FD1CA1A147A3002501F9
:106A14003CA1BC2097D5FB1F938545451105A30FC9
:106A2400F5FE194697A0FB1FE7808092A830A28547
:106A3400EFD0AFEFB8208D47631FF70097D7FB1F48
:106A440083A7874389CB9C4799C72244B240924489
:106A5400024941018287B2402244924402494101E1
:106A64008280797122D406D626D24AD04ECE52CC18
:106A740056CA09444DCD2A890A212E8A514497C009
:106A8400FB1FE780400AAA845DC197EAFB1F938A33
:106A9400AA8A83C74A0005474944FD1793F7F70FAD
:106AA4006377F7085825A1476314F70063110A08B0
:106AB4009C5C4544ADEF9165938545711305C00217
:106AC4009790FB1FE780405988DCAA894D4425C173
:106AD4001306C002814597A0FB1FE780E08D835712
:106AE40009009386490036852391F9007146930580
:106AF400490036C697A0FB1FE7808085894723801D
:106B0400F900DC24B2460356090083C50A00E117E4
:106B140013B51700EF90B07D2A8463060A00D2856E
:106B24002685EF90807201C42685EFF00FF6B250EF
:106B34002285225492540259F249624AD24A45614A
:106B4400828097D7FB1F83C7677FFD1793F7F70FE3
:106B540005476377F70801114AC806CE22CC26CA36
:106B64004EC652C4328989472DC22A8AAE893684D8
:106B740097C0FB1FE78020FBAA84D14739C548553D
:106B840009C59790FB1FE780405AF1454A8597A0B5
:106B9400FB1FE7808088C8D4AA85CD471DC5D824AB
:106BA400A147631DF70209C8382D12299306250150
:106BB4005285EF90E06F2A84D8209367470063845E
:106BC400090093676700DCA0A287F2406244D244C4
:106BD4004249B249224A3E85056182800144E9BFA7
:106BE400C9473E8582809307000463EAA70097D7CC
:106BF400FB1F9387274A3325F5200A2182804165AC
:106C04007D158280011122CC2A842E8526CA06CEC7
:106C1400AE8497C0FB1FE78000F10DCDB7470F008E
:106C24009387F723094563E2870281450A85414634
:106C34009790FB1FE7804078A68560800A85418095
:106C44004081A3010100EF90504AF2406244D244D3
:106C5400056182804945D5BF97D7FB1F238FA76C59
:106C640082806F903063797152CC2A8A328526D221
:106C74004AD04ECE56CA5AC85EC662C406D622D47C
:106C84002E8CB28A368BBA8B3E89C289C68497C051
:106C9400FB1FE78040E905C92A84631A0A18937721
:106CA4004B000343450085CF1363230163940B1604
:106CB40063100914639F090885E81C5C1373B3FF10
:106CC40023026400C5EBB250225492540259F24993
:106CD400624AD24A424BB24B224C456182801373C2
:106CE400D3FF13630301D9B7136343002302640082
:106CF4009C484146A6851CD4130584019790FB1F2C
:106D0400E780006563130C12638C0B0A485409C5B1
:106D14009790FB1FE7806041F1455E859790FB1FCC
:106D2400E780A06F48D4005C59DC1C5091EB91655E
:106D34009385357171459790FB1FE780E03108D04A
:106D440008500DC17146DE859790FB1FE7804060B7
:106D540011A81363430023026400D9F8005C630C98
:106D64000C0235D0639A0902A5E029A0005C21DC5D
:106D7400639409022254B2509254F249B24B224C09
:106D8400CA865A860259424BD6855285D24A624AED
:106D940045616FF08FEA05D85C5091EB916593855E
:106DA40025715D459790FB1FE780002B48D0485024
:106DB40045DD5D46CE859790FB1FE78060596DB732
:106DC400005C11D0E39A09FC1C5491EB9165938506
:106DD400157151459790FB1FE780002808D408548B
:106DE40051D95146A6859790FB1FE780605659B745
:106DF4001363430023026400E39C04EEE3080CF6EF
:106E0400485405EDF1454A859790FB1FE780E06003
:106E140048D431A81363430023026400E39A04ECCA
:106E2400E3060CEEE31E09FCFDBDE31B09FC005C5C
:106E3400E30B04E8E39B0BEE35B79790FB1FE78069
:106E4400C02EC9B7011126CA52C406CE22CC4AC8E4
:106E54004EC62A8AAE8497C0FB1FE780C0CC35C1DA
:106E64002A8939459790FB1FE780C03E2A8431C99F
:106E740097D9FB1F83C90925639409008349090035
:106E84009307000D1EA0AD473CA0930569001305B0
:106E9400340019469790FB1FE780804B93F714004A
:106EA4005CA493D4144844B423154401A2856244D9
:106EB400F240D2444249224A4E85B24905616FD01C
:106EC400CFA6F2406244D2444249B249224A056103
:106ED400828001114EC652C456C206CE22CC26CAA6
:106EE4004AC8AA8A2E8AB28997C0FB1FE780A0C32A
:106EF40035CDAA841305C0029790FB1FE780803527
:106F04002A842DC517D9FB1F0349C91B6314090023
:106F140003C904009307000D1EA0E9473CA0938514
:106F240064001305340019469790FB1FE780404224
:106F3400D285231554011305C40041469790FB1FC5
:106F4400E7800041CE851305C40141469790FB1F9D
:106F5400E7800040A2856244F240D244B249224A0A
:106F6400924A4A85424905616FD02F9CF24062449F
:106F7400D2444249B249224A924A0561828017D5D5
:106F8400FB1F0325A5ED11CD411106C69790FB1FEC
:106F9400E780A019B24097D7FB1F23A107EC41015A
:106FA40082808280411122C406C626C24AC02E8431
:106FB40097C0FB1FE78020B729CD00D517D9FB1F49
:106FC40003494910AA846314090003490500414593
:106FD4009790FB1FE78000282A8405CD9307000DB6
:106FE4001EA1A5473CA1DC30938564001105A30FC5
:106FF400F5FE19469790FB1FE78080359C54A285C7
:10700400B2405CC4224492444A85024941016FD093
:10701400CF91B240224492440249410182805D7181
:10702400A2C4A6C286C6AA842E8497C0FB1FE7808A
:1070340080AF0DC954251147AA874945639FE600CF
:107044009C5F91C3E02B97B60000938646990A860D
:10705400894526854080EF904016B64026449644E4
:10706400616182805145D5BF97D7FB1F83C7072D28
:10707400FD1793F7F70F0547637AF704411126C20A
:1070840006C622C44AC0B284894715CA2E8997C04D
:10709400FB1FE78040A92A84D14715C16306090074
:1070A4005C2193E727005CA14146A6851305840172
:1070B4009790FB1FE780C0299C481CD48147B240AD
:1070C4002244924402493E8541018280C9473E855B
:1070D4008280011122CC26CA06CE2A84AE8497C0AF
:1070E400FB1FE78040A419C96C0022854486EF90F9
:1070F4006012F2406244D244056182805145D5BF9A
:107104006F80901BC1671387E7FF6393E50297D7EE
:10711400FB1F83A7A7D691EB494582804945B2401E
:10712400224492440249410182809C43F5D78287DC
:10713400411122C426C24AC006C6FD172A892E84DC
:10714400B284639AF50297D7FB1F83A727D389C715
:107154009C4399C3829711C5A6854A85EFE03FD029
:107164005DFD97D7FB1F238F27D197D7FB1FA38BD9
:1071740097D001456DB72E8597C0FB1FE780A09A75
:1071840051DD1C210D45E39C27F922852244B240A0
:107194000249A685924441016FC0705293070004CE
:1071A40063E1A7064111C16722C426C206C6FD17C2
:1071B4002A84AE8409456380F502C5476312F4024C
:1071C4002E85EFC0705797D7FB1F9387A7EC332406
:1071D400F420014506A0B240224492444101828039
:1071E4009307A0036316F4002E85EFC0104EE1BF91
:1071F4009307B003E319F4FC13F5F50FEFC0304D1A
:10720400D9B709458280011106CE2AC6EFE03FC7EF
:10721400EF20404EEF10C07CEF503231324597D70B
:10722400FB1F938767EF130700F0BAA323820700BD
:107234007D5797D7FB1F93872710B8A388A3F240E5
:10724400954505616F70402A757126C306C722C52E
:107254004AC1CEDED2DCD6DADAD8DED6E2D4E6D241
:10726400EAD0EECEAE849397556063D1075817DA0F
:10727400FB1F130A6A0C03450A00130B200A930B25
:10728400F00F9790FB1FE780E002C167FD172A8487
:10729400130C1009954C394D97DDFB1F938DCDE7E9
:1072A4003ECC15E01395F468BA402A449A440A493E
:1072B400F659665AD65A465BB65B265C965C065D02
:1072C400F64D496182801C20639A670103C93D0021
:1072D400E2452A202286EFF06F87E1A003492A00C5
:1072E400639A87091C30639097032285EFF06F8AB5
:1072F4002285EFC07FDE03450A009790FB1FE780DD
:1073040060FB2A8479BF639BA7194A208567A50778
:10731400631AF5040C4497D9FB1F9389E9DF88218C
:1073240015E51946850517D5FB1F130565E09790EC
:10733400FB1FE780E00103C709008547631CF702D0
:1073440089472380F900EFC0503A5DB703C70900AD
:1073540085476311F70297D7FB1F238F07DAEFF0F6
:10736400AFB979B709679307C70063EFA7040507A7
:10737400636BA702E30E79F7A2854A85EFC0FFDAB3
:107384009DBF370700181307F770B357F748E5CBCD
:1073940097D7FB1F83A747AEA1DF9C43B1DB2285B0
:1073A400829739F5C1BFF977F917AA972947B3C767
:1073B40007086366F70C176702001307675BB3C718
:1073C400E7209C43BA978287F9779387A7FCAA970B
:1073D400F146B3C70708E3F6F6FA3907E31CE5F804
:1073E40097D7FB1F83A787A9E38407F0DC43E381D6
:1073F40007F00965A2853905A5A883298400E38BD4
:1074040009F603C7090097D7FB1F9387E7D019EB49
:1074140003C7290083C619002207558F9AA703C7FB
:10742400390098B394230947E396E6F403C70900A7
:1074340001CB97D7FB1F238107CE03C5090005B7EE
:107444008C338A270D4798A3EF70A00CFDB71C441A
:107454008823EFF06FD869BD97D7FB1F83A747A296
:10746400E38807E89C43E38507E80965A2852D05C1
:10747400829705BF1C449C23E39E07EE95BD896754
:1074840093871704E318F5EE97D7FB1F83A7479F4D
:10749400E38007E69C43A285E1FF99BD3D476394E1
:1074A400E7064A2089671387D7006306E500138738
:1074B4009701631AE50097D7FB1F83A7279CE389ED
:1074C40007E2DC43C9BFCD07E316F5EAC16717D766
:1074D400FB1F0357C7C4FD17631FF70097D7FB1F94
:1074E40083A7C799E38607E0DC43E38307E00965E4
:1074F400A2854D05B5BF97D7FB1F83A7A797E3893F
:1075040007DE9C43DDB71307E003E395E7E63C2081
:1075140005476398E7127C2097DAFB1F938A0A9445
:107524006390071083A70A006387070E83C90700C7
:107534002149683093078400BE853ECEEFE09FD298
:1075440068B013064002814568109790FB1FE780DE
:10755400A0E63C30194693058400A307F1027C3071
:107564004818A309F1029790FB1FE78060DE5E20B4
:107574007010CA852318F1027E244E852313F1046A
:107584001E282314F1043E282315F1045C28230645
:10759400F104FD57A306F1042317F104EFF02FB60D
:1075A4003C309DE3DD47835804010358E400743004
:1075B4004E203EC23E28130784003EC0CA870546BB
:1075C4004E85EF80A07128B083A70A0081C71145BA
:1075D400EFF0FF9A97D9FB1F9389C98A03C5090065
:1075E400E30805D097D5FB1F83C5D589EFE03F8716
:1075F400E30005D03430930710036389F60052206A
:1076040083C509004A873685EFE03F9897D7FB1F6B
:10761400238A0786F1B997D9FB1F83C919B009BF1B
:1076240097D7FB1F83A7478597D9FB1F83C9F9AE5B
:1076340099C3DC4399E31149EDBD81450145829726
:10764400DDBFF91793F7F70F13077002E364F7D25E
:107654001767020013078734B3C7E7209C43BA9720
:1076640082877C2097CAFB1F938A4A7FA9EB83A752
:107674000A00A9C383C9070021496830937725000C
:10768400A5C305891307440168B02286CA854E85BF
:107694003ACEEFF0CFA63C3072479DF7DD478358D2
:1076A400C4010358A40174304E203EC27E2C3EC057
:1076B400CA8731B797D9FB1F83C939A675BF97C746
:1076C400FB1F83A7677B97D9FB1F83C919A599C3A0
:1076D400DC4399E3114955B7814501458297DDBFE4
:1076E40013078400BA853ACEEFE0DFB7724769BF6B
:1076F40097C7FB1F83A7C778E38C07BEDC43E389E6
:1077040007BE22858297EDB697C7FB1F83A74777ED
:10771400E38007BE9C47E5B722868D454A2065BEB7
:107724009305A10213051031EF5002686C10130584
:107734002031EF50626772208357C1024A2063E709
:10774400C70016240357A10263F7E600930500025D
:10775400EFC0807D71BE6373E6007AA063F3D70047
:107764001EA45A24362412246E2001488147EFC0F7
:10777400607BBDBE2286B14555B797C7FB1F83A763
:107784002770E38707B6DC479DBF2285EF00607B47
:1077940085B697C7FB1F83A7A76EE38B07B49C4BE3
:1077A400B9BF2285EF00F003A1B60145EF00301305
:1077B40081B697C7FB1F83A7276CE38D07BADC4309
:1077C400E38A07BA8145054582976DB697C7FB1FC3
:1077D40083A7876AE38007BADC43E38D07B8A285F1
:1077E4000945DDB72286930560020DBF93F71500A6
:1077F40089CF97C7FB1F83A7A76889C7DC4399C3B1
:107804000145829713C5140045B493F7250091CF21
:1078140097C7FB1F83A7476691C7DC4381C7814590
:107824000545829713C5240041B413F54500E30DC3
:1078340005A697C7FB1F83A7A76217D4FB1F1304D2
:10784400A48D89CF85475CA097C7FB1F83A7C76218
:1078540091C7DC4381C781450545829748446C1034
:10786400EF8030756810EFF02F9297D7FB1F83D706
:10787400878481CF130600643386C702914517D5E8
:10788400FB1F034565ABEFC07FB013C5440029BCA3
:10789400011122CC2A84554506CE26CAEFF0AFB496
:1078A400AA8413054002EFF00FB42AC61305500250
:1078B400EFF06FB3AA86228562443246F240B335B4
:1078C4009000D24405616FC0006E397122DC06DE7F
:1078D4000D472E84631AE500BA259625F221283037
:1078E400CE21EFE0BFE899A809679306D700AA87DD
:1078F400631BD504BC21B9C317C4FB1F130404566E
:107904000C408DCDDC87BC31194691054808A3098C
:10791400F1009790FB1FE780A0A3930700F03ED6E9
:107924001C40231801002313010202D48823700091
:107934008145EFE0DFFC0545EFF06FE40545F250CB
:107944006254216182809306E700E309D5FE930621
:1079540037016319D500A82175D101478146014635
:10796400814541B76507E30BE5FC31476319E50041
:1079740017C5FB1F0345757AEFE09FEAC1B71307EC
:1079840060026319E50017C5FB1F03451579EFE095
:10799400FFED6DB741677D170145E392E7FAD831F2
:1079A400C947E31DF7F8F625D2250A24AE25EFC012
:1079B4002067854711C55D45EFF0EFA2B337A000FE
:1079C4004C202A2030007C84EF70F06B3C84BDF79F
:1079D4009305A10013051031EF50023D6C0013050F
:1079E4002031EF50623C3C851A246373F7001EA4D7
:1079F4003C863A2463F3E7003EA41E243A246373CE
:107A0400F7003EA42A20EF4001227A24562432248F
:107A14000E242A2001488147EFC0A04E05B741112A
:107A24004AC006C622C426C217D9FB1F1309C9902F
:107A3400034779009307F00F6302F706AA8439CD50
:107A4400682551059790FB1FE780C0802A8439C5BB
:107A54009307000D1EA1D9473CA1DE205EA1FC20A6
:107A64007CA1FC307CB19C241CA5DC345CB5F024E6
:107A740070A515C28C48510508C89790FB1FE78074
:107A8400208DA285224403457900B24092440249E4
:107A940041016FC08FE923280500E5B7B2402244B5
:107AA4009244024941018280C1679386E7FF2A8795
:107AB400639DD50097C7FB1F83A7473A8DC39C23BB
:107AC4000D45639FE7006FC00043FD174945639967
:107AD400F50097C7FB1F83A76738F5F782804945F0
:107AE4008280397122DC06DE26DA4AD84ED652D498
:107AF40056D25AD0182185472A84630BF7001025E3
:107B0400930695009305E1010545EFE0CFDA0DED0D
:107B14008147014514201147638FE60217C7FB1FF5
:107B24000327073718338D466307D7028DC705C768
:107B340011ED0145F2506254D2544259B259225ABD
:107B4400925A025B216182801C21E9B78546631148
:107B5400D7048D8BF9DF0830930524002EC6EFE09F
:107B64006FF008B017C9FB1F1309C9328327090036
:107B7400AA8981449DC3B24517CAFB1F130ACA319F
:107B8400130BF00F83470A0063EBF400814481A0D8
:107B94008946E310D7FA858B75BF054561BF8327F6
:107BA4000900939A4400D6979823630C6705983389
:107BB400631937051946138527002EC69790FB1FB6
:107BC400E780808AB24515CD83240900D694182015
:107BD4009147C1E8E30FF7F483240900B9D8834639
:107BE4000A0081471306F00FE385F6F403C8040086
:107BF40013850401630BC800850793F7F70FAA8464
:107C0400E5B7850493F4F40FB5BF98A01C30138531
:107C1400240019469CB09780FB1FE78060730824FA
:107C240091659385F57105059780FB1FE780C04238
:107C340005C1182091476314F702C8C410249305A2
:107C440094000505A30FC5FE9780FB1FE7804070D5
:107C54001C24A1F708207D1513351500E1BD88C447
:107C6400F1BF6311F706C8441C2405C11021630D3C
:107C7400F604182091476317F706C84419C597807E
:107C8400FB1FE780804A23A604000824916593859E
:107C9400E57105059780FB1FE780003C05C11820AE
:107CA4009147631AF704C8C410249305940005058A
:107CB400A30FC5FE9780FB1FE78080690824333536
:107CC400A0008DBD88444DB79305940005059780A9
:107CD400FB1FE78060798547E31DF5F85545EFE024
:107CE4009FF09DBF884455D19780FB1FE780E043F8
:107CF40023A4040059BF88C445BF397122DC4AD883
:107D04004ED652D406DE26DA56D25AD05ECE2A8415
:107D1400130925000831CA8517CAFB1F130A4A171D
:107D2400EFE04FD408B083270A000D47AA899C339B
:107D34006391E70217CAFB1F130ACA1583270A00B7
:107D4400814497CAFB1F938A2A156393071005453C
:107D54002DA0EDD3144C70389305E1000545EFE0F8
:107D64008FB5AA841DC903270A0085461C21183330
:107D74006310D7028D8BDDFF0145F2506254D2545B
:107D84004259B259225A925A025BF24B21618280C3
:107D94008946858BE310D7FAF9BF1C201147638508
:107DA400E7002D47E39AE7FC97CAFB1F938A8A0EE4
:107DB40083A70A00014A97CBFB1F938BEB0DCDDF02
:107DC40003C70B00B3470A0863E4E700A5F46DB7E3
:107DD40003A50A00131B4A001C205A95182163109E
:107DE400F7021C31639D37011946CA85090597803E
:107DF400FB1FE780606701C583A40A00DA94050AC3
:107E0400C1B783A9840059A80C4C13851900978025
:107E1400FB1FE780606585476317F5085545EFE06C
:107E24009FDC4DC191BF1C2011476385E7002D479E
:107E3400639DE700C8C470380505A30FC5FE0C4C4C
:107E44009780FB1FE780C050B5A888C4EDB78504B0
:107E540003C70A00B3C7040863F8E70603250A004A
:107E6400139B44001C205A951821E312F7FE1C3181
:107E7400E39F37FD1946CA8509059780FB1FE780F4
:107E8400A05E71D583240A001C201147DA9463850F
:107E9400E7002D47E397E7F683A9C4007C3803C6BF
:107EA4000900E303F6F64E859780FB1FE780E02781
:107EB400683891659385E57105059780FB1FE78018
:107EC400A01935F1E39504E803C70A0083240A00E6
:107ED40081479306F00FE3FCE7E68C201386040148
:107EE4006387D5008507B284B3C70708EDB7E3807D
:107EF40004E61C20CA85138524009CA01C30194666
:107F04009CB09780FB1FE780A044683891659385F7
:107F1400F57105059780FB1FE7800014E30905E26E
:107F240018209147631DF700C8C470380505A30FD6
:107F3400C5FE0C4C9780FB1FE780804109BD88C4B7
:107F4400EDB701114AC806CE22CC26CA17C9FB1FB9
:107F54001309893E034779009307F00F630DF70671
:107F6400AA8435C961459780FB1FE780A02E2A8427
:107F74003DC19307000D1EA1D5473CA1BC3093859C
:107F840084002EC63CB1DE205EA1FC207CA1E8303A
:107F9400EFE04FADB24568B01946130584009780F1
:107FA400FB1FE780E03AFC24A285034579007CA40A
:107FB4009E281EA8BC283CA8BC383CB8DC285CA879
:107FC400DC385CB8FC287CA86244F240D2444249C4
:107FD40005616FC08F95F2406244D2444249056105
:107FE4008280411126C206C622C497C4FB1F938413
:107FF400A434F8309307F00F6309F7022A8415C5F7
:1080040019459780FB1FE780E024AA8519CD9307C3
:10801400000D1EA1DD473CA15E202244B2405EA1BA
:10802400E830924441016FC04F90B24022449244E0
:1080340041018280011126CA97C4FB1F938484E501
:108044009C4006CE22CC4AC84EC652C49DC32A893F
:10805400AE89131A45000144884063144403638CB9
:1080640009049780FB1FE780400C97C7FB1F23A3DD
:1080740007E2F2406244D2444249B249224A0561CD
:108084008280B3078500884709C99780FB1FE78072
:10809400C0099C40A29723A407009C40A297C8470C
:1080A40009C99780FB1FE78040089C40A29723A63C
:1080B4000700410455B755DD228681459780FB1F93
:1080C400E780802F944081477D5613F7F70FE372C2
:1080D40027FB13974700369710A38507FDB77971DF
:1080E40052CC17CAFB1F130AAADA83270A0006D642
:1080F40022D426D24AD04ECE56CA5AC85EC6E9C742
:108104002A8997CAFB1F938A2AD9814419ED97C6F5
:10811400FB1F83A626D891CA03C60A00814793058C
:10812400F00F13F7F70F6369C702139534002105A5
:108134009780FB1FE78000122A8415E92145978068
:10814400FB1FE78020112A8435C1C5679387073D4B
:108154001CC123220400A9A01397470036971823B3
:108164006305B700850493F4F40F85075DBF930797
:1081740000FD1CA18547A30025013CA124B1F1D831
:108184001309850023222501814917CBFB1F130BFB
:108194006BD0930BF00F83C70A0063F3F900A1E0DF
:1081A40083270A00A2858823EFB03FF803C50A009D
:1081B4008145493503250A009780FB1FE780E0F6D7
:1081C40097C7FB1F23A607CCB250225492540259DE
:1081D400F249624AD24A424BB24B456182808325BE
:1081E4000B0093974900BE959C216383770323007A
:1081F400F9009C3113052900FD14A300F900194668
:10820400890593F4F40F9780FB1FE780601421091C
:10821400850993F9F90F41B797C7FB1F83A747C790
:10822400A9C7411122C406C62A8415E10945EFE015
:108234009F9B2A8601C9854517C5FB1F0345C50FAA
:10824400EFC0CF940545EFF0AFE42A8411C985450A
:1082540017C5FB1F0345450EEFC0AFBC2285413552
:10826400B2402244054541018280014582808967EC
:108274009386B7006315D5009C45882371BF938608
:10828400C7006317D5009C458546882319C9FDB7E7
:1082940093861704E302D5FE938727048146E304FB
:1082A400F5FE36858280011106CE22CC26CA4AC844
:1082B4004EC652C456C261C13C312A898DC3444161
:1082C40099CC5945EFE03F92814997CAFB1F938AA5
:1082D4002ABC131A45608347390063EBF900F24066
:1082E4006244D2444249B249224A924A0561828098
:1082F4008387840263C8470783A70A00A5C7268526
:10830400EFF02FFE25C1882451059780FB1FE780DD
:1083140060F42A8421C99307000D1EA1B5473CA12E
:108324009C201946938524003CB18387840215055B
:108334007CA19C30A30FF5FE9780FB1FE7804001D2
:10834400902450A415C61305440108C893859400CD
:108354009780FB1FE780C0FF83A70A00A2858823BC
:10836400EFB0BFDC85099384940293F9F90FA5B7A4
:1083740023280400D5B797C7FB1F83A767B1A5D3EC
:10838400B93B6244F240D2444249B249224A924A39
:10839400014505616FF0CFCF797106D622D426D27C
:1083A4004AD04ECE52CC56CA5AC85EC655CD3C3180
:1083B4002A898DC744419DC05945EFE0DF82890475
:1083C400814997CAFB1F938AAAAC130B00FDC14BCA
:1083D400131A45608347390063EDF900B250225403
:1083E40092540259F249624AD24A424BB24B456115
:1083F40082808387D40063C4470783A70A00A5C388
:1084040051459780FB1FE780E0E42A8429C92300B3
:108414006501A30005002301750183C7E4FF194624
:10842400A6853CB18387D40015055CB583C7F4FFEA
:10843400A30FF5FE9780FB1FE78080F1FC20938556
:1084440074001305C4003CB419469780FB1FE780F1
:1084540020F083A70A00A2858823EFB01FCD8509E9
:1084640093F9F90FC104BDB797C7FB1F83A747A2B0
:10847400B5D7B5312254B25092540259F249624AE6
:10848400D24A424BB24B014545616FF06FC07971DE
:1084940006D622D426D24AD04ECE52CC56CA5AC878
:1084A4005EC662C466C2630C05223C312A8985CB50
:1084B400404115C45945EFE00FF30904814917CA37
:1084C400FB1F130AEA9C914B354C175B0200130BFC
:1084D400EB56931A45608347390063EFF900B250B5
:1084E400225492540259F249624AD24A424BB24B44
:1084F400224C924C456182808307A40063CA5715BD
:1085040083270A0063860714834CE4FF93F70C0166
:10851400CDC793870CFF93F7F70F6369FC00B3C7CC
:1085240067219C43DA978287230F04FE1305E4FF37
:10853400EFF0AFFC630E05108347E4FF63EFFB101D
:1085440005476398E70A51459780FB1FE78080D071
:10855400AA84630F050E930700FD1CA1C147A30065
:1085640005003CA18347E4FF1946A2853CB183077B
:10857400A40015055CB58347F4FFA30FF5FE9780AF
:10858400FB1FE780E0DC7C2419469305F400BCB4AF
:108594001385C4009780FB1FE78080DB65A08547B7
:1085A400230FF4FEA30A040051B78947230FF4FEF6
:1085B400B5BF8D47E5BF9147D5BF93F78C0099C3ED
:1085C400AD47EDB713F71C0093F74C0011C799C3DF
:1085D4009547F9B7A147D9BF13F72C0011C799C321
:1085E400A5477DBF9947D9B799C3A947C1B79D4747
:1085F40075BF483851059780FB1FE780A0C5AA8442
:1086040021C99307000D1EA1B5473CA18347E4FF90
:108614001946A2853CB18307A40015057CA18347B4
:10862400F4FFA30FF5FE9780FB1FE78060D250385C
:10863400D0A419C61385440188C88325640199BF51
:1086440023A8040083270A00A6858823EFB0FFAD82
:10865400850993F9F90F7104BDBD48381305050266
:108664009780FB1FE78000BFAA847DD19307000D8C
:108674001EA1C9473CA18347E4FF93FC0C0619469D
:10868400B3E797013CB18347F4FFA2851505A30F17
:10869400F5FE9780FB1FE780A0CB7C20194693054D
:1086A400F400BCB47C3013853401DCA41C24DCB499
:1086B4001C34FCA48307A400FCB45E249EA87C2480
:1086C400BCA89780FB1FE780A0C8503890BC09C69F
:1086D40013850402C8CC95B723AE0400A5B797B799
:1086E400FB1F83A7E77AE38C07DEEFF05F9F22543A
:1086F400B25092540259F249624AD24A424BB24BA6
:10870400224C924C014545616FF08F9817B7FB1FBF
:108714000327077805CB1823AA870D456315F702AD
:108724004111854517C5FB1F034505C106C6EFB0BA
:108734005FEF13050003EFF09F9AB240014541013A
:108744006FF00F954945828079714AD017B9FB1FA4
:10875400130909748327090006D622D426D2CDEB47
:1087640017C4FB1F130444BD5820C947298B51CBA0
:108774009165AA849385D57111459780FB1FE78085
:10878400A08D2320A900CD472DCD78309307F00F7D
:108794006314F7009C207CB01146A6859780FB1FCC
:1087A400E78000BB930531011305F041EF20122F40
:1087B40097C7FB1F93874796A023034731013334A0
:1087C400800011C3090413051002EFE0CFC1137632
:1087D400F50F0589E14715C5154532C6EFE0AFC071
:1087E400BC20E8841945230AF100EFE0CFBF3246EC
:1087F400AC30E8867C08380854082285EFB0607AEB
:10880400AA87B2502254925402593E85456182800F
:10881400C547C5BF1971A2DCA6DA86DECAD897C4DB
:10882400FB1F938464B1DC204944A18BB9CF97B773
:10883400FB1F83A7E7654144A9EB2A89EFE05F8C1E
:108844009C2455446373F50497B4FB1F938404611B
:108854009C4045449DEB91659385C571294597706E
:10886400FB1FE780607F88C04D4405C12946CA8547
:108874009780FB1FE780C0AD13056002EFE0AFB641
:108884001374F50F058909E96144F650228566548D
:10889400D654465909618280130600038145880035
:1088A4009780FB1FE78040B14145EFE0CFB323162B
:1088B400A1043D45EFE02FB32319A1043545EFE0B2
:1088C4008FB2231CA1043945EFE0EFB1231FA104AB
:1088D4002145EFE04FB12312A1061D45EFE0AFB0F3
:1088E4009C402315A106136424009C33F1C72D4535
:1088F400EFE06FAF2310A1043145EFE0CFAE2313B7
:10890400A1041305C002EFE00FAE2317A104130561
:10891400B002EFE04FAD231AA10413059002EFE07B
:108924008FAC231DA1041305A002EFE0CFAB2310ED
:10893400A10613058002EFE00FAB2313A106130574
:108944007002EFE04FAA9C402316A106A83393853A
:108954004700EFD09F8D2AD69305F1031305F0410C
:10896400EF20D21397B7FB1F9387077BAC230347F2
:10897400F1033256B335B00011C389059440FC00AD
:108984002287A8223EC8930721053EC6BC083EC4E0
:108994009307E1053EC2DC103EC09308A10613080C
:1089A40061049C009106EFB040602A84E30F05EC5B
:1089B4000D45EFE0CFDCD1BD2545EFE0CFA223107C
:1089C400A10429451DBF97C7FB1F83C72797A18B08
:1089D40017B5FB1F1305454B91E301456FD0AFE17C
:1089E40097B7FB1F238A074AFD5717C7FB1FA30826
:1089F400F79497B7FB1F23AF074897B7FB1F23A92B
:108A0400074897B7FB1F93872773170700001307BF
:108A1400478698C31707000013072789D8C3170789
:108A240000001307A79798C717070000130767A646
:108A3400D8C717F7FFFF1307C7FE98CB97B7FB1FDD
:108A44009387874417F7FFFF1307470698C317F761
:108A5400FFFF1307C7E7D8C38280411122C426C28F
:108A640006C617B4FB1F13042443AA8408208545B3
:108A7400EFF04FDC97C7FB1F83C7478CA98BBDC79B
:108A840017B5FB1F1305456B04A0EFD02FD697B481
:108A9400FB1F938424409C4099C74D45B240224417
:108AA400924441018280082019E10145C5BF9165C6
:108AB4009385B57112059770FB1FE780E05988C054
:108AC40069DD1020814512069780FB1FE780C08E68
:108AD400142090408147FD5513F7F70FE377D7FC37
:108AE4001397470032970CA38507FDB7014597B745
:108AF400FB1F2383073AEFD06FCF45BF17B5FB1F8A
:108B04000325053611CD411106C69770FB1FE7807A
:108B1400C061B24097B7FB1F23A407344101828090
:108B2400828001111305700306CEEFE0CF8B2AC6B5
:108B340013058003EFE02F8B2AC413059003EFE0A5
:108B44008F8A2246B245F240AA86054505616FB078
:108B540080445D711305D00386C6A2C4A6C2CAC0F0
:108B6400EFE06F882A841305C003EFE0CF87AA845F
:108B74001305E003EFE02F872A891305F003EFE0E4
:108B84008F868A871377F50F9376F90F13F6F40F10
:108B94009375F40F0545EFB04042B6402644964421
:108BA400064961618280011122CC06CE26CA0D4796
:108BB4002E846317E504B831E947CA2197B4FB1F33
:108BC400938484556315F700FE206387A70497A058
:108BD400FB1FE78040F5722011C172A53A241624C8
:108BE4004E202830EFD09FB85A20FE206314F7009F
:108BF400FD57FEA00545F2406244D24405618280DF
:108C040009674D07AA87631CE500BC2131476385CA
:108C1400E7004547E390E7FEEFD00FC5E1BF3147DA
:108C24006319E50017B5FB1F03455571EFD05FBF0E
:108C3400D1B7130760026319E50017B5FB1F03459D
:108C4400F56FEFD0BFC27DB741677D170145E3944F
:108C5400E7FAD831C947E310F7FACC212A203000CB
:108C640023140100EF60303D71B71971A2DC17B411
:108C7400FB1F1304E41E1C4086DEA6DACAD8CED637
:108C8400D2D4D6D2DAD00545638A070C9305F10510
:108C94001305F041EF2082609305F1051305F041BF
:108CA400EF20C25F97B7FB1F93870747BC23034797
:108CB400F105B337F00011C389071840BEC6283345
:108CC40093054700EFD06FD61840AAC40D452C2356
:108CD400AEC2EFD05FF1AAC01145EFD0DFF0832A16
:108CE40004002ADE654503C7AA0003CBBA003ADCB8
:108CF400EFD07FEF2A846945EFD0FFEEAA84714557
:108D0400EFD07FEE2A896D45EFD0FFEDAA89754536
:108D1400EFD07FED2A8A7945EFD0FFEC2648B6479D
:108D24006257F256064696451375F50F137AFA0FF5
:108D340093F9F90F1379F90F93F4F40F2ACC131460
:108D4400446002D002CE52CA4EC84AC626C422C2C9
:108D54005AC093884A000545EFB0C01EF6506654C9
:108D6400D6544659B659265A965A065B09618280EA
:108D7400411122C44AC006C626C217B9FB1F1309F3
:108D84003913834709001307E00F2E846382E70435
:108D94001307F00F6385E70211459770FB1FE78007
:108DA400604BAA8509CD930700FD1CA189473CA10E
:108DB400854700B13CB103450900EFB00FB7F9573F
:108DC4002300F900B24022449244024941018280C6
:108DD400AA8411459770FB1FE780C047AA857DD1FF
:108DE400930700FD1CA1894700B13CA124B1224492
:108DF400B2409244024917B5FB1F0345650B41017C
:108E04006FB0AFB279714AD017B9FB1F1309490586
:108E14008327090022D406D626D24ECE52CC45440E
:108E2400C5EB97B4FB1F93842451DC204944958BF4
:108E3400C5C32E8A916597B7FB1F238BA706AA8902
:108E44009385757131459770FB1FE780E0202320DF
:108E5400A9004D4435CD23003501A3000500294662
:108E6400D28509059770FB1FE780804E0327090010
:108E740091463C2363E7F606CD4691CF0546F54679
:108E8400638BC7000946C9466387C7000D46C146C0
:108E94006383C700D54634A3930571001305F041DD
:108EA400EF20C23F9C83C5E317B7FB1F0347E726A8
:108EB4008D47631AF708EFD00FC52C00EF70700FC1
:108EC4002800EFD07FAC4545EFD0FFD125E5014424
:108ED400B2502285225492540259F249624A4561A1
:108EE4008280ED1793F7F70F95460544E3E2F6FE0B
:108EF40097560200938606B8B3C7D7209C43B6970B
:108F0400828789473CA319A0230107006545EFD058
:108F14009FCD9307F007E301F5F8032709003C23ED
:108F240093E707043CA38DBF8547E9BF9947D9BFA1
:108F34009147C9BF130600643306C50288209145D2
:108F4400EFB0CFC469B715332A8451D1EFF01FBBFA
:108F540041B7011126CA97B4FB1F938464F09C4067
:108F640022CC06CE4AC84944A1C79C230D44639130
:108F7400A70417B9FB1F1309293C034509008945B8
:108F8400EFB02FEA03450900914597B7FB1F239FD4
:108F940007F0EFB00FE99C400147814680B3130608
:108FA400F100854785450145DC87EFA0907E2A8442
:108FB400F24022856244D244424905618280011113
:108FC40006CE22CC26CA4AC84EC68547631EF5067D
:108FD40017B4FB1F130484ED1E20B1CB17B7FB1F7E
:108FE4000347C71329E71307B003636EF70297B467
:108FF400FB1F9384643488208945EFB08FE21220EC
:109004009307006488203306F6028945EFB00FB851
:1090140097B7FB1F239C07E8F2406244D2444249BD
:10902400B24905618280938747FC1EA0F5B797B7C4
:10903400FB1F83A7E7E2EDD36244F240D2444249E6
:10904400B2498823056131B797B9FB1F938949E178
:1090540083A70900F1D317B9FB1F1309E92D83472F
:109064004900918BD5DB89476311F5062D45AE8404
:109074009770FB1FE780001E2A8459DD930700FDCB
:109084001CA1E547A30005003CA1BC301505194609
:10909400230FF5FEDC2093855400A30FF5FE977093
:1090A400FB1FE780E02A034559009307F00F63157F
:1090B400F50083A709008823A2856244F240D244C4
:1090C4004249B24905616FB04F860345090089459D
:1090D400EFB02FD56244F240D2444249B24997B727
:1090E400FB1F239507DC05616FF05FA197B7FB1F9A
:1090F40083C7C724958B89CF97B7FB1F83A747DA0C
:1091040091CB854717B7FB1FA303F7DA6FF07FA155
:10911400494582804145828097B7FB1FA38907D8C0
:10912400854501456FA0B06797B7FB1F83C707212B
:10913400958B81CB854717B7FB1F230AF7D66FF0B2
:109144005FA14945828097B7FB1F238207D68145DB
:1091540005456FA0D06697B7FB1F83C7271E958B65
:10916400638B0712011122CC06CE26CA4AC84EC60A
:109174009307C01C328463FAC7000945F240624475
:10918400D2444249B2490561828097B7FB1F83A745
:1091940027CD6384071097B7FB1F938777D1B689D0
:1091A40094231307E00F639AE60E88A31305860041
:1091B40033450508ADC99165938565719770FB1FAB
:1091C400E78080E9AA8455D917B9FB1F1309C9CDD3
:1091D4000325090009C59770FB1FE78000F5138577
:1091E400840088C022868145232099009770FB1F44
:1091F400E780801C832709002286CE8588439770E8
:10920400FB1FE780E01483270900A286F240C2A373
:109214006244D2444249B249984305468D450545C6
:1092240005616FA090569165938555719770FB1FEA
:10923400E78080E2AA8431D117B9FB1F130989C6DC
:109244000325090009C59770FB1FE78000EE13850D
:10925400840088C022868145232099009770FB1FD3
:10926400E7808015832709002286CE85884397707E
:10927400FB1FE780E00D83270900A286F240C2A30A
:109284006244D2444249B249984305468D45054556
:1092940005616FA0D04F494582804945C5B5930704
:1092A400C01C63FCA700094582800945F240624462
:1092B400D2444249B24905618280011122CC06CED2
:1092C40026CA4AC84EC62A8425C1AE89916521059D
:1092D40093856571334505089770FB1FE780C0D7F8
:1092E400AA8461D517B9FB1F130909BC032509001A
:1092F40009C59770FB1FE78040E31385840088C08D
:1093040022868145232099009770FB1FE780C00ABD
:10931400832709002286CE8588439770FB1FE78048
:10932400200383270900C2A397B7FB1F83A747B372
:1093340085CF97B7FB1F83C76700958B85CB97B7FE
:10934400FB1F83A767B691CF9843D6236244F240AC
:10935400D2444249B24905468D45054505616FA091
:10936400D04201478146DDB7014589B749453DBF34
:109374009307C01C63FCA700094582800945F2409D
:109384006244D2444249B24905618280011122CC2F
:1093940006CE26CA4AC84EC62A8425C1AE8991651E
:1093A400210593855571334505089770FB1FE780A8
:1093B400A0CAAA8461D517B9FB1F1309A9AE032556
:1093C400090009C59770FB1FE78020D61385840028
:1093D40088C022868145232099009770FB1FE7806F
:1093E400A0FD832709002286CE8588439770FB1F42
:1093F400E78000F683270900C2A397B7FB1F83A762
:1094040027A685CF97B7FB1F83C747F3958B85CBDB
:1094140097B7FB1F83A707A991CF9843D62362442C
:10942400F240D2444249B24905468D45054505619D
:109434006FA0F03501478146DDB7014589B749453D
:109444003DBF9307C01C63F4A7000945828079716E
:1094540022D406D626D24AD04ECE2A842DC1AE8935
:109464009165210593857571334505089770FB1F38
:10947400E78080BEAA840945A9C817B9FB1F130950
:1094840029A20325090009C59770FB1FE780E0C9DD
:109494001385840088C02286814523209900977013
:1094A400FB1FE78060F1832709002286CE8588436D
:1094B4009770FB1FE780C0E983270900C2A397B711
:1094C400FB1F83A7E79989EB0145B25022549254BC
:1094D4000259F2494561828097B7FB1F83C707E6AB
:1094E400958B4945FDD36C001305D030EF30D20B7A
:1094F400B24793F7070FE9DB97B7FB1F83A7479A98
:109504009443D2238D450545EFA030297DBF97B7FD
:10951400FB1F83A7679989CFD2238C43411106C6C9
:109524009770FB1FE780C0E2B24001454101828091
:109534000945828097B7FB1F83A7079785C717B78D
:10954400FB1F03272796894719CF52230C43411148
:1095540006C69770FB1FE780A0DFB24081473E85B7
:109564004101828089473E85828097B7FB1F83A78C
:10957400A79385C717B7FB1F03278792894719CF7E
:1095840052230C43411106C69770FB1FE78040DC51
:10959400B24081473E854101828089473E85828071
:1095A400797126D206D622D44AD04ECE97B4FB1F68
:1095B400938484B68D4783C9240063FAA7000945C0
:1095C400B250225492540259F24945618280982043
:1095D4002A844145E316F7FE9307F4FF93F7F70F48
:1095E400854663E8F60A2E89B1ED99452800EFC057
:1095F4007FA2A0A0914517B5FB1F0345E5D3EFB0AB
:109604004F822800EFD04FB855E993057100130538
:10961400F041EF10B2489C83D1EB8D476318F408F6
:109624004545EFD04FDC59C137761800130606A024
:109634003306C502914517B5FB1F0345E5CFEFA0DF
:109644005FF6ADA01946814528009770FB1FE7809F
:10965400A0D619462C004A859770FB1FE780C0E00E
:1096640039FD19469305F00F28009770FB1FE7801A
:10967400A0D419462C004A859770FB1FE780C0DEF2
:109684001DFD1946CA8528009770FB1FE78040CC52
:109694008DB7630FE400914517B5FB1F0345C5C99A
:1096A40097B7FB1F238B07A6EFA0BFF7014509BFA0
:1096B400C8442C00EF70E00FA0A00DDD238134011D
:1096C40001B797B7FB1F83C767C7918B8DC3411140
:1096D40017A5FB1F1305857C06C6EFC01F93B24078
:1096E400FD5717B7FB1F231CF7A2410182800145D8
:1096F4006FC0BF91FD5717A7FB1F230BF77AF957CC
:1097040017A7FB1FA306F77A97A7FB1FA381077A66
:1097140097A7FB1F238D077897A7FB1F239807782C
:1097240097A7FB1F23A2077897A7FB1F23AC0776F5
:1097340097A7FB1F23A6077697B7FB1F938707A15D
:10974400170700001307E72098C317070000130743
:109754004787D8C317F7FFFF1307675198C717F751
:10976400FFFF1307473CD8C717F7FFFF1307A73EB0
:1097740098CB97F7FFFF9387474317A7FB1F232F28
:10978400F7708280411126C297A4FB1F9384446D15
:109794009C4006C622C495CB2A840D459770FB1FB6
:1097A400E78040ABAA8519C9930700FD1CA18D472A
:1097B40000B13CA19C408823EFA03F9719C42244E8
:1097C400B240924441016FF06FB3B24022449244DC
:1097D4004101828079714AD017A9FB1F1309496896
:1097E4008327090006D622D426D24ECE6383070EE1
:1097F40098338547AA8497B9FB1F9389E99163013C
:10980400F70483C749008DE70D459770FB1FE78078
:1098140060A4AA8501CD930700FD1CA1914704B162
:109824003CA1832709008823EFA03F90EFF00FAD00
:109834000545B250225492540259F249456182803E
:1098440097A7FB1F83A7476689CB9443D22393052D
:10985400E1000545EFC03F8611ED0145EFD0AFB8FB
:109864002A8621C6894517B5FB1F0345E5ACEFA041
:10987400FFB125A81C21858BEDD30545EFD0AFB6EC
:109884009307B0032A8463F1A7045D661306067088
:10989400894517B5FB1F034525AA130444FCEFA013
:1098A4005FD097A7FB1F239387608327090009478D
:1098B40098B383C7490091C797B7FB1F23800786D6
:1098C40085BF2685C135ADB7930700643306F5021D
:1098D40049BF0145B9BF411122C42A840D4506C6BA
:1098E4009770FB1FE78000970DC1930700FD1CA133
:1098F400CD4700B13CA12244B240AA8517A5FB1F65
:109904000345055B41016FA05F82B24022444101DF
:109914008280411122C42A840D4506C69770FB1F1C
:10992400E78040930DC1930700FD1CA1ED4700B1F2
:109934003CA12244B240AA8517A5FB1F0345455705
:1099440041016FA08FFEB2402244410182805A211E
:109954000111896606CE22CC26CA13866600AA8720
:109964006316C7009C4701458C2371A8138606041F
:109974006365E60413865603636FE6001386960058
:10998400630BC7081386A600630DC712A1066309FB
:10999400D7060145A5A8F9769386A6FC3697A9466D
:1099A40033470708E3E7E6FE974602009386060E70
:1099B4003347D72018433697028713861605630763
:1099C400C71893862605E316D7FC1C45802397A762
:1099D400FB1F83C7C74D2285639D07160D459770EE
:1099E400FB1FE7802087AA850DC1930700FD1CA1FA
:1099F400F14700B13CA117A5FB1F0345654B91A29C
:109A04009C4705458C23EFF0AFB60545F240624410
:109A1400D2440561828017A7FB1F032767440145D1
:109A240075D79C47882359E985471CB30545EFA0A2
:109A3400404CE1BF1C4597A4FB1F93847447130754
:109A4400E00F80239C20638BE7021307F00F6384ED
:109A5400E70211459760FB1FE780C07FAA8501CD0F
:109A6400930700FD1CA1894700B13CA1A301050097
:109A74008820EFA08FEBF9579CA041BF97A4FB1F50
:109A84009384043E9C400145D1D305E805447D45BB
:109A94004085EFD04F95688613050002EFD0AF9450
:109AA4009C40C8851307B10080B374001306A1005D
:109AB40085450545EFA0E04D89BF2285EFF09FCC99
:109AC400A9B79C476244F240D244882305616FF0F1
:109AD4007FD01C4509458C233DB71C4588232DE5C3
:109AE4006C001305D030EF30222CB247414793F776
:109AF400070FE38CE7F09305B10013056031EF30F5
:109B0400A22A88858545EFA0804901B71C4580239A
:109B140097A7FB1F83C7B73922859DE70D4597603B
:109B2400FB1FE7802073AA85E30105EE930700FD80
:109B34001CA1D14700B13CA197A7FB1F83A74732C3
:109B44008823EFA08FDED1B57933C1B51C458823B6
:109B540019C1C1335DBD85450545EFA0404675B5C6
:109B6400411122C417A4FB1F0344447D06C6158873
:109B740009CC17A5FB1F1305655DEFC06FC84D44E5
:109B8400B24022852244410182800145EFC04FC783
:109B9400C5BF9821937625009377D70F99C2936711
:109BA400270093F6F707131745606354070093E6FD
:109BB40007081378850093F7760F6304080093E78A
:109BC40086009376050299CE93E707029CA163571A
:109BD40007001C2293E7C7001CA282801375A5020C
:109BE4006DF9828093F7F7FD9CA1E34407FE937718
:109BF400A502E5F37DF11C22CD9BF9BF2D45631C25
:109C04000710011126CA4AC84EC606CE22CC982196
:109C1400BE8989472E89B684631EF704DC413284E9
:109C2400983394232207558F8D66938746A0131685
:109C3400576063C9C7029386F69F63DDC602F57752
:109C44009387F75F3E978D47C8453347070863E717
:109C5400E70297460200938626E63347D7201C4343
:109C6400B6978287938766AA630EF608938686B8AA
:109C7400630FD60823900400054525A09760FB1FB9
:109C8400E780A076334605083356360B92A0832529
:109C9400C9001DA01E2109479AA01CA0A1831CB0C5
:109CA4000145F2406244D2444249B249056182808E
:109CB40099479EA01946AA8522859760FB1FE780D5
:109CC4002069F9BF85479EA01C211CA0D1BF05C9EE
:109CD400A1479EA01E211CA01E21A1831CB03E21D1
:109CE4003CA03E21A1833CB05E215CA05E21A18307
:109CF4005CB07E217CA07E21A1837CB055B72390EB
:109D0400040079BF85479EA0DC459C237DBFE147C5
:109D14009EA06146ADBF8280797122D44AD006D616
:109D240026D24ECE52CC56CA3A89982189472E84DF
:109D3400631DF7025C40B684B28503C81700942300
:109D44008D6722083368D800938627A013185860BB
:109D5400630BD8102A8A63CC0601938607A0630B91
:109D6400D802938717A06300F80A854711A81387C0
:109D740037A0630FE80A138767AA8D47E317E8FE45
:109D8400B250225492540259F249624AD24A3E8550
:109D940045618280484432C69760FB1FE780E064D7
:109DA4009D4733450508E36D25FD97AAFB1F938A5C
:109DB4006A1183C70A00B3099900B24563D4370115
:109DC400B5477DBF48442686B3C909084A959760BC
:109DD400FB1FE780E05703C60A0048448145050697
:109DE400330636414E959760FB1FE780E05C97A7EA
:109DF400FB1F83A7670D99E3814759B79C438145AE
:109E0400E5DF528525A0AD47E31C09F6E39AE4FAA1
:109E14001C321822A207D98F58441EA397A7FB1FF0
:109E240083A7870AF1DB9C438545F9D78297E9B775
:109E340017A7FB1F0347B7088D4739D3AD47E31175
:109E440009F49947E39EF4F6484419469760FB1FCA
:109E5400E780005097A7FB1F83A70707D1DF9C4328
:109E6400C1DF8D4579BF17A7FB1F0347C7F4218BBB
:109E74008D4719D7AD47E31509F08547E392F4F40C
:109E8400182293070008E3EDE4EE5C4498A3ADB711
:109E9400411122C4094497A7FB1FA38F87F097A7FA
:109EA400FB1FA38A87F097A7FB1F238687F097A73A
:109EB400FB1F23AB070097A7FB1F238C07FE97A765
:109EC400FB1F2381070097A7FB1F239C07FE97A76F
:109ED400FB1FA38607FEA1471946814517A5FB1F53
:109EE400130585FD06C617A7FB1FA305F7EC9760AE
:109EF400FB1FE780604C97A7FB1F238D87EAB707FA
:109F0400A00017A7FB1F130767EA938707051CC365
:109F1400B707E8035CC397A7FB1F238787E8854738
:109F24006146814517A5FB1F1305853617A7FB1F3F
:109F3400A30BF7E697A7FB1F238787E697A7FB1FCB
:109F4400A38287E697A7FB1F238607F69760FB1F6C
:109F5400E780804613060013814517A5FB1F1305F0
:109F6400252097A7FB1F238F87E297A7FB1FA382B8
:109F740007F49760FB1FE780204497A7FB1F938794
:109F840067DCB240224417070000130767C798C371
:109F940017070000130787D8D8C323A4070041017B
:109FA4008280797122D426D206D64AD04ECE52CCA3
:109FB400A1472E84B28463EBA7001747020013075E
:109FC400A7B03345E5201C41BA9782879307100850
:109FD4006304F51C63ECA70093072004630EF516D5
:109FE400930700086303F518094591A09307200817
:109FF400E31CF5FE8547639BF50208229377250051
:10A0040095E797A7FB1F83C787EB1387F7FF97A5F0
:10A01400FB1F9385E514120792072E97A10750475B
:10A02400BE9585AA9307800F63FBB7006145B250C4
:10A03400225492540259F249624A4561828017AA15
:10A04400FB1F130A6AD783470A0017A9FB1F1309CA
:10A0540029119207CA97C84709C99760FB1FE7806F
:10A06400C00C97A7FB1F238F07E413061400137675
:10A07400F60F916593850571328583490A0032C6CE
:10A084009760FB1FE78040FD83470A009209CA9945
:10A09400920723A6A900CA97C84749D932468145E1
:10A0A4009760FB1FE780403183470A002286A6851C
:10A0B40092073E990325C9009760FB1FE78040295A
:10A0C40097A7FB1F238087E0014595B78947E39F46
:10A0D400F5F41E2217A7FB1F2315F7DEF5B78547F6
:10A0E400E396F5F41C2217A7FB1FA30AF7DCE9BFCC
:10A0F4009947E39DF5F21946A68517A5FB1F13059D
:10A10400A5DB9760FB1FE780A0247DBFA147E39FE9
:10A11400F5F02146A68517A5FB1F130525C9D5B75C
:10A124008547E395F5F01C2217A7FB1FA30DF7C67F
:10A1340061BFE147E39CF5EE6146A68517A5FB1FC9
:10A14400130505157DBF8547E392F5EE1C2217A77D
:10A15400FB1FA300F7D68DBF8547E399F5EC1C22BE
:10A1640017A7FB1F2309F7C485B78547E390F5ECD0
:10A1740097A7FB1F83C747C41387F7FF97A5FB1F48
:10A18400938505FE12072E97920750478820A10752
:10A19400BE95EFF01FA00DBF8547E399F5E897A79B
:10A1A400FB1F83C7E7D1C9BFAA8721472E85636DEB
:10A1B400F7001747020013076793B3C7E7209C43D0
:10A1C400411106C6BA97828713072004638BE708F8
:10A1D40089473E85828017A7FB1F0347E7BD120707
:10A1E40097A7FB1F9387C7F7BA97CC47894785C1C1
:10A1F40017A6FB1F034606CD9760FB1FE78040159B
:10A2040031A097A7FB1F83D7C7CB9EA18147B2403C
:10A214003E854101828097A7FB1F83C757CA1CA1B3
:10A22400F5B7194697A5FB1F938505C9F1B72146D4
:10A2340097A5FB1F938585B7EF909FDBC1BF97A7B9
:10A24400FB1F83C757B6E1BF614697A5FB1F9385E4
:10A2540025045DB797A7FB1F83C7B7C5C9B789474F
:10A264007DB797A7FB1F83C707B59CA1814795B707
:10A274006300053A97A7FB1F9387A7C39823631925
:10A284000738054798A397A7FB1F938767ED89466F
:10A2940098A717A7FB1F231A07EC17A7FB1F130781
:10A2A400A7B394A397A6FB1F9386C6B6D8C7D4C3F7
:10A2B4007D57630CE53413771500854529C717A628
:10A2C400FB1F231C06EA094797A6FB1F9386C6B308
:10A2D40017A6FB1F130656AE98ABD4CBD0CF85463A
:10A2E40017A6FB1F230AE6AC2380E70217A7FB1F70
:10A2F400130707B1D8D394AF2384D70217A7FB1F42
:10A30400231507E88D451377250025C313974500CA
:10A314003E9797A6FB1F938626AF094654C317A8FA
:10A32400FB1F130858A9854610A314A72326070169
:10A3340023150700138715003347070817A8FB1FC9
:10A344002300E8B812073E9710A314A717A6FB1F13
:10A354001306C6AA97A6FB1F9386A6B6890550C303
:10A364002315070054C7B3C505081377450025C353
:10A37400139745003E9797A6FB1F9386E6A80946C8
:10A3840054C317A8FB1F130808A3854610A314A7DA
:10A3940023260701231507001387150033470708F1
:10A3A40017A8FB1F230DE8B012073E9710A314A7AC
:10A3B40017A6FB1F130646A497A6FB1F938636B069
:10A3C400890550C32315070054C7B3C5050813777F
:10A3D400850021CF139745003E9717A6FB1F130650
:10A3E400A6A250C30546894610A717A6FB1F13064D
:10A3F400769C14A32315070050C713871500334711
:10A40400070812073E9714A397A6FB1F9386869E00
:10A4140054C3A14614A797A6FB1F9386E6A98905F2
:10A424002315070054C7B3C505081377050121CFC9
:10A43400139745003E9797A6FB1F9386E69C094613
:10A4440054C317A8FB1F1308E896854610A314A746
:10A454002315070023260701138715003347070830
:10A4640012073E9710A314A717A6FB1F13064698BE
:10A4740097A6FB1F93868693890550C3231507006F
:10A4840054C7B3C505081377050221CF13974500B8
:10A494003E9797A6FB1F93862697094654C317A891
:10A4A400FB1F13086890854610A314A72315070003
:10A4B40023260701138715003347070812073E9721
:10A4C40010A314A717A6FB1F1306069297A6FB1F3B
:10A4D4009386768D890550C32315070054C7B3C5E9
:10A4E40005081377050421CF139745003E9797A6D7
:10A4F400FB1F93866691094654C317A8FB1F1308D4
:10A50400888A854610A314A723150700232607016C
:10A51400138715003347070812073E9710A314A7A3
:10A5240017A6FB1F1306868C97A6FB1F9386869897
:10A53400890550C32315070054C7B3C5050813770D
:10A54400050821CF139745003E9717A6FB1F130656
:10A55400A68B50C35146894610A717A6FB1F1306A6
:10A56400768414A32315070050C7138715003347B7
:10A57400070812073E9714A397A6FB1F93868686A7
:10A5840054C3854614A797A6FB1F938666D08905F6
:10A594002315070054C7B3C505081375051039C939
:10A5A400139745003E9797A6FB1F9386E68554C3F1
:10A5B400094685461795FB1F1305C57E10A314A7EE
:10A5C4002315070048C713871500334707081207E8
:10A5D400BA9717A7FB1F1307E780D8C317A7FB1F5A
:10A5E4001307378D890590A394A723950700D8C72F
:10A5F400B3C505089796FB1F9386C674414617A5F5
:10A60400FB1F1305E5B56F3000421305300345B950
:10A61400014582800111FD1522CC06CE328426CA62
:10A624003E864AC813F8F50FAD4763E8070B3A892D
:10A63400173702001307C74D3348E8208327080063
:10A64400B684BA9782878545EFB0FFB801E5EFF08D
:10A654002FD10145F2406244D244424905618280CF
:10A664008945EFB05FB77DF52285EFE00FBFD5B721
:10A67400914532C6EFB03FB6324669FDCA8526859C
:10A68400EFB01FACEFF0CFCDEFF0AF83EF60A07A67
:10A69400C9B7A14532C6EFB01FB4324645FDCA85DD
:10A6A4002685EFB0FFA92285EFE02FBBEFE0AFB125
:10A6B400EF60407679BFB14532C6EFB0DFB13246C4
:10A6C40051F9CA852685EFB0BFA72285EFE0EFB820
:10A6D400EFE06FAFEF60007475B70945A5BF7971FE
:10A6E4004ECEAE896C0022D426D24AD006D62A8910
:10A6F400B284EF00306E2A840DE1CE854A85EFB036
:10A70400AF8C2A8419E93245268797B6FFFF9386D2
:10A71400260B2D468145EF100006B25022852254A7
:10A7240092540259F24945618280397126DAAE8425
:10A734004C0022DC4AD84ED652D406DEAA8932898D
:10A74400368AEF0030692A8421E9A685630D090061
:10A754009E202C007C84BE207C85930720307C8640
:10A76400930780025C874E85EFB02F832A840DE522
:10A774005946A6851305A100230421019760FB1FF8
:10A78400E78000BD1245528797B6FFFF938666FEA9
:10A7940025462C00EF00307EF25022856254D254BC
:10A7A4004259B259225A21618280797126D2AE84EB
:10A7B4006C0022D44AD04ECE06D6AA893289EF0044
:10A7C40070612A840DE1A6854E85EFB0AF812A849D
:10A7D40019E932454A8797B6FFFF93862600354626
:10A7E400A685EF005079B250228522549254025922
:10A7F400F249456182807547AA876365B7021147AC
:10A8040001456378B702ED1593F5F50F6147636170
:10A81400B702973602009386A632B3C5D520984175
:10A824003697028793F5F50713072005638AE50039
:10A8340001458280C847828088438280884782801D
:10A84400C84382809307F00F630FF506011126CAEF
:10A85400AA841305000222CC4AC84EC652C456C26A
:10A8640006CE2E8AB28AB6893A899760FB1FE780A2
:10A87400609E2A844D450DC8930700FB1CA0A300CD
:10A884005401231144012302340113058400614659
:10A8940063050902CA859760FB1FE78060ABA28548
:10A8A4002685EF909F880145F2406244D244424994
:10A8B400B249224A924A0561828081459760FB1F12
:10A8C400E78080AFE9BF09458280011122CC06CE22
:10A8D4002A844C86D0869780FB1FE780C02405C15C
:10A8E4005425214797A7FB1F938707A5639DE6007F
:10A8F400E82378009306E0070146A285A137F240D9
:10A90400624405618280C83378009306E0070146FB
:10A91400A285EDB7930700643306F6026F905FBC1F
:10A9240015C1411122C406C62A8408219307D00FF9
:10A9340063E6A700EF909FD8FD571CA0B2402244C5
:10A94400410182808280797122D406D626D24AD0EF
:10A954004ECE9E2509448DEBAE846C00AA893289C3
:10A96400EF0050472A840DE1A6854E85EFA05FF3E2
:10A974002A8419E932454A8797B6FFFF938606F27F
:10A984004D468145EF00305FB250228522549254E7
:10A994000259F249456182801A219307000B631022
:10A9A400F7025C214947639AE700183985476398A1
:10A9B400E7002A2185456F30902A6D47CDBF8280FC
:10A9C40001116C846C0022CC26CA4AC806CE2A899E
:10A9D400B6847085EF0010402A840DE12C004A856E
:10A9E400EFA07FD22A8419E93245268797B6FFFF64
:10A9F400938626CD15462C00EF00F057F2402285B1
:10AA04006244D244424905618280797193072030BF
:10AA14006C8470857C862C0093078002014606D6E0
:10AA24005C87EFF09FD0B25045618280C177797125
:10AA340085073EC4894726D27C86AE84930780026C
:10AA44004C0022D44AD006D62A895C87EF0090387D
:10AA54002A840DE12C004A85EFA0FFE12A8419E93C
:10AA64001245268797B6FFFF938626DE45462C00BF
:10AA7400EF007050B250228522549254025945611D
:10AA84008280B28605466FF05FCA797126D2AE84A1
:10AA94006C0022D44AD04ECE06D6AA893289EF0061
:10AAA40070332A840DE1A6854E85EFA07FBD2A84EC
:10AAB40019E932454A8797B6FFFF938626BB0D46B0
:10AAC400A685EF00504BB25022852254925402596D
:10AAD400F249456182807971930720206C847085E6
:10AAE4007C862C0093078002014606D65C87EFF033
:10AAF400DFC3B25045618280011122CC26CA4AC804
:10AB040006CE2A84AE84328936C69780FB1FE7803E
:10AB1400800115C95025A146324797A7FB1F93878B
:10AB2400A781631DD600E823CA862686A2856244CF
:10AB3400F240D244424905616FF0DFD0C833CA867F
:10AB44002686A285EDB7F2406244D24442490545C7
:10AB5400056182806FF0BFB86FF07FB86FF0FFC4FB
:10AB64006FF0BFC479714ECEAE896C0022D426D268
:10AB74004AD006D62A89B284EF00D0252A840DE172
:10AB8400CE854A85EFA0DFC72A8419E93245268796
:10AB940097B6FFFF938646C63D468145EF00B03D1C
:10ABA400B2502285225492540259F249456182805E
:10ABB400B28601466FF07FB7011122CC2E846C005F
:10ABC40026CA06CEAA84EF00F020DD476309F5000B
:10ABD400930710101EA4A2852685EFA07FCCF24017
:10ABE4006244D24405618280239405006FF0BFD58E
:10ABF400E5BF1797FB1F0347A731854763F8E702B3
:10AC0400011122CC2E846C0026CA06CEAA84EF0041
:10AC1400701C01E9930700101EA4A2852685EFA0ED
:10AC24003FC8F2406244D244056182805945828023
:10AC34009797FB1F23AEA72882809797FB1F23A714
:10AC4400A7288280011122CC26CA06CE2A84AE848B
:10AC54009780FB1FE78020EDA6852285EFA04FF6A5
:10AC640005E9228564869780FB1FE780C0EB0DC150
:10AC7400542521479797FB1F9387076C639FE60032
:10AC8400E82378009306F0070146A285EFF09FBB06
:10AC9400F2406244D24405618280C833DDB77971E1
:10ACA40022D44AD0AE8706D6BA8526D24ECE754770
:10ACB400328436896364F7042147636CF7001547CF
:10ACC4006388E7021947638DE708C167FD17854468
:10ACD4001DA037061400DD1713060620B317F0284D
:10ACE4007D8E49EE19677D8F25EB93F71710F1DF01
:10ACF400C167FD1789446316F40221A813F7F70707
:10AD040093062005E313D7FC41677D17631EE60411
:10AD14008D442EC6EFA08FEEB245330495403344E4
:10AD240004083385840033450508EF30D000AA8732
:10AD3400B3C9040821C963040900231089002254FB
:10AD4400B25092540259B3053041F2493E854561EF
:10AD54001753FB1F6700E34AC167FD17954461BFA2
:10AD6400C167FD179D4441BF1307200D8D44E39A2D
:10AD7400E7FA1304C6003344040865B7C167FD1736
:10AD84008D4495BFB250225492540259F249456100
:10AD94008280011122CC26CA06CED0212E8413072C
:10ADA400000281469945AA84DD3D2AC621C51E209C
:10ADB4005020930554007C803E207C8189477C820E
:10ADC400930780025C839750FB1FE78060585C20E8
:10ADD4008A8526857C84EFA0BF952A8411C53245D7
:10ADE4009750FB1FE7806034F24022856244D244CE
:10ADF400056182804D44CDBF397122DC26DA4AD800
:10AE040006DE89472A84AE8436896306F600C14784
:10AE140009456315F60432C6A9C04C082285EF0023
:10AE2400607B324605EDC1778507A6851305D10100
:10AE34003ECC230EC1009750FB1FE78060512C08C5
:10AE44002285813F01ED52454A8797B6FFFF9386DD
:10AE5400C68C1D462C08EF0010120145F2506254B6
:10AE6400D254425921618280397126DA4AD84ED6A9
:10AE74003289AE893686BA84814613071002D945D1
:10AE840022DC06DE2A8432C6EFF07FE12ACE1DCD15
:10AE94003246A685231A3101F084231B21019750E1
:10AEA400FB1FE780E04A22854C08EFA01FA92A84F3
:10AEB40011C572459750FB1FE7802027F250228569
:10AEC4006254D2544259B259216182804D44FDB733
:10AED400011122CC06CE26CADD472A84639FF508D9
:10AEE4005439B1441C49B38696023287B6979043CD
:10AEF40014436306D6020A20230601006C00EFA067
:10AF04007FA70824B165938505B8EF904FBAE5474C
:10AF14003CA097B7FFFF9387A7A55CC091A85623D1
:10AF2400D223E31AD6FC88470C479750FB1FE780CF
:10AF3400A053AA870A2089E7230601006C00C1B741
:10AF44005C385828850793F7F70F5CB863F4E70279
:10AF5400B38797021848BA979847D623B2238E230B
:10AF6400213751F90824B165938505B8EF902FB4C2
:10AF7400D94431A87C285C86D1B70A21AE846C0000
:10AF840023060100EFA01F9F8547E39CF4F6F240DF
:10AF940062442685D24405618280011122CC06CE0A
:10AFA40026CADD472A840A216398F508EFA00FC555
:10AFB400522C3E284E286D162A963346060833072F
:10AFC400F64052ACAA86334707080A206372B706D4
:10AFD4001388C6FFB388E54063D40803AE97918F06
:10AFE400B3C607081C4C0E283E97EFF0FFE709EDA7
:10AFF4000824B165938505B8EF906FABD944B1A02F
:10B00400ED16B3C60608F9BF0A20230601006C003A
:10B01400EFA05F960824B165938505B8EF902FA93A
:10B02400E5473CA097B7FFFF938787945CC0F9B7C7
:10B0340085475C866C00E9BFAE846C002306010082
:10B04400EFA05F938547E397F4FCF24062442685C2
:10B05400D24405618280397126DAAE842C0022DC68
:10B064004AD84ED606DE2A89B289AD232A8431E530
:10B074004A85EFA0AFB8D6206D1563C4A600B346C9
:10B0840005089844B2208E204A85EFF0FFDD2A841B
:10B094000DE53146A6850808230601009750FB1FDD
:10B0A400E780002BBE2022454E8797B6FFFF93868C
:10B0B400C6855D466C00FC867D2DF2502285625467
:10B0C400D2544259B2592161828071B769B77971FA
:10B0D40022D406D626D24AD04ECE52CC56CA5AC80C
:10B0E4000944C1CD3289094449CAAE84BA8A2A8A3C
:10B0F400368BEFA0AFB01387440081477115162338
:10B1040063DEA608850793F7F70F3107E319F9FE05
:10B114008A855285C1212A842DE131453305A9024E
:10B124009165938515704D449750FB1FE780C0F2DD
:10B13400AA8921C531463306C902A6859750FB1F4B
:10B14400E78000219844D620B2208E205285EFF06B
:10B15400BFD12A8415ED02458547568797A6FFFF80
:10B164009386A67A5D464C005C824EC42306210178
:10B17400A306010023076101FD2BB250228522544E
:10B1840092540259F249624AD24A424B4561828042
:10B194004E859750FB1FE78040F9C5B76D44F1BF5A
:10B1A40079714ECEAE89C16526D20147AA848946FB
:10B1B4001796FB1F1306C6C2FD15054522D406D6F5
:10B1C4004AD0EF101001054429C92A891307300217
:10B1D40081461146F5452685EFF07FAC2AC65544D5
:10B1E4000DCD0357A900CE86014678841147788592
:10B1F400054718A1B2472C002685A38007003247D3
:10B20400FD573CA332473CB3EF10E0712A8411C5CB
:10B2140032459750FB1FE78040F1B25022852254FB
:10B2240092540259F24945618280411106C6EFF0F9
:10B234008FDC19C5B24041011753FB1F6700E3EED1
:10B24400B24041018280011106CE2AC6EFA04F818F
:10B25400324591459797FB1F23AC07C69797FB1F71
:10B2640023A607C69797FB1FA388A70CEF30C02718
:10B27400F24005616F20700F79714AD006D622D44E
:10B2840026D201499397556063D807041795FB1F8D
:10B294000345950A2E899750FB1FE780A0012A8455
:10B2A4005DC518219307000A6310F70A85474C0807
:10B2B400DC85EFA06F88AA841DC59C8599C70844C6
:10B2C40009C59750FB1FE78040E62A208545EF30EB
:10B2D4000019CD47639AF406B250225492544A8519
:10B2E4000259456182808347610191CF714763634D
:10B2F400F7064D476378F7069386C7FE13073014A5
:10B304003357D74825C31797FB1F032727BC01C70B
:10B31400034751012DCB9C8599C7084409C5975013
:10B32400FB1FE78080E05247B7070001938707F0CF
:10B334007D8FB7071200938707106307F700034751
:10B344006101ED476302F70A2285EF80FFD81319E4
:10B35400F96859B7138717FE1377F70F930600029E
:10B36400E3F3E6FA858B9DCB9797FB1F83A747B63C
:10B37400A5C72A201306B1004C0882979C85AA848D
:10B38400ADEBD5D099B75C8699472308F1002A2004
:10B394006C0023170100EFA0CF9CB5BF9797FB1F4C
:10B3A40083A7C7B285CB2A201306B1004C08829725
:10B3B400AA8435D183475101E39107F02308910012
:10B3C400834761012A206C005C8623170100EFA0EB
:10B3D4004F99E5B59944F9BF9C8599C7084409C5B7
:10B3E4009750FB1FE78060D42A208545EF30200763
:10B3F400A1BF084459D59750FB1FE78000D351B72C
:10B404005D71A2C4A6C286C6CAC04EDE52DC56DA3C
:10B414005AD85ED6A5472A84B2846392F50E834730
:10B4240045021A22322285072302F5029307F7FF09
:10B43400B307F602D440B3C70708B697542503CB25
:10B44400070003C917008547638BF6049317890027
:10B45400B3E7670141677D17638AE70A1A2863F730
:10B46400E70A50248507B3C7070885467EA40A2047
:10B474009305E400631BD6007C84930720307C860C
:10B484009307800278855C872C00EFA00FB1082415
:10B49400B165938505B8EF809FE159458DA83307C1
:10B4A400C702239004008149014A930B3501B34A32
:10B4B4000708E3FD59F9B620DC402C28138659000F
:10B4C400ED163E965E85B3C60608EF907FDE1DC17D
:10B4D400630B3A01C840B220B30535015295975029
:10B4E400FB1FE780E0E6BE203E9A9E20334A0A080E
:10B4F40085079EA0BE20BE99B3C909085DBF582226
:10B50400A9476311F7028347450289CF0145B64035
:10B51400264496440649F259625AD25A425BB25BB7
:10B52400616182803428130934014A86894517955C
:10B53400FB1F1305258EEF90BFD739ED34284A86BB
:10B5440089451795FB1F1305A58CEF907FD629E538
:10B5540034284A8689451795FB1F1305258BEF90E0
:10B564003FD51DE934284A8689451795FB1F1305E5
:10B57400A589EF90FFD30DE1DC2009476380E70242
:10B58400ED1793F7F70F29476368F70013079048FF
:10B59400B357F700858B99E3054595BF834744026C
:10B5A40085072302F402BE2075B5411122C406C6E4
:10B5B4002E849770FB1FE780C04C09C93C25138774
:10B5C40017006315E40093F707F83CA5B240224442
:10B5D40041018280411122C406C62E849770FB1F4C
:10B5E400E780204A1DC111C008C01C251307E00FC5
:10B5F4005D456388E7001307F00F59456393E7003F
:10B604000145B2402244410182800945DDBF411118
:10B6140022C42A84210526C206C64AC0EFF04FB0D0
:10B624002420A51493F4D40F81E858248547631D7E
:10B63400F7041C483149A1E3FD57230104001CB45D
:10B64400230204021305C4002244B2409244024976
:10B654006146814541011753FB1F6700E3D5B3875A
:10B6640024033E95084509C59750FB1FE780E0ABCE
:10B67400850493F4F40F5C280848E3E2F4FE975041
:10B68400FB1FE78080AA4DBF084C75F975B74111BF
:10B6940022C4416406C626C29307E4FF6301F5028F
:10B6A400AA849DE19770FB1FE780A03D09E913057B
:10B6B400F4FF9770FB1FE780C03C11C106A1B240A4
:10B6C400224492444101828085476392F504977035
:10B6D400FB1FE780003B2A847DD1FD571EA11C245B
:10B6E4001307F00F6382E7021307E00F6389E70093
:10B6F4003420083401475146A685EFF0AF942285E3
:10B70400EFF0FFF0FD571CA4230504004DBF89474B
:10B71400E397F5FA8545EF40C04655F126859770C5
:10B72400FB1FE78000362A845DF951BF21C5011152
:10B7340022CC06CE18259307F00F2A846308F7025B
:10B7440034210E21083501475D46EFF0AF8F3820D4
:10B75400E1476318F7000A206C0023060100EFA0FC
:10B764006FA1F9571CA42285EFF07FEAF2406244EE
:10B774000561828082809307F00F6306F70601114A
:10B7840022CC26CA2A844AC84EC652C4B689328AF2
:10B794003A8993068500AE847946AA851705000088
:10B7A400130505F906CEEFF0EF96A3042401230157
:10B7B40044012322340185C01305C4006244F240CD
:10B7C4004249B249224AA685D244614605611753CB
:10B7D400FB1F6700E3B7F2406244D2444249B249D6
:10B7E400224A0561828082809787FB1F2386A76E89
:10B7F4008280411122C406C695472A846391F506C6
:10B8040083474502854685072302F5021E225842D6
:10B814003022FD17B3C70708631ED602B3C7E7205B
:10B8240098239C330145A207D98F7A2463F0E70259
:10B834000A2085075EA49305C400EF90DFEC08247A
:10B84400B165938505B8EF809FA65945B24022445F
:10B8540041018280C946B387D702BA97D1B758222B
:10B86400A9470545E314F7FE0345440213351500C3
:10B87400F1BF411122C406C69D472A846396F5048C
:10B884008347450285072302F5021E225842FD170D
:10B89400B3C7E72098239C33A207D98F7A250145A3
:10B8A40063F0E7020A2085075EA49305C400EFF065
:10B8B4004FCE0824B165938505B8EF805F9F594545
:10B8C400B2402244410182805822A9470545E31928
:10B8D400F7FE0345440213351500DDB7411122C4B8
:10B8E40026C206C6B5472A84B2846394F504834706
:10B8F400450285072302F5020A21EF903FB09E20FE
:10B904001307F5FF014563C1E7027A240A20930572
:10B91400C400BA977EA4EF90FFEC0824B165938528
:10B9240005B8EF80DF985945B24022449244410162
:10B93400828058229D470545E318F7FE03454402DB
:10B9440013351500D5B7411122C406C6C5472A844C
:10B954006390F5061E223A22FD17B387E7020347D8
:10B96400450205072302E5025842B3C707083E977C
:10B974003C333823A207D98F41677D176397E700CB
:10B984000145B240224441018280138717005AA521
:10B994007A25E3F7E7FE9305C5000A21EF90BFED92
:10B9A4000824B165938505B8EF807F905945D1BFD0
:10B9B4005822A9470545E316F7FC0345440213350D
:10B9C4001500C1B7011126CA4AC84EC656C206CED2
:10B9D40022CC52C4BC211547AA8A2E89B289B684C6
:10B9E400639EE7023686CE854A85EFF09FE02A847F
:10B9F400631E05108547034599006393F910D82009
:10BA0400A9476319F70C054A8346290003459900A1
:10BA140001476946D685EFE0FFE2F9A83547638C14
:10BA2400E7086361F7041D47638BE7062547638EC8
:10BA3400E706A547638FF90A05440345990026875D
:10BA4400CE860146D685EFE0FFDF054A19E5CE85AF
:10BA54002685EFE05FDA133A15005DD4D947630613
:10BA6400F40259A84547638EE7045D47E393E7FC76
:10BA7400D82585473686CE854A85631AF704EFF0C4
:10BA84002FC58547054AE306F5FAF2406244D244DD
:10BA94004249B249924A5285224A056182803686D9
:10BAA400CE854A85EFF0FFDC99B73686CE854A8588
:10BAB400EFF01F952DBF3686CE854A85EFF01FE245
:10BAC4003DB73686CE854A85EFF0FFE70DB7EFF038
:10BAD400CFCC45BF268785460146D685EFE09FD665
:10BAE400E31305F285452685EFE0FFD0133A1500F0
:10BAF40021BF9E20B1F3054A4A85EFF05FB171B7CB
:10BB0400A547E39CF9F29E208DFBF5BDA547E3967E
:10BB1400F9F29E20E39307F2054A89B79E21639FB9
:10BB2400071C397126DA4ED652D406DE22DC4AD8F6
:10BB3400A021ED47AA89AE84328A6315F4021787DF
:10BB4400FB1F034767399307F00F0144631FF70492
:10BB54009947F2506254D2544259B259225A3E85FE
:10BB640021618280F5476311F4089786FB1F83C621
:10BB7400A6361307F00F9947E38DE6FC9770FB1F79
:10BB8400E78020F02A8415C1302505C2931746604A
:10BB940063D40700814775BFF5454E85EFE0FFD2BA
:10BBA4003C2493E707F83CA4F5B7D62090448C30A6
:10BBB40088203800EF901FDDAA8741FDB4203800AB
:10BBC4000146CE851785FB1F03450531EFE09FC76E
:10BBD400AA8741F1B24799C323000A00BC207547E4
:10BBE400E39AE7FA69F07DB79770FB1FE78060E995
:10BBF4002A894DD185476317F404CE208844300048
:10BC0400EF90BF81AA8731F58347290015476382E6
:10BC1400E702E51793F7F70FC14663E1F60433171C
:10BC2400F0281377574411E7639AD7028327090151
:10BC340095C7B0203400CA854E85EFF0BFD82300E5
:10BC4400AA0089BF38219147E31587F05841E302E0
:10BC540007F0CE208844300002976DB70345990061
:10BC64009787FB1F83C7576D6381A702B4203800F1
:10BC74000146CE85EFE01FBD2A8409E9AC202800E7
:10BC8400EFE07FB719C123000A00014403472900EC
:10BC94008D476318F7043C840357C90063F4E70035
:10BCA4002316F9008355C9004E85EFE0BFF91787C5
:10BCB400FB1F0357E737ED4763F5E7028357C900D6
:10BCC400DD4663F0F6029386370063D1E60211661F
:10BCD4009385470013060629B3C505084E85EF80F2
:10BCE400801E4A85EFF0BF92A287A5B51166930521
:10BCF400B00F13060629B355B70ACDB799473E8549
:10BD04008280011106CE26CA4AC822CC4EC652C42D
:10BD14009784FB1F9384446288249307800291656F
:10BD24003305F502938565701789FB1F1309891A7A
:10BD3400334505089740FB1FE780003290249307A2
:10BD4400800281453306F6022320A9009740FB1F99
:10BD5400E7808066832709004D459DCB0144130A83
:10BD64008002FD599C24636DF4021705000013053D
:10BD740025DBEFE0FFEB1705000013054583EF908B
:10BD84006FDA170500001305C590EF30B056014572
:10BD9400F2406244D2444249B249224A0561828057
:10BDA400B307440303250900614681450504137460
:10BDB400F40F3E95231035012301050023143501AA
:10BDC400230505002302050231059740FB1FE78088
:10BDD400A05E49BF014582801787FB1F0347575662
:10BDE400814763E4E7000145828092219386450000
:10BDF4006314A6002E8582808507B685DDB71DC530
:10BE0400411122C406C638219307D00F2A8463EB5C
:10BE1400E7000E2128310147F9465D46EFE09FA275
:10BE2400F9573EA0B24022444101828082801787A4
:10BE3400FB1F0347F7508147FD5663E3E700828009
:10BE440016A12301050085071105C5BF01458280A0
:10BE54009785FB1F938555F79307000285469CA1A0
:10BE6400FD571787FB1F2301F7F61787FB1FA30C4A
:10BE7400F7F41787FB1F2308F7F49787FB1F239317
:10BE8400D7F49787FB1F239707069787FB1F23A1E8
:10BE940007069787FB1F23AB07049787FB1F23A580
:10BEA40007041786FB1F130666F19787FB1F93870A
:10BEB400A7F65CC29787FB1FA38007029787FB1F27
:10BEC4009387C7E9094718A298A398AB2380E70290
:10BED4002388E7021787FB1F1307C7F294A7D0C76D
:10BEE40094AFD8DB1785FB1F1305C5F20D471786E2
:10BEF400FB1F130666F19786FB1F938666EE238C61
:10BF0400E702C8C323950700D0CB239D0700CCCFFD
:10BF1400D4D3238407022395070223A60702239D73
:10BF240007021787FB1F032767FBD8DF9787FB1FD1
:10BF3400938707E2170700001307870B23A0070066
:10BF4400D8C323A407008280411106C6EFF0DFE8BE
:10BF540009C52821B240410182800145E5BF411154
:10BF640022C426C24AC006C6AA842E893284EFF0AF
:10BF7400BFE6AA8711E94165CA857D15EFF0DFE5C3
:10BF8400AA87454581C786A3A0A30145B2402244A0
:10BF9400924402494101828021E309483547639E66
:10BFA4000603011106CE22CC182210322206598E25
:10BFB40032C6B377F64085E7CC452A842EC4EFF029
:10BFC400BFF832460147630EC50022856244A2458C
:10BFD400F24005616FF0BFF82D473A858280130760
:10BFE4000008F24062443A850561828083C80500F6
:10BFF400094863910803DC4103C807009C33A20786
:10C00400B3E707010D681308289063950701894772
:10C014006FF09FF80545828001114EC606CE22CCF2
:10C0240026CA4AC89789FB1F9389F9D903C709000F
:10C034009307F00F630FF7022A892945AE843284EF
:10C044009740FB1FE7800021AA8505C59307100BC5
:10C054001EA12302050002A562442311250166A145
:10C06400F24003C50900D2444249B24905616F80D8
:10C07400CF8BF2406244D2444249B2490561828086
:10C08400411126C2AE849785FB1F83A525E522C4F2
:10C0940006C62A84EFF05FEB098909C92285224488
:10C0A400B240A685924441016FF08F8FB240224482
:10C0B4009244054541018280411122C426C24AC0EE
:10C0C40006C6AA84130445001309850B1E209DC3CC
:10C0D400084409C59740FB1FE780200522853146A7
:10C0E40081459740FB1FE780202D3104231A04FE6D
:10C0F400E31E24FDB2402244FD579EA0024992440F
:10C10400410182809786FB1F83C696239787FB1F76
:10C1140083A747DD01476394E600014582808E23AF
:10C124001386870B6394A5003E85828005071377E9
:10C13400F70FB287CDB7AA871785FB1F032505DB49
:10C1440001C95A216314F700084582800841CDBF14
:10C154008280411106C6EFF01FFE09C50845B240B2
:10C16400410182800145E5BF797122D413844500E1
:10C1740026D24AD052CC5AC82E8A06D64ECE56CA99
:10C184005EC622892287014B814481468147BD4591
:10C19400122345CAB5EE46233E23B286A697B3C7FB
:10C1A4000708050B3107E315BBFEADC49165938504
:10C1B400457026859740FB1FE78000EAAA8B39C9A2
:10C1C4000C44D1C9814A8149522033853B019740AF
:10C1D400FB1FE780E0175E200844BE99B3C9090835
:10C1E4009740FB1FE78060F463980A003109854A91
:10C1F400832589004A84E9F9314681452285850AE7
:10C204009740FB1FE780401B63826A053109CDB765
:10C21400630ED6000145B250225492540259F24999
:10C22400624AD24A424BB24B456182803223E313C5
:10C23400F6FE5223B294B297B3C40408B3C70708F6
:10C244008DB78547E3E367F70545F1B723267A0100
:10C2540023149A00D5BF1309C400854A814949BFF4
:10C26400AA871785FB1F032525C811E1828018457D
:10C274003A276314F700110582800841FDB7411184
:10C2840006C6EFF0FFFD09C50A21B24041018280D4
:10C294000145E5BF411106C6EFF09FFC09C5282101
:10C2A400B240410182804145E5BF41111786FB1F21
:10C2B400130686C322C40042AA8606C62E850147F9
:10C2C4001DCC1C44AE271C406396D5021DC71CC35D
:10C2D40001C92146930544009740FB1FE7804007AE
:10C2E40022859740FB1FE78040E40145B240224489
:10C2F4004101828022873E84E1B71CC2D1BF05453B
:10C30400F5B701119786FB1F938646BE26CAAA84F9
:10C31400884222CC06CE2E8401470DCD52211C41E9
:10C324006315960215C71CC39740FB1FE780E0DF27
:10C334002C002685EFF07FF701E519C0B2471CC039
:10C34400F2406244D244056182802A873E85F1B777
:10C354009CC2D9BF0545EDB7411122C42A84090501
:10C3640006C6EFE0EFDBFD573CB0B240224441018A
:10C374008280411122C4416406C626C29307E4FFA9
:10C384006301F502AA849DE19760FB1FE780807238
:10C3940009E91305F4FF9760FB1FE780A07111C141
:10C3A40006A1B240224492444101828085476392AF
:10C3B400F5049760FB1FE780E06F2A847DD1FD5769
:10C3C4001EA13C201307F00F6382E7021307E00F5E
:10C3D4006389E70028300147F9465146A685EFE016
:10C3E4006FC62285EFF05FF7FD573CA023020400DF
:10C3F4004DBF8947E397F5FA8545EF30807855F1CD
:10C4040026859760FB1FE780E06A2A845DF951BFA7
:10C414005D71A2C4CAC086C6A6C24EDE52DC56DA1C
:10C424005AD82E84AC21F9472A896392F50497607F
:10C43400FB1FE78020682A8405C138219307D00FA9
:10C4440063ECE70028310147F9460146CA85EFE06D
:10C454006FBF2285EFF05FF00145B6402644964455
:10C464000649F259625AD25A425B61618280832A38
:10C474000400B7070001938707F037071200B3F7EA
:10C48400FA0013070710B28981446388E7022EC6B5
:10C494009760FB1FE7800062B245AA8419CD502142
:10C4A40009CE93174660E3C907FA4A85EFE0EFC166
:10C4B400DC2093E707F8DCA045B7178AFB1F130AB3
:10C4C400AA9003470A009307F00F1945E307F7F80A
:10C4D400E147E3E4B7F893D71500FD1717170200F7
:10C4E40013070772B3E7E72003A80700E30708F67A
:10C4F40003AB4700E3030BF6B3CA0A0863850A00DB
:10C50400C947E39CF5F4562010440C300820380841
:10C51400029821F52C084A85029B1DCD183015FF81
:10C524003820230AA100B9472308E1006314F70265
:10C53400E24798239C33A207D98F0C084A85FC81D3
:10C54400EF902F8211D914080546D9454A85EFE0AA
:10C55400AFDA21B7BC84D5B734209147E38EF6EE29
:10C5640003450A0038080146CA85EFE0AFADE3167B
:10C5740005EE2C202808EFE00FA819C1238009003C
:10C584001840B7070001938707F07D8FB7071200A3
:10C5940093870710E302F7ECE38004EC3C2021BF0F
:10C5A400411122C406C62E849760FB1FE780805089
:10C5B40009C95C21138717006315E40093F707F892
:10C5C4005CA1B240224441018280397152D42E8A46
:10C5D4004ED69305E100AA89528522DC4AD856D268
:10C5E4005AD05ECE06DE26DA3289368BBA8BBE8A04
:10C5F4009760FB1FE780804E054425C1AA842887E5
:10C604003944EFF05FB331C90328450063070804D8
:10C61400D6875E87DA864A86A6854E8502982A845E
:10C624000DED9307E00F638AFA0298208947631699
:10C63400F702DC4098239C33A207D98F0D671307B8
:10C644002790639CE7008347190003460900D285BD
:10C65400A2075D8E4E85EFF03F9CF2502285625416
:10C66400D2544259B259225A925A025BF24B216176
:10C674008280797122D422214ECEAA89228556CA7B
:10C6840006D626D24AD052CC5AC85EC662C4AE8AF6
:10C69400EFF05FA705E52285EF902FF5594411E1EE
:10C6A4000144B2502285225492540259F249624AFA
:10C6B400D24A424BB24B224C4561828003C7890067
:10C6C40085476307F700EFF03F9F03D52900E9B7DB
:10C6D400AA85AA8413858900EFF01FA92A8415CDA1
:10C6E400FA209624D044CE2003D52900E147EFF068
:10C6F400DFEDD9472A846318F50023A604002685B4
:10C70400EFF09F9B71BF19E1268575BFDE2026855A
:10C714002390FA00EFF05F9A69B713894400014A45
:10C72400B94B594C3D4B8355090085CDE14763070F
:10C734007A010357C900D94711E3E1470357290098
:10C74400835649000326890003D52900EFF0FFE74B
:10C754002A846310850323240900050A3109E3149C
:10C764006AFD2685EFF05F952DD0D947E31BF4F2DF
:10C7740005BF65D5835709002390FA00F9BF01115D
:10C7840070879307E00F1306E1000147894606CE40
:10C79400EFF0BFE3F2400561828079714AD003591A
:10C7A400850022D426D22A84AE844A8593052101A9
:10C7B40006D69760FB1FE780603279C51C252AC620
:10C7C40093F707029DC7A881EFF0BF98B245AA87E7
:10C7D40011E9239024013945B2502254925402594C
:10C7E400456182802A204946829701C51E249EA065
:10C7F400E5B7035924004A85EFF0DF9001ED416568
:10C804007D15EFF03F9009E51E2425459EA0E9B76C
:10C8140023102501130745008147BD46122339EE35
:10C824003147B387E7029305840031462EC691074A
:10C834003E959740FB1FE780A0B1B24531464808BA
:10C844009740FB1FE780C0B052242A20414781460D
:10C85400DD45EFE0CFC42ACE09E51E2445459EA060
:10C86400A5BF0C4852249740FB1FE78060AE2A20E6
:10C874004C08EF904FD32DD15945B9BF85073107E7
:10C88400E39ED7F825459DB705458DB7797122D428
:10C894002A840A254AD02E899305E1004ECE06D675
:10C8A40026D2B2899760FB1FE78040232DC91C253F
:10C8B400AA8493F707028DEF18389307200511E334
:10C8C4005C20362450440E242A200147EFF0FFCF89
:10C8D40021E11C38B9E32A20EF902FC9AA875945D2
:10C8E4008DCFB250225492540259F249456182804C
:10C8F4002887EFF01F86AA870DC52A204946A685FA
:10C9040082975DD91E242310F9001C3899E7D1BF02
:10C91400D947E319F5FE238009000145D9B7054538
:10C92400D5B73945C5B7797122D44AD04ECE52CC49
:10C9340056CA06D626D2AA892E8AB28A3689976022
:10C94400FB1FE780201709440DC53C211307E00FA6
:10C95400AA845D44638FE7001307F00F5944639A78
:10C96400E70063920A02D2854E85EF900FCC2A84A9
:10C9740021C1B2502285225492540259F249624A8A
:10C98400D24A4561828003550A009305E1002317CA
:10C9940001009760FB1FE78060142887EFF09F8FEA
:10C9A400AA8505464E85EF20107D2A844DDDD1B73A
:10C9B4009307F00FE30FF9FA938624007946A685CE
:10C9C40017F5FFFF1305E543EFD0DFF4A38124013E
:10C9D4004DB7797126D24ECE52CC56CA5AC85EC6CD
:10C9E40006D622D44AD062C466C2AA8A2E8BB28BDF
:10C9F400368ABA899774FB1F83A4044FB9C0804454
:10CA040083DC44000149035CA4006314990184405D
:10CA1400F5B73E2463F75701050941043349090872
:10CA2400EDB7E36BFBFE63090A000C204840D28695
:10CA34005E86EF80FF876DD16384090023908901AE
:10CA4400A284B25022540259F249624AD24A424B59
:10CA5400B24B224C924C26859254456182809A2195
:10CA6400B621854763E3E60429C3D4210111138663
:10CA7400550022CC1775FB1F1305C5392E84894533
:10CA840006CE32C6EF80DF82C14719C95420324630
:10CA94002E200A200147EFF0DFF3A94711C1814797
:10CAA400F24062443E85056182803E8582802E8606
:10CAB4000A22AE21854763E1A50219CD5422411112
:10CAC4000147150606C6EFF0DFF0A94711C18147FB
:10CAD400B2403E85410182803E8582802E860A22B4
:10CAE400AE21854763E1A50219CD542241110147C6
:10CAF400150606C6EFF0FFEDA94711C18147B24004
:10CB04003E85410182803E85828039714ED6BE21A8
:10CB140083D9050006DE22DC26DA4AD852D456D25E
:10CB24005AD05ECE62CC66CA63E437152A8A0545BC
:10CB340063830912416BAE8A2314010002C60144C7
:10CB440001497D1B894B054CC94C83D52A000147FB
:10CB5400814601464E8523130100EFF09FE7AA8426
:10CB640071C509EC13072002930661005A869545A6
:10CB74005285EFE0CF922A84630E050E38849C2000
:10CB840025C718856301870541476394E70ABE24D6
:10CB94004146130524001CA0BE24A1831CB0CC4034
:10CBA4009730FB1FE780C07A49043C848507B3C7EC
:10CBB40007087C8463FC2707BE246389670785090B
:10CBC400B3C9090859B763967707BE240946130504
:10CBD40024001CA0BE24A1831CB0CC409730FB1FB2
:10CBE400E78000771104D1B722C603596100B82445
:10CBF40013052400638F77013359990323057101C9
:10CC040018A0BE244146A1831CB0CC401379F90F6F
:10CC140041BF2305810118A0BE24135929001379AB
:10CC2400F90FA1831CB0CC4009464DBF3C84294573
:10CC34009DC32C005285EF80DFE609CD34001546F4
:10CC4400D9455285EFD05FEB11C532459730FB1FB4
:10CC5400E780A04D0145F2506254D2544259B25972
:10CC6400225A925A025BF24B624CD24C216182806E
:10CC74000545D5B74545C5B71777FB1F0347472972
:10CC8400854763F7E706011122CC26CA4AC806CEB7
:10CC94002A84AE8432899760FB1FE780A0E111C526
:10CCA40038219307E00F6307F704631B090022850B
:10CCB4006244F2404249A685D24405616F90AF9325
:10CCC4008A209305E100231701009760FB1FE7808A
:10CCD400E0E02887EFF00FDCAA8505462285EF20E7
:10CCE400904971D5F2406244D24442490561828040
:10CCF400594582805D45FDB7411122C406C626C24E
:10CD040093F705022A84328585C3EFF0AFD8AA854C
:10CD140005462285EF20304695476305F500BD475B
:10CD24006315F502214515A093F78500B6849DC3CC
:10CD3400EFF04FD6AA8505462285EF20D04309C5DA
:10CD44009C3481C79C2491C30145B240224492443F
:10CD5400410182809397456063D70700EFF08FD33A
:10CD6400AA850146D1BF89890D45F9FDF9BF7971BD
:10CD7400AE8622D42A848A229305E10106D636C6D9
:10CD84009760FB1FE78080D511C90C2522852254AA
:10CD9400B246B087B25045616FF01FF6B2502254CC
:10CDA400054545618280411122C406C693F70502F8
:10CDB4002A8432858DC3EFF0EFCDAA8505462285FE
:10CDC400EF20703B1547AA876305E5003D47631DC7
:10CDD400E502A14715A893F7850099CBEFF08FCB17
:10CDE400AA85054622852244B24041016F20B0380D
:10CDF4001397456063570700EFF0CFC9AA85014632
:10CE0400D5B7898991E18D47B24022443E854101DD
:10CE140082807971AE8622D42A848A229305E10124
:10CE240036C606D69760FB1FE78040CBB24609C9D9
:10CE34000C2522852254B087B25045616FF0BFF6AD
:10CE4400B25022540545456182803E25797141677F
:10CE540022D426D24AD04ECE06D6231701007D17FF
:10CE6400AA84328436898149638DE7009420D040B6
:10CE7400138517001307E10033450508EFF07FB56C
:10CE8400AA899420D04089451775FB1F130585F89E
:10CE9400EF800FC215C5A2242285EFF04FBE09C54D
:10CEA4007D142A9433440408630409002310890080
:10CEB400B2502254925402594E85F24945618280FF
:10CEC4009420D04089451775FB1F130565F4EF8046
:10CED4002FBE71F19420D04089451775FB1F1305AF
:10CEE400A5F2EF80EFBC11C9E38809FA3C87E3950A
:10CEF40087FA03D4A9007D1475B7A22475B73971D4
:10CF040022DC26DA4AD84ED652D456D25AD05ECE35
:10CF140006DEBE8B9C252A8AAE84C18BB28A3684F7
:10CF24003A89C289468B9DEF942089476383F6062C
:10CF34005685EFF04FA005CD8328050063890802CC
:10CF440022866254F250925A5A88CE87025BB259B2
:10CF54005E87CA86F24B4259A6855285D254225A1C
:10CF6400216182883285EFF0CF9EAA8709ED394589
:10CF7400F2506254D2544259B259225A925A025B24
:10CF8400F24B216182802946A6855285829749DD2C
:10CF9400C5B7DC4003C3170098238D6722033363AE
:10CFA400E3001386479013175360E343E6F81386B0
:10CFB400F78F634BE60293862780630FD70863C815
:10CFC400E604F977938707803E9385473343030844
:10CFD400E3E067F62D45E39D0BF8DC449023CC4356
:10CFE4002310C90022851DA2F5779387F76F3E931E
:10CFF4008D473343030863E06712171702001307D2
:10D0040067BA3343E32083270300BA978287938761
:10D014003780E31FF7F02D45E39C0BF4854723107D
:10D02400F900DC4481459C231CA0AA240505334552
:10D0340005089760FB1FE78060AA835709004DE944
:10D0440091072310F9001146814513051400973008
:10D05400FB1FE780603641A82D45E39B0BF0DC44C1
:10D064006C0083C917009823A209B3E9E9001147AA
:10D074002310E9009C234E851CA0DC449C331CB087
:10D084009760FB1FE78080A5AA8425C13086C1650F
:10D094009306E100FD158329C500EFF01FDB09EDC0
:10D0A4009420D04089451775FB1F130565D6EF8082
:10D0B4002FA019E1FD577C8703C709008947631036
:10D0C400F70283A549000946130544009730FB1F66
:10D0D400E78000288357090089072310F9003C875B
:10D0E4003CA0A1833CB0014561B523173101C5BF04
:10D0F40018218907BA972310F9003E251CB03E2554
:10D10400A1833CA010214C41130534009730FB1F30
:10D11400E7800024C9BF2D45E39C0BE42310D9000C
:10D12400DC449C231CA0DC449C331CB06DBFC8446D
:10D134009730FB1FE780602B334705081D45E369E3
:10D1440077E36380EB02B386790163C6E6003307B5
:10D154007741B3490708CC44231039014E86DE9544
:10D1640051B58149CDBF2D45E3940BE0CC445285A4
:10D17400EFE09FDD89472310F90008A0218108B062
:10D184009DB72D45E3960BDE89472310F90049BF6F
:10D194002D45E39F0BDCDC441D472310E900982355
:10D1A40018A0983318B0BA2338A0BA23218338B012
:10D1B400D82358A0FA2358B0FE23A1837CA025B716
:10D1C4005D71A6C2AA842A214EDE52DC56DA5AD8F0
:10D1D4005ED662D466D26AD06ECE86C6A2C4CAC0F7
:10D1E400AE8AC16BEF808FA1130CF5FF2A8A8149A7
:10D1F400977DFB1F938D4D0B977CFB1F938C4CCF1E
:10D20400177BFB1F130B0BCFFD1B334D0C08DE24C8
:10D2140063F6F90083D70D0063CD8701AA209775C3
:10D22400FB1F93856508EF807FA92A841DCD59448F
:10D234002DA89C449305E100B3A7F92003C9170066
:10D244009C2322093369F9004A859760FB1FE78014
:10D25400E088AA851DE923902A0103A54D0009C58C
:10D264009730FB1FE78060EC0544B64022852644D6
:10D2740096440649F259625AD25A425BB25B225C26
:10D28400925C025DF24D6161828083C8440083A692
:10D294000C003087AA206A8881475A87EFF03FC67E
:10D2A4002A8419C923902A0103A54D005DDD973016
:10D2B400FB1FE78080E755BF83A74D0099EFAA20A5
:10D2C400514781465E86BD45EFD07F9D23A2AD00C8
:10D2D40009E523902A01454449BF83D70D0003572C
:10D2E4000B003E97634747013307FA407D1723102D
:10D2F400EB0003A54D0003560B0083A50C003E95DF
:10D3040085099730FB1FE780A00483D70D000357DE
:10D314000B00B3C90908BA972390FD00CDBD39713C
:10D3240026DAAA842A214ED65AD006DE22DC4AD82E
:10D3340052D456D25ECE62CC66CA6AC82E8BEF80B7
:10D34400EF8BAA89D424AE248A2478001386D400CF
:10D35400EFF02FE805C5938BB9FF2A84E51901493D
:10D36400177CFB1F130CCCB8977CFB1F938C8CB8D9
:10D3740033CA090863497901631B09109E242945AE
:10D384002310FB009DA8035DC10083C844008326CD
:10D394000C00AA205288814766876A86A285EFF02E
:10D3A4001FB619C9AE2422859306E1006A86EFF000
:10D3B400DFA92A8461F0C9B783D70C009228E3134C
:10D3C400F6FE83250C00C8489730FB1FE780C00990
:10D3D40071D99779FB1F938929ED83A7490095EFAC
:10D3E400AA204166454781467D169D45EFD03F8B77
:10D3F4001DE19E2445452310FB00F2506254D25493
:10D404004259B259225A925A025BF24B624CD24CA4
:10D41400424D2161828023A2A900AE24835AA40034
:10D4240022859306E1006A86EFF03FA22A84E38313
:10D434000AF883A749001307190033470708CA9756
:10D444002380570183A7490093DA8A0093062900B1
:10D45400BA972380570113073900110983A749009C
:10D46400B3C60608334707083349090811C930878A
:10D47400B69790A383A749002182BA9790A3DDBDF4
:10D48400B697FD5694A383A74900BA9794A3AA20FC
:10D494009775FB1F938545E11359290023902501B6
:10D4A400EF808FEB39D9594589BF411122C406C693
:10D4B40093F705012A84328585C3EFE0BFDDAA8591
:10D4C40005462285EF20204B95476305F500BD47AF
:10D4D400631DF502214515A893F7450099CBEFE0AC
:10D4E4007FDBAA85054622852244B24041016F2094
:10D4F400804893F7050491C7EFE0DFD9AA85014678
:10D50400DDB713C5F5FF05890605B2402244410184
:10D514008280797122D426D252CC06D64AD04ECEFD
:10D5240056CA5AC82A8AAE840144DE206364F400D1
:10D53400014581A083AA04009319140013891900DA
:10D54400B327542103CB0700B3872A01882393050B
:10D55400E1002205336565019750FB1FE780005801
:10D564001DE123806A019C4005453E99034709005B
:10D5740098B3B250225492540259F249624AD24AA0
:10D58400424B456182800C2530875285EFF0FFF1D4
:10D5940001CD9C40BE9903C7090098A39C403E99C5
:10D5A4000347090098B3F1B7050433440408B5BF31
:10D5B4000111AE8722CC2A848A239305E10006CE8A
:10D5C4009750FB1FE780805109C90C2522856244CE
:10D5D4003087F24005616FF05FEDF240624405452B
:10D5E4000561828039715AD02A8B2A2126DA4AD8D9
:10D5F40006DE22DC4ED652D456D25ECE62CC66CA49
:10D60400AE84EF70BFDF2A898346CB008355AB001D
:10D6140003558B0078001306DB00EFF08FBB630526
:10D624000516C16A130AA9FFAA8B01449779FB1F47
:10D634009389098C977CFB1F938C0CC7FD1A6D1979
:10D64400334A0A08035CC10083C58B0003552B00D1
:10D654006286EFF09FE56318051483484B0083A6A8
:10D66400090003552B00528881471777FB1F1307C6
:10D6740067886286DE85EFF09F886316051205CC05
:10D6840083D72C001777FB1F0357C78611076395B1
:10D69400E700A29763C427079775FB1F9385C5C04E
:10D6A400BE2103552B003354F40282A1EF80CFE452
:10D6B40015C1594505A003552B0049478146568697
:10D6C400C545EFD0CFDD23A2AC0015E183D7AB0075
:10D6D40045459EA0F2506254D2544259B259225A3E
:10D6E400925A025BF24B624CD24C21618280977752
:10D6F400FB1F83D7278091072391FC0083A74C004D
:10D7040003D7AB006286A29798A383A74C001307A4
:10D71400140033470708BA9703D7AB009306E10018
:10D724005E85218398A38355AB00176CFB1F130CF4
:10D734006C7CEFF08FF103A74C003C8713062400A8
:10D744003346060832971CA303A74C009306340003
:10D75400A183B3C6060836971CA3AA8B03A54C0065
:10D7640011043344040803560C0083A509002295D0
:10D7740063910B029730FB1FE78080BD83570C0039
:10D78400A29733C4070809F883578B0029459EA044
:10D7940091B79730FB1FE780A0BB83570C003E94E2
:10D7A4003344040845B583D7AB009EA0E31604EECA
:10D7B40083578B009EA039BF1D71A6CACAC8AA840C
:10D7C400035985002A21A2CCCEC6D2C4D6C2DAC05F
:10D7D4005EDE62DC6AD886CE66DA6ED6AE8AEF701A
:10D7E400FFC1130BD5FF01447115138CD400976B43
:10D7F400FB1F938BEB6F176AFB1F130AAA6F177D2E
:10D80400FB1F130D6DAAB3490508635D6411D4248D
:10D81400AE241307E10162864A85EFF08F9BAA8C40
:10D82400630205100359A500B0870C25AA2032C64F
:10D83400EFF0BFC7631D050E83C8440083A60B0029
:10D844003246AA204E8881475287E685EFF02FEBB7
:10D8540079ED15C483570A0003572D008907630225
:10D86400F7069775FB1F938525A4BE21AA20B357FD
:10D87400F4029EA1EF80CFB60DC1594539A8AA2064
:10D8840041664D4781467D16A545EFD04FC1232201
:10D89400AD001DE123902A014545F6406644D64477
:10D8A4004649B649264A964A064BF25B625CD25C0C
:10D8B400425DB25D2561828083570A008907231186
:10D8C400FD0083570A00A29763DE670583274D0096
:10D8D40003D7AC00930D2400A29798A383274D008F
:10D8E40003D7AC000504334404082183A29798A30A
:10D8F40003254D0003560A0083A50B00B3CD0D0884
:10D904006E959730FB1FE780A0A483570A00BE9D45
:10D91400C167FD1733C40D08E309F9EE050933495E
:10D924000908E5B5294515FC23902A01BDB76DDC2E
:10D934000DBF1E21411126C206C622C44AC044415D
:10D9440089EB8947B2402244924402493E85410111
:10D9540082809420D0402A8489451765FB1F1305D3
:10D96400654BEF70FF9411C93C202547E51793F7E9
:10D97400F70F637FF700E147F1B79420D040894562
:10D984001765FB1F1305C548EF709F9271FD55BFC6
:10D994001769FB1F13090943835609008547DDD224
:10D9A4001A203697C166E3CFE6F891659385257012
:10D9B40031459720FB1FE780206AAA84CD4759D1BF
:10D9C400314681459730FB1FE780009F1A2083551D
:10D9D400090001468147B386F500B3C6060863E92A
:10D9E400E70201C62E972310E90023A00400214674
:10D9F400A285138544009730FB1FE7806095176765
:10DA0400FB1F1307674E1C4381CF3E879C43EDBF2A
:10DA140050401395470085072A9636A6054665BFEC
:10DA240004C3814705B7011106CE22CC26CA4AC8D1
:10DA340009E90944F24022856244D244424905611D
:10DA440082802AC6AA84280036896C845085EFF027
:10DA54005FEE2A8465F1E30F09FCBE24F9DB9165CE
:10DA64009385557031459720FB1FE780E05EAA87B8
:10DA740015C1BA249766FB1F9386464723200500E9
:10DA84005AA198422324250101C7BA861843EDBF41
:10DA94009CC24DB74D4479BF9767FB1F9387D7430B
:10DAA40098230DE3054798A3058909CD9766FB1FC5
:10DAB4009386062A414691451765FB1F1305052ADF
:10DAC4006FF07FF6014582809767FB1FA38DA72E19
:10DAD400828041677D176315E5002E856FE02FB5C1
:10DAE400411106C6EFE04FAF09C5FD571EA1230142
:10DAF4000500B24041018280011126CA06CE22CC23
:10DB04004AC88547AA846392F5042685EFE08FDF2F
:10DB140031E941699305F9FF1307E1008946176666
:10DB2400FB1F1306262E0545EFE0BFEA2A847D1964
:10DB340005C44C442685EFF0DFF930872285814601
:10DB4400CA85EFF08FB02A84E5B789476396F5005C
:10DB54008545EF20000355D9F2406244D24442493E
:10DB640005618280EFE04FD56DB7411122C406C62E
:10DB740026C21764FB1F1304247C08349767FB1F19
:10DB840023A207369767FB1F23AC07349767FB1F55
:10DB940023A6073459C59307200C3305F502916574
:10DBA400938515709764FB1F9384C433190533451B
:10DBB40005089720FB1FE780204A10349307200CA8
:10DBC40081453306F60288C019069720FB1FE780BB
:10DBD400A07E9C4018348145938647007D5563EAB6
:10DBE400E5069306800BB306D70201460507FD55EB
:10DBF400B6979766FB1F23A5F62EBE868EA2ACB2FF
:10DC0400ACA22382060005069906E369E6FEF956EE
:10DC140096A399463307D702BA971767FB1F232F9A
:10DC2400F72A17E5FFFF1305E57EEFD00F8117F5FF
:10DC3400FFFF13052597EF708FEF17E5FFFF13051F
:10DC44008573EF10306BB240224492440145410188
:10DC54008280239EA6FE36861388460B2310060078
:10DC6400232406003106E31B06FF85059386860BF5
:10DC7400BDB7411106C622C42A84EFC06FA1EFE0EC
:10DC84002F9D1765FB1F032565259767FB1F238CB5
:10DC94008712EFE0CF999767FB1F238787122244EF
:10DCA400B24017050000130565E541016F1090644B
:10DCB4009397556063DB072E79711765FB1F034546
:10DCC400851022D44AD006D626D24ECE2E8997204D
:10DCD400FB1FE780205E2A8441CD18219307000BA7
:10DCE4006315F70885479764FB1F93846420DC84DD
:10DCF4009C402315010081EFEF00C0759165938569
:10DD040035709720FB1FE780203588C031C96146F4
:10DD140081451765FB1F130525599720FB1FE780D5
:10DD2400A0698349440089476393F90825279764C8
:10DD3400FB1F938464578AA02A20A685EF70DFD244
:10DD4400AA869E202A201A248DEE6363F7001EA45F
:10DD54000E24EFC03FEF2285EFC01FC49C8491C7FF
:10DD64004C2013058400EFD04FCC2285EF60CFB652
:10DD7400B25022549254F2491315F968025945617C
:10DD840082806363F7001EA41E24D9459766FB1F97
:10DD9400938686510D469EA0EFC01FD68D4545DD66
:10DDA4001765FB1F13054550EFD02FC86DB7938738
:10DDB400A9FF93F7F70F4947E36FF7F81707020036
:10DDC400130747DFB3C7E7209C43BA9782879305BD
:10DDD400A1002285EFF0AFD4AA8435DDD94763943E
:10DDE400F40A85092A2093F9F90F9766FB1F938695
:10DDF400A64B4E86D945EFC03FD031DDCE854DB719
:10DE04009305A1002285EFF03F9BF9B78359840065
:10DE14006C004E859750FB1FE78040CCAA842DC12F
:10DE24002A2041669306E10055477D16AD45EFC0B3
:10DE34001FE79769FB1F9389294723A2A900AA8694
:10DE440055CD834844000358E10030862A20A68536
:10DE540081474E87EFF0AF8AAA846312050E2A2009
:10DE6400CE85EF709FDDE30805EE2A20D945CE86E6
:10DE74002D46EFC07FC8AD45E30F05EC4E852DB7A9
:10DE84002315310185441830D147E306F7EC5C20B3
:10DE94009769FB1F938949412A202380F9003C8517
:10DEA400CE85238299002391F900EF708FEBE30470
:10DEB40005EA2A20CE860546D945EFC0FFC3E30C08
:10DEC40005E8854565BF835984006C004E859750ED
:10DED400FB1FE780A0C0AA8445D52A20416693068B
:10DEE400E10059477D16B545EFC07FDB9769FB1FFD
:10DEF4009389893B23A2A900AA8609E51E24C54467
:10DF04007C8551B7834844000358E1003E243086A1
:10DF14002A20A6854E87EFE09FFEAA840DE12A20E1
:10DF2400CE85EF70FFD4E30805E22A20D945CE86DA
:10DF34003546EFC07FBCB545E30F05E081B7D9474F
:10DF440003A549006397F4009720FB1FE780E01DB9
:10DF540019B59720FB1FE780401D1E247C8525B73B
:10DF64009305A1002285EFF0AFA5BDB59305A100EF
:10DF74002285EFF02FE78DB5130691009305A100DC
:10DF84002285EFE0BF9089BD9305A1002285EFE0D3
:10DF9400DF80AA84E31405E4A30401006DBB9305A8
:10DFA400A1002285EFE0EFEC05BD01458280F1CEB2
:10DFB400011156C2AE8A854526CA4EC652C406CE43
:10DFC40022CC4AC82A8AB284B689EF10903BD14742
:10DFD4001DC51767FB1F0347B7F39767FB1F83C76D
:10DFE400F7F2014999E03E89BA871317490017648B
:10DFF400FB1F0324E4F03A94636DF900D547F24023
:10E004006244D2444249B249224A924A3E85056159
:10E01400828036201307040191C605091379F90F8C
:10E024003A84D9BFB1C89565938525C0130500020C
:10E034009720FB1FE780400248C469D11306000201
:10E044008145130909049720FB1FE780E03623006C
:10E05400040023112401231344019C341767FB1F7C
:10E06400032747EA998C1CA45C4491849180C4AF33
:10E0740023A08900814761B72326040023000400FC
:10E084002313440123045401E5B785473E85828068
:10E09400AA869765FB1F83C5B5E71767FB1F032790
:10E0A40027E681476394F5000145828032233A854F
:10E0B40019C2E30CD6FE850793F7F70F4107DDB7C6
:10E0C400AA861766FB1F0346B6E41767FB1F0327E0
:10E0D40027E381476314F600014582802E233A85A5
:10E0E40081C54C23E38BD5FE850793F7F70F4107D2
:10E0F400D5B7AA869765FB1F83C565E11767FB1F24
:10E10400032747E081476394F50001458280122389
:10E114003A8519C2E30CD6FE850793F7F70F41073A
:10E12400DDB7AA861768FB1F034858DE9767FB1FF5
:10E1340083A707DD01476314E80001458280B22309
:10E144003E8509CAF2236317D600D04701C632229E
:10E15400E306B6FE05071377F70FC107E9BF4111C0
:10E1640026C2444522C406C62A8495C0C84409C5AB
:10E174009720FB1FE78060FBC84809C59720FB1F59
:10E18400E780A0FA26859720FB1FE78000FA228506
:10E19400414681459720FB1FE7800022FD571CB4B0
:10E1A400B2402244924441018280011122CC2A844B
:10E1B4002A2106CE2EC6EF102069324622858145DB
:10E1C400EF00505822856244F24005616FF03FF938
:10E1D40005C53E21411122C406C62A8491CBDD45E2
:10E1E400EF00505922852244B24041016FF03FF7BD
:10E1F400B2402244410182808280411122C4B1474D
:10E204001304C5FFB307F40226C29764FB1F93846B
:10E21400240B06C6A697BA276315B702C84315C1CF
:10E224009307F00F6305F6001C21639CC700972039
:10E23400FB1FE78080EFB1473304F402A29423A2CA
:10E244000400B2402244924441018280411122C41C
:10E254002E8426C24946AA848145228506C6972073
:10E26400FB1FE78060158DCCD82C9767FB1F83A715
:10E2740067C91207BA979A231AA0BA23FE233AA0B1
:10E284001767FB1F035747C85AA09A207AA0BA20E1
:10E294001AA4DA203AA4FA205AA49A241EA87AA42A
:10E2A400B24022449244410182802A869765FB1F32
:10E2B40083C515C61768FB1F0328C8C49766FB1FD0
:10E2C40083A606C4014701456393E50082809C222E
:10E2D40081CFDC4691CBDC2F9207C2976316F60000
:10E2E4009307150013F5F70F05071377F70FC1060A
:10E2F400E1BF130600643386C50293069500AA8520
:10E3040017050000130505ED6F608F9D411122C4B0
:10E3140006C62A840835EF606FBAFD571CB4B240B4
:10E32400224441018280011122CC4AC84EC652C403
:10E3340056C25AC006CE26CA2A89AE890144176A33
:10E34400FB1F130ABABC976AFB1F938A6ABB1D4B57
:10E3540083470A006369F404639D09029769FB1FFC
:10E36400938919BB176AFB1F130A8AB9930AF00F22
:10E3740083C709006364F4061144A144228513068B
:10E38400F00FCA850504EFF05FE733440408E31790
:10E3940094FEF2406244D2444249B249224A924A2B
:10E3A400024B0561828083A40A0093174400BE9443
:10E3B4009C208DC3FE20639F270163956901AA20D9
:10E3C400EF10804826854E868145EF00B0372685BC
:10E3D400EFF0FFD805041374F40F9DBF83240A00E3
:10E3E40093174400BE949C208DC39C34638F5701C3
:10E3F400FE20639C27012685EFF05FF12685D14539
:10E40400EF0050372685EFF09FD505041374F40F01
:10E4140085B7C167F917630BF502411122C406C61B
:10E4240085472A846399F50022852244B2408145B8
:10E4340041016FF05FEF89476396F5008545EF1062
:10E4440040747DD1B24022444101828082809D4546
:10E454006FF07FED1765FB1F035505AB828001113B
:10E4640006CE68876C861767FB1F034727AA854774
:10E474006318F70070009305E1000545EF5070251F
:10E48400F24005618280A947631DF6029C31982100
:10E49400A207D98F1EA1BC31B821A207D98F3EA1F2
:10E4A400DC31D821A207D98F5EA1FC31F821A20763
:10E4B400D98F7EA19C359825A207D98F1EA5014529
:10E4C4008280054582809147631EF6009C31982125
:10E4D400A207D98F1EA1BC31B821A207D98F3EA1B2
:10E4E40001458280054582809387C5FF0D47B3C6E9
:10E4F4000708636ED70031473387E7029767FB1F2E
:10E50400938707DCBA97A8A38EA3014582800945A7
:10E514008280930740203355F50A71159767FB1FD6
:10E524002394A79E9767FB1F2384B79E9767FB1FBF
:10E53400A38FB79C8280956541111905938535C0D9
:10E5440006C6334505089720FB1FE780E0B001C9E4
:10E55400B240E95541011723FB1F670083CAB2404B
:10E56400410182809767FB1FA384079A9767FB1F6B
:10E574002380079A9767FB1F238B07989767FB1FD6
:10E58400A38607989767FB1F238207988547411145
:10E594001767FB1FA30BF79606C622C426C22A845C
:10E5A4009767FB1F238307969767FB1F239E079498
:10E5B4009767FB1F23A60794EF10E0311765FB1F35
:10E5C400130505D01306000381459767FB1F2382BB
:10E5D40087949720FB1FE78020DE1764FB1F13043A
:10E5E400A49108209764FB1F938454921DC99565D8
:10E5F400938545C012059720FB1FE780E0A51767A8
:10E60400FB1F2321A79011CD1C30102081459CA015
:10E614009767FB1F238DC78E12069720FB1FE78089
:10E62400A0D99C201765FB1F034585D11764FB1FE8
:10E634001304148E3E951375F50F956508A0938504
:10E6440055C012059720FB1FE78000A19764FB1FAC
:10E654009384048B88C035CD102081451206972001
:10E66400FB1FE78060D598401420814725077D561D
:10E67400639BF604EF106047B1473305F5029565D7
:10E68400938565C0334505089720FB1FE780C09C30
:10E694009767FB1F23A4A7862A8401CDEF10E044CB
:10E6A40031463306C502814522859720FB1FE7804A
:10E6B400A0D02244B2409244170500001305A5D50A
:10E6C40041016F102043850710A393F7F70F41070B
:10E6D40045B79767FB1FA38D07829767FB1FA38727
:10E6E400078249BF411126C206C622C44AC0AE846D
:10E6F4009397556063DB07081769FB1F130969814A
:10E70400034509009720FB1FE780C0BA2A8421C96A
:10E714001821930700096311F7041831CD476314D6
:10E72400F7069756FB1F9386A67E28219C2217681E
:10E73400FB1F0348D88F1306640081450147631803
:10E74400E50291C19CA29C2281CB03450900854529
:10E754009740FB1FE78060262285EF50FF971395B3
:10E76400F468B240224492440249410182800E225C
:10E7740005071377F70FAE9793F7F70F090685454B
:10E78400B3D7070B6DBF0123C1BF13F5150071D9B2
:10E79400EF00105319CD9757FB1F83C7677791CBB1
:10E7A40085451755FB1F0345C5769740FB1FE7803A
:10E7B400C02013C5140075B70547637EC7029C319A
:10E7C4009421A207D58F1EA16399E700BC31B8211B
:10E7D400A207D98F3EA1014582800947E39DE7FE48
:10E7E400BC31B821A207D98F3EA1DC31D821A207C0
:10E7F400D98F5EA1CDB7054582809147631EF6008F
:10E804009C319821A207D98F1EA1BC31B821A2073F
:10E81400D98F3EA101458280054582809147631EC0
:10E82400F6009C319821A207D98F1EA1BC31B821D2
:10E83400A207D98F3EA10145828005458280A14768
:10E844006318F6029C319821A207D98F1EA1BC310E
:10E85400B821A207D98F3EA1DC31D821A207D98FD4
:10E864005EA1FC31F821A207D98F7EA101458280E7
:10E874000545828089476319F6009C319821A207D7
:10E88400D98F1EA101458280054582803E2279717F
:10E894004ECE06D622D426D24AD01307F007AE892C
:10E8A4006371F70209473AC47C86300093F5F50F8B
:10E8B400EF007078B250225492540259F2494561E3
:10E8C40082805A22D9462A89328463F7E6007E225E
:10E8D40063F4F6006379F70023140100300093F524
:10E8E400F90F4A85F1B70A2202C4EFF09F80AA8487
:10E8F40035C5EFF09F9B9C246369F5001146A24641
:10E90400CE854A85EF00F06975B7340026869305F5
:10E91400F00F4A85EFF0AFE975F1A2471A24DC47FE
:10E924009AA33A20BAA35A20DAA37A20FAA3DA20C7
:10E934009AA7DC4495C793F4F90F2286A6854A85E5
:10E944008297C167FD172A86E31BF5FA224599478A
:10E95400F9451CA144A1EFF0DF99A9BF094645B7C9
:10E96400014671BFA947631DF6029C319821A20795
:10E97400D98F1EA1BC31B821A207D98F3EA1DC31A9
:10E98400D821A207D98F5EA1FC31F821A207D98F23
:10E994007EA19C359825A207D98F1EA501458280AA
:10E9A400054582809C211CA19C311CB1BC31B8213D
:10E9B400A207D98F3EA1828023220500D82189474E
:10E9C4006304F70005458280F62101114EC606CE88
:10E9D40022CC26CA4AC80D47AE896379D7049C4520
:10E9E40084339023A033A204D18CB02322049387D0
:10E9F4004400518C639CD7029307C4FF2A89B3C790
:10EA040007086361F70203A5890023119900231005
:10EA14008900F1559710FB1FE780A07E2322A900EF
:10EA2400014531A02285EFF0AFE671FD0545F240C6
:10EA34006244D2444249B24905618280797122D448
:10EA440026D22E8406D64AD01C201947AA84B28521
:10EA54006390E70630202800EFF03FDA0DE92884C0
:10EA6400EFF00FE30C302A890DC92E86171700002A
:10EA74001307E7D134009D452685EF00D0304A8541
:10EA840009468145C1214A85EFF06FED0145B25039
:10EA94002254925402594561828089477C803C8487
:10EAA4000A867C813C857C822685EF00D058F9BF9C
:10EAB40049476395E70232202800EFF05FD861F9F7
:10EAC4001755FB1F1305C57F5E25E9D3183068254C
:10EAD4003C00C9460146A685DD2C4DBF5147639DC8
:10EAE400E70032202800EFF01F9A55F10C30300077
:10EAF4002685EFF0BFD959BF5947639CE7043220FC
:10EB04002800EFF05F9C41F52C842685EFF06FE13F
:10EB140015C9584534851E23B697B3C707081EA3E5
:10EB2400B5D75C47A5D79757FB1F83C7673EB9DFA7
:10EB340085451755FB1F0345C53D9740FB1FE780DF
:10EB4400C0E7A9B789473EC03C840C300A867C8262
:10EB5400A1BF0C30231001000A8681BF5D71A2C4DD
:10EB640056DA86C6A6C2CAC04EDE52DCAA8A8831EC
:10EB74002E8432C6EFF0CFD4B24501ED0144B64045
:10EB84002285264496440649F259625AD25A616152
:10EB94008280230205002311050083490400854770
:10EBA400AA846399F90030202808EFF0FFC02A8472
:10EBB40005491DA09D476391F90418218D47E31F62
:10EBC400F7FA302028080549EFF05FC52A8409E5E3
:10EBD400054681452685BD262685EFF02FF388243A
:10EBE4003C080147CE862286D685D522E30909F85A
:10EBF4002685EFF0CFD661B7CD47639BF900182186
:10EC04009147E31DF7F630202808EFF0BFC645B75B
:10EC1400D547E395F9F6034A05008947E310FAF668
:10EC2400302028080549EFF0FFD32A8455F583578F
:10EC34000102A1EBB8841306F003DC44930607FC3D
:10EC4400B3C60608636AD600B085D94663F6C60023
:10EC5400B486D94563EDD500BAA30145EF00D03E93
:10EC6400054903560102D2852685AD2CB5B7AC877C
:10EC7400BAA3D2A38EA3F6A385479CA0014A014957
:10EC8400CDB7014AF9BF7971AA8522D426D22221AF
:10EC9400AA84280806D64AD0EFF01FD2F24599E597
:10ECA4003DE185452285EFF08FFB75A0BC841547B7
:10ECB4006395E706B8858D4763F7E7046800EFF0CE
:10ECC4007FCE0359E100DD4763FB27018C86B7073C
:10ECD40017008507100822853EC8EF00D035BC8593
:10ECE4001109638527012285EFF06FF61C867246B1
:10ECF4006C00858B1106228591CFEFF03FE601C5AC
:10ED04002285EFF0CFF4884449DD9710FB1FE7809C
:10ED1400C04141BFEFF09FD2DDB711476389E700DF
:10ED24001387A7FF85463347070863ECE60231479C
:10ED3400F117B387E7021757FB1F13076758BA97F2
:10ED44009A2371D3A8233008A2850D204DFDB884E1
:10ED54009147E318F7F4B250225492540259456192
:10ED640082802C082285212E59FDF5B701114AC84D
:10ED74002A89314526CA4EC606CE22CCAE89B28433
:10ED84009710FB1FE780004D29C19307000A231148
:10ED940035011EA12A842146110595C0A685971028
:10EDA400FB1FE780E05AA2854A85EF500FB8014562
:10EDB400F2406244D2444249B249056182808145AD
:10EDC4009710FB1FE780405FF9BF0545D5B70111D8
:10EDD4004AC82A891305000226CA4EC652C456C21E
:10EDE4005AC006CE22CCAE8A328BB6893A8ABE8409
:10EDF4009710FB1FE780004621C9930720FA1CA146
:10EE0400A30065012311550123024501A302350125
:10EE14002A84614621059DC0A6859710FB1FE780C3
:10EE24002053A2856244F240D244B249224A924A13
:10EE3400024B4A85424905616F502FAF81459710B7
:10EE4400FB1FE7806057F1BFF2406244D24442495D
:10EE5400B249224A924A024B056182805C4579712B
:10EE640022D406D62A84AE86A5C7BA23F88513070A
:10EE740020066396E504FA231756FB1F0356C608BB
:10EE84003357C70AB22B9E2B1377F70F918F93F743
:10EE9400F70F01E6890793F7F70FBA97FD17B3C782
:10EEA400E702FC863E206E200824FC8401473C08CF
:10EEB4000146EFF0DFF1B250225445618280D82F31
:10EEC4009757FB1F83A707041207BA97FE23D1BFE6
:10EED4002EC61946814528089710FB1FE780C04DB0
:10EEE400B246C9B7797122D406D626D22A8491CDE6
:10EEF40008242E866E202254B25092548147014732
:10EF04009306000645616FF09FECB28428005946D1
:10EF14009710FB1FE780404A648499E43E204844EC
:10EF24006C007C85EFF08FB26E2008243C00014712
:10EF3400930600060146EFF09FE9B2502254925422
:10EF440045618280797106D6814799E53E217086B4
:10EF54007C845C4589EF3C002E866E2108250147A0
:10EF640093060006EFF0BFE6B25045618280BE23EF
:10EF74007C85D5B7411122C406C61C2111472A84B9
:10EF84006392E7022E866E21082581470147CD460C
:10EF9400EFF0FFE349466E202244B240154541019B
:10EFA4006FF0AFA513F7B70F89466317D700014673
:10EFB400EFF05FF35146C5B70D476398E70022446D
:10EFC400B240014641016FF0FFF7B24022444101D3
:10EFD40082809A21B14771173307F7029757FB1FB5
:10EFE4009387072EBA97D84301EBD841AAA70145C6
:10EFF400D8C3BA219AA7828059458280797126D2D2
:10F00400444522D44AD006D62A842E89B1C4C844A1
:10F0140019C59710FB1FE780401123A604009E200A
:10F024006E2008247C85BE200147930640067C861A
:10F034009E244A867C879C483EC83E207C843C00B3
:10F04400EFF0FFD8A38E240123A80400B250225469
:10F0540092540259456182802800314681459710B7
:10F06400FB1FE78060353E206E2008247C84014726
:10F074003C00930640064A86EFF07FD5C1BF797104
:10F0840052CC2A8A8A2126D206D622D44AD04ECEFF
:10F0940056CAAE84EFE0DFFF6302051240452A89B9
:10F0A400630E04107E21639B47111E24638A07109C
:10F0B400542C975AFB1F938AEAE403A70A0092068A
:10F0C400FD1736977A23B3C707081EA46316F70003
:10F0D40093053006EFF09FD85C48B5EBC8408349F0
:10F0E40015001C21A209B3E9F900BE2013872900E9
:10F0F400631AF702F9559710FB1FE7808010C8C008
:10F1040023913401034589002686D285EFF01FC67A
:10F114001DEDB250225492540259F249624AD24A25
:10F12400456182809565938515C04E859710FB1FB8
:10F13400E78080F248C8C840231C3401F955971071
:10F14400FB1FE780000CBE20C8C0F917BEA04848CA
:10F154002DCDB220362C1E2C3308D60063C90707E8
:10F16400582C83A70A0095451207BA97BE2363CA91
:10F174000705CC4036959710FB1FE780601D3A2C9D
:10F18400BE20BA971A2CB3C707083EAC6398E702AF
:10F194000357290003458900300078845848D285F4
:10F1A4007C853AC6EFF09FBC11C548489710FB1FF9
:10F1B400E780A0F7232A0400232C0400054591BF0F
:10F1C40099454A85EFE07FFED5BFA545DDBF914552
:10F1D400CDBFBE21F9C3011126CA06CE22CC1757D2
:10F1E400FB1F035767D2AA846D456363F70A2E8415
:10F1F400484091459710FB1FE780A0003E20AA8657
:10F204001CA13E20A1831CB11E203CA11E20A18371
:10F214003CB13220C167F917110633460608639FD3
:10F22400F4022AC4314532C69710FB1FE7808002DE
:10F23400AA854D45B1CD930700F93246A2469CA15B
:10F24400F957BEA18947DCA1F2A194C51755FB1F4C
:10F25400034525CCEF407FED01451DA8814526855A
:10F26400EF40D05B11E91757FB1F130767CA1C2334
:10F27400E5D7FD171CA3CDB789476302F5029D4767
:10F284006301F502C9476300F502FD47E30DF5FC90
:10F29400F2406244D244056182806D4582805145CA
:10F2A400C5BF1145F5B70945E5B7011122CC4AC8D8
:10F2B40031441309C5FF3304890226CA9754FB1F3E
:10F2C4009384040006CE26945C40A9C31757FB1F01
:10F2D400034707C40DC768843EC62A241E242C0095
:10F2E4007C85EFF01FEF11C548409710FB1FE780A6
:10F2F400C0E3B1473309F902CA9423A204000545C7
:10F30400F2406244D2444249056182800145CDBF46
:10F31400797126D244454ECE52CCFE20BA28975954
:10F32400FB1F83D969BE06D622D44AD056CAB3D9A4
:10F33400F90A2A8A9E282DCF998F4E8463D43701E7
:10F3440033C4070889452285EFF0EF9E2A89CD4A08
:10F3540031C5BE202AC660857C84BE2899EB9E28D0
:10F36400130925001CA19E28A1831CB163743405D4
:10F374008228BE28CC4422864A85BE959710FB1F5E
:10F38400E78000FD03556A002C00EFF09FE4AA8A91
:10F3940015C54A859710FB1FE78020D9B250225427
:10F3A40092540259F249624A5685D24A4561828092
:10F3B400890761B779143344040865BFBA289E20CD
:10F3C4003A949A28FD17B3C70708334404089EA04B
:10F3D400A2A86376E400F9F3FD57DCBCC1B781450C
:10F3E4005285EFF0BFC15DBF797122D44ECE56CAAB
:10F3F4005AC85EC662C406D626D24AD052CC9759A1
:10F40400FB1F938989B003CA0900975AFB1F938A8B
:10F414002AAF054B5284930BF00F175CFB1F130CA0
:10F42400FCAE83A40A0093174400BE9403C90400ED
:10F43400631D6907DC44B5CBD84725CB9A2339CB68
:10F444009757FB1F83C7C7AC99CF2685EFF05FECB6
:10F45400AA8505ED05049757FB1F83C737AB635196
:10F46400F40223808900B25022549254F249624A31
:10F47400D24A424BB24B224C4A85025945618280A2
:10F484009757FB1F238307A8F9BF2685EFF01FB703
:10F494000149D1BFDC3F639A770193052006268595
:10F4A400EFF0DF9BDC44A38E070083470C000504C8
:10F4B4001374F40F6363F4000144E31444F7C9BF05
:10F4C4004111154506C6EFF05FDE09C50545B2409A
:10F4D400410182801945EFF05FDD6DF91145EFF0D0
:10F4E400DFDC6DF51D45EFF05FDC6DF11755FB1F9B
:10F4F4000345D5A169DDB24041016FF0FFEE9E21C5
:10F504000D47F117B3C707086363F706DC414111E0
:10F5140022C406C626C22E84A9CF8545AA84952571
:10F5240039CD2685AD2BC167F917638FF40009ED3A
:10F534003E2099CB162019476395E6041757FB1F05
:10F544000357879C63FFE7029757FB1F83C7479CBA
:10F55400A285268599C72244B240924441016FF0A6
:10F564005FC72244B240924441016FF09FA609450F
:10F5740082800945B240224492444101828051452F
:10F58400D5BF6D45C5BF797126D252CCAA842E8AC7
:10F594005D4589454AD04ECE56CA06D622D4B28994
:10F5A400B68A3A89EFE03FF925C52A840145630606
:10F5B4000900D685130544000299935785003CB091
:10F5C40093074500230044017C85954728A07C844B
:10F5D400A300340122C69757FB1F83C767932C00EF
:10F5E400268585C7EFF0FFBEAA8411C52285971032
:10F5F400FB1FE78080B3B25022540259F249624A99
:10F60400D24A2685925445618280EFF09F9CE9BFDF
:10F61400CD44D5B7797126D24AD052CC56CA2E8958
:10F6240006D6BE8522D44ECE9947B284368ABA8A8B
:10F634006314F9062A220944EFE09FA52AC625C5CA
:10F644005C4583596500BE239EA0B24715472380BD
:10F654005701BAA31757FB1F1307378B10239305C2
:10F66400160093F5F50F0CA3D0A399E1854614A3D6
:10F6740051476317E9001547BAA0DC479A249AA7B3
:10F684005287A686CA854E85EFF0FFEF2A8432455D
:10F694000DC4EFE0DFAC01A842867400AA89EFE054
:10F6A4001F912A845DD1B25022852254925402596A
:10F6B400F249624AD24A45618280F945EFE07FC34C
:10F6C400DDB79E211CA19E21A1831CB1BE213CA1BA
:10F6D400BE21A1833CB1114582809E211CA19E21A3
:10F6E400A1831CB1BE213CA1BE21A1833CB1DE217A
:10F6F4005CA1DE21A1835CB1FE217CA1FE21A1835A
:10F704007CB1214582809E211CA19E21A1831CB134
:10F71400094582809E211CA19E21A1831CB1BE218A
:10F724003CA1BE21A1833CB1DE215CA1DE21A183E9
:10F734005CB1FE217CA1FE21A1837CB19E251CA588
:10F744009E25A1831CB5294582809A218546AA87D6
:10F7540018A19A21218318B19A216319D700BA21DB
:10F7640038A1BA21218338B1114582800945631D2E
:10F77400A700BA211945B8A3BA212183B8B3DA2165
:10F78400D8A3DA212183D8B382809E211CA19E2193
:10F79400A1831CB1BE213CA1BE21A1833CB1114572
:10F7A4008280797126D24AD04ECEB2842A89AE891B
:10F7B40029468145480022D406D636849710FB1F7B
:10F7C400E78080BF64868DE43E207C829747FB1FE0
:10F7D40083D787737C845C4481CFD42F1747FB1F66
:10F7E400032747729E27920636973A237C857883AF
:10F7F4004A8517070000130727F2540013F6F90F80
:10F80400D545EFF05FD82A8911C195E085471CA042
:10F8140023020400014681452285EFF0AFECB2508B
:10F8240022549254F2494A850259456182802285C4
:10F83400EFE0FF92EDB7B28617070000130727F138
:10F844002E8685456FF03FD40111688741657000AD
:10F8540001489307F00F0D47970600009386A6E62C
:10F8640099457D1506CEEFF0FFDAF24005618280FE
:10F87400B28701482E86114797060000938626E634
:10F88400C9456FF03FD9B286170700001307E7E7B1
:10F894002E86CD456FF03FCF011122CC26CA4AC82F
:10F8A4004EC606CEAA842E891754FB1F130444A403
:10F8B4009759FB1F9389C9A61C4081C7CA85268511
:10F8C40082971104E31A34FFF2406244D24442495D
:10F8D400B24905618280411122C406C626C2174777
:10F8E400FB1F1307E7737C2B783B1754FB1F130490
:10F8F400A4A41CB4BA9793F7F70F1CA4A5CB1305C3
:10F90400C0033385A702A56585059744FB1F93842F
:10F9140064609700FB1FE780207410249307C003E2
:10F9240081453306F60288C09710FB1FE780C0A804
:10F9340014249C4001477D566341D7022244B240BF
:10F9440092441306000381451755FB1F1305459A7E
:10F9540041011713FB1F670023A6B2A323820700EC
:10F9640023A6070205079387C703F9B7B2402244C9
:10F97400924441018280411122C426C24AC006C673
:10F984002A892E84B2849730FB1FE780C01909EDC1
:10F99400C167F91751456313F9000145B240224488
:10F9A400924402494101828054555C2195C213F767
:10F9B40027014146630BC700C18B3D45E5D3BC2EEF
:10F9C4000145E3FD87FC3145D1BF1545F5D4F9B7B1
:10F9D400C18B0145E1F71545D1B779714AD0416929
:10F9E40022D426D24ECE52CC56CA5AC806D6AA849F
:10F9F40001449759FB1F93892994174AFB1F130A43
:10FA04006A51930AC0037D19054B83C78900636457
:10FA1400F400014525A83307540383270A00BA9745
:10FA2400BA236316270105041374F40FF9BFC8330E
:10FA3400300093856700EFB051271946A68528004A
:10FA44009710FB1FE78040A2E31F65FDB2502254CC
:10FA540092540259F249624AD24A424B4561828029
:10FA64004166AA869755FB1F83C5858D1747FB1FE3
:10FA74000327474A81477D166394F5000145828038
:10FA8400035827003A856306C80003480700E308C3
:10FA9400D8FE850793F7F70F1307C703F1BF41118A
:10FAA40006C69730FB1FE780000809C54A29B24003
:10FAB400410182800145E5BF1747FB1F03278745A6
:10FAC4009756FB1F83C6C687110781470145639379
:10FAD400F6008280102301C605051375F50F85070E
:10FAE40093F7F70F1307C703DDB71755FB1F03453C
:10FAF400258582801747FB1F1307877F81473A8636
:10FB0400B1460C4391E5B3C7C72088C30145828041
:10FB140085071107E397D7FE4D458280411106C63C
:10FB240022C49730FB1FE78000000DCD2A842A21D0
:10FB34008545EFF07FD6485409C59700FB1FE78041
:10FB4400C05E22851306C00381459710FB1FE78022
:10FB5400A086FD573EA0230204000145B240224482
:10FB6400410182800945DDBF411106C69730FB1F64
:10FB7400E78060FB09C54825B24041018280014508
:10FB8400E5BFC167F9176305F502411122C406C632
:10FB94002E849730FB1FE78000F9AA87014589C7A7
:10FBA400DC237D8C33358000B240224441018280C5
:10FBB40005458280411122C406C62E849730FB1F5E
:10FBC400E78060F601CD5A29AA87054563048700BA
:10FBD400C2AB0145B2402244410182800545DDBFEC
:10FBE40039CD01114AC8416922CC26CA4EC652C435
:10FBF40056C206CEAA8401449749FB1F9389C97350
:10FC0400174AFB1F130A0A31930AC0037D1983C7DD
:10FC14008900634BF400F2406244D2444249B24941
:10FC2400224A924A05618280B307540303250A00DD
:10FC34003E953E216383270182940504C9BF8280D7
:10FC44009747FB1F83A7072DC1661746FB1F034673
:10FC5400266F890701450147FD1691456313E600A8
:10FC6400828003D807006309D80003C8A70063157E
:10FC7400B80005051375F50F05071377F70F93877C
:10FC8400C703E9BF9746FB1F83A6C6281746FB1F79
:10FC94000346066B910601478147631FE60085838F
:10FCA40093C7F7FF0545B3C707086361E50233153A
:10FCB400A0283345050882808C2299C1CE36CD8F89
:10FCC40005071377F70F9386C603C1BF93F6170092
:10FCD400F9FE050585831375F50FC1BF797156CA01
:10FCE400AA8A2E8526D24AD04ECE52CC5AC85EC697
:10FCF40062C406D622D4AE84328B368CBA8B3E8A4A
:10FD0400C28946899730FB1FE780E0E13DED4165FC
:10FD14007D159730FB1FE78000E12A84554531C8E3
:10FD24001946DE8513056400A30284019700FB1FB6
:10FD3400E78000628357010326A0230264013EA8E2
:10FD44008357410323005401232604025EA823069B
:10FD540044012317340123182401EFF0BFF20AB839
:10FD6400232A04022685232C04028145EFF0DFB206
:10FD74000145B250225492540259F249624AD24A7D
:10FD8400424BB24B224C456182804545DDB79746D4
:10FD9400FB1F83C6E65A1747FB1F0327A717814794
:10FDA4006395F60041657D1582800E3B1306C703FB
:10FDB4006394A5002A238280850793F7F70F32877F
:10FDC400C5B741661748FB1F034888579746FB1F72
:10FDD40083A6461401477D16954811436314E80031
:10FDE40001458280BE223685638EC702CC5A9DC9E6
:10FDF400BC31AC2189CD938597FD93F5F50FE37262
:10FE0400B3FE9387D7FA93F7D70F89EF8280938550
:10FE1400F7FD93F5F50FE3F6B8FC9387D7FA93F75C
:10FE2400D70FE1D305071377F70F9386C6037DB782
:10FE340041669745FB1F83C5A5501747FB1F032742
:10FE4400670D81477D1625486394F500014582803E
:10FE540036233A85638BC600545B81CAB4329386D9
:10FE6400E6FD93F6F60FE374D8FE850793F7F70FD4
:10FE74001307C703D1BF011122CC2A84494506CEFA
:10FE8400EF607FD61DC12AC622859730FB1FE7800D
:10FE940080C901CD624432460E39F2401745FB1F3A
:10FEA4000345B54905616F406FCEF2406244056178
:10FEB400828079714ECE52CCAE892A8A9305300560
:10FEC400414526D24AD056CA5AC806D622D4328BC5
:10FED4003689BA8A9700FB1FE7800018CD4429C9E8
:10FEE4002A848944638109044146814523126101BE
:10FEF4009700FB1FE780404C5686CE8522859700ED
:10FF0400FB1FE780E0442146630F0902CA852800ED
:10FF14009700FB1FE780C043A28650002C00528547
:10FF2400EF30F07EAA8422859700FB1FE780E01F54
:10FF3400B25022540259F249624AD24A424B2685AF
:10FF4400925445618280814528009700FB1FE78019
:10FF5400A046D9B7411122C4405926C206C6AA8474
:10FF640029CC085409C59700FB1FE780001C2858BA
:10FF740009C59700FB1FE780401B685809C5970017
:10FF8400FB1FE780801A285C09C59700FB1FE780E8
:10FF9400C019685C09C59700FB1FE7800019032599
:10FFA400040809C59700FB1FE780201822859700E5
:10FFB400FB1FE780801723AA040222448E38B24034
:10FFC40092441745FB1F0345553741016F406FE5C8
:10FFD400411126C206C622C4AE849730FB1FE780B7
:10FFE40080B431C9032345032A84630603048328A8
:0CFFF400C3070328830783274307032764
:020000025000AC
:1000000003078346630003560300834523002685C8
:10001000EF60BFC52285EFF03FF4EFF0BFE111CDF7
:100020002244B24092441745FB1F03455531854594
:1000300041011733FB1F67008398B240224492446A
:1000400041018280411122C426C206C6AA842E84A0
:100050009730FB1FE78060AD5C5989CF9E23639B7F
:10006000970085476318F4002244B240924441014E
:100070006FF09FEEB24022449244410182804111D0
:1000800006C622C426C2EFF01FD429C144592A84CF
:1000900095CCBC209DC79747FB1F83A767E889C7FE
:1000A000DC4399C326858297B8309307F002631F1B
:1000B000F7002A202244B2409244814541016FF06A
:1000C0007FF19747FB1F83A767E5D1BFB24022446A
:1000D000924441018280411126C24AC006C622C410
:1000E000AA842E899730FB1FE78020A405CD4059B4
:1000F00055C41E206394970A3C3013071002639581
:10010000E7083C20ADCF7C5403270408DE2B15E321
:1001100013F7170019CF18545A23058B19CB9307DF
:1001200020023CB0B24022449244024905454101BC
:10013000828013F7270001CB18545A23098B01C77B
:1001400093074002F9BF918B81CB1C54DE23918B26
:1001500081C793076002F1B79747FB1F83A747DC6E
:10016000F1D3DC43E1D32285829738309307F00244
:100170008145E319F7FA2685EFF0DFE565B7974784
:10018000FB1F83A7A7D9E9BF1307A0026398E70065
:100190006304090013092003CA85F1BF631C090029
:1001A00026859730FB1FE780409809C55C2193E7BF
:1001B00007015CA1A6854A85EF60EFBAA5B70111DA
:1001C00026CA99476C85AA842E858D4522CC4AC8BB
:1001D00006CE328936847C84EFE02FB62AC61DC94C
:1001E000AA854A8502942A8419E52C002685EFF019
:1001F0004FB12A8411C532459700FB1FE78020F3D9
:100200002685EFF09FC7F24022856244D2444249DE
:10021000056182804D44EDB7411122C42E862E84A3
:10022000971600009386867A894506C626C24AC07C
:100230002A89EFF0DFF80C20AA844A85EFF09FD9D5
:10024000B240224402492685924441018280974768
:10025000FB1F83A7A7CC85CB9C4395C71D71A2CC60
:1002600086CE984110082A843AC8D84185453ACAB2
:10027000829711C548862A206C00EFF0FFF9F640FE
:100280006644256182808280AA872E8591CFFC57A3
:1002900081CF982398A1983398B1B82BB8A1982F03
:1002A000DC4BB8B1DCC18280414681451703FB1F9E
:1002B0006700C3109747FB1F83A787C681C79C476A
:1002C00091C38287094582801747FB1F032787CB8D
:1002D0001DC75843AA8705450DC703A50708411147
:1002E00006C6930605021306050C930505061305BD
:1002F00005040297B2401375F50F41018280054550
:10030000828082804DC9357122CD2A840A2126CB74
:1003100052C556C35AC106CF4AC94EC7DEDE2E8A21
:10032000B28A368B9730FB1FE7802080AA8431C5C4
:100330000C182285EFF05FF53C20938B6400A9CB6D
:10034000EF501FFC2A89014583C95400EF50DFF8A4
:10035000AA840C100818EF10A04908542C10EF10B4
:10036000C049DE88A68B5AC04E88DE874A871410A3
:100370003010D6855285EF20E074FA406A44DA44A2
:100380004A49BA492A4A9A4A0A4BF65B0D61828069
:10039000EF501FF7AA89014503C95400EF50DFF35E
:1003A0002ACE08540C10EF10A0442C100818EF109F
:1003B000C044F2484DBF8280AA8701CD18554145FF
:1003C00011CBFC5781CB28333D476375A700882F9D
:1003D0008280414582806DC5411122C406C626C275
:1003E000AA872E840945E1C998337D761306F67FE6
:1003F00098A1B8234D4598B1B833B8A1D823B8B166
:10040000D433DA21858AA2061377F7EF558FDAA164
:10041000D433334707081377F7DF93D61648A60679
:10042000558FDAA1D433334707081377F7BF93D634
:100430002648AA06558FDAA1D43333470708718FAF
:1004400093D63648AE06558FDAA1F4233347070812
:10045000799B858A558FDAA1F42333470708759B6A
:10046000898A558FDAA1F423334707086D9B918A57
:10047000558FDAA1F823DE21218BDD9BD98FDEA1F8
:10048000EF60AFF6AA845145EF602FF6383093F451
:10049000F40FAA8749456360970293F7F70F63EC5F
:1004A000E70018209147614563E7E700183085476A
:1004B00063E3E7000145B240224492444101828057
:1004C0000945828015C52A87AE87094585C5411132
:1004D00006C6143313851700194694A19305270007
:1004E0009700FB1FE78000E7B24001454101828091
:1004F0000945828082800DC9AA872E8709459DC53E
:10050000411106C6B423903313052700A206D18EED
:1005100096A12146938537009700FB1FE78080E373
:10052000B2400145410182800945828082801DC11F
:100530002A87AE8709458DC141113E854146930505
:10054000170006C69700FB1FE780C0E0B2400145D8
:1005500041018280094582808280AA87094591CB2A
:1005600089C99C333D4761456365F7009CA10145FE
:100570008280828005C52A87AE87094595C14111D1
:100580003E85130600049305170006C69700FB1F5F
:10059000E78040DCB240014541018280094582800C
:1005A00082801D71A2CC2A84084586CEA6CA230665
:1005B0000100042135479387F4FF93F7F70F636237
:1005C000F70A17D701001307E769B3C7E7209C4371
:1005D000BA9782870C08EFF01FE0C947631CF50447
:1005E00099475C862A206C00EFF01FC3F6406644F2
:1005F000D644256182800C08EFF03FF61DED2A20DD
:100600009720FB1FE7806052A14705C15825631C56
:10061000F7041747FB1F0327A7909D4719C71843E7
:1006200009C71008A6850297AA875C8629A00C082E
:10063000EFF07FEC69D51C86D5F72A20EFF0FF8319
:1006400075B70C08EFF01FE8F5B71C312308F1006F
:100650007DB70C08EFF01FF2F1BF0C08EFF03FED93
:10066000D1BF9D47BDBF1747FB1F0327278B75B71A
:10067000411122C406C626C24AC018219307200988
:100680002A84631AF7101C3139476395E70A56210B
:100690000967610781476398E6089744FB1F9384C5
:1006A0006488884049C10C4403C90500631D0900E2
:1006B0001C2185052146B9CB29059700FB1FE78042
:1006C00060C99C40A5C349459700FB1FE780C0B89F
:1006D0002A841DC1930710FC1CA1A30025018C4096
:1006E0000905414689059700FB1FE780A0C69C408D
:1006F000A2858833EF30BFA388409700FB1FE780B7
:1007000000A39747FB1F23AF078029A8090597007F
:10071000FB1FE78020C4EF30807F05495DF19C40DE
:10072000238027018547B2402244924402493E85F6
:10073000410182801307E003639DE7063821954756
:100740006319F7024A21EFF06FC29147E31CF5FCF1
:100750009737FB1F83A7877CF1D79C47E1D772248B
:100760004A20930564002244B24092440249410168
:100770008287A147631BF7006C204A202244B240C5
:100780009244024941016FF01F959306000381478F
:10079000E31BD7F8D5B79306000A8147E315D7F8CE
:1007A000EFF03FE008443DDD9700FB1FE780209815
:1007B00095BF81478DBF011122CC06CE26CA4AC8FB
:1007C000094415CDAE8409449DC92A898D45680028
:1007D000EF509F841C8726866C0093F7F70393E7FE
:1007E00007044A855C87EF20E0242A8409E90D4646
:1007F0006C00138534009700FB1FE780A0B5F24022
:1008000022856244D2444249056182805D714EDE98
:1008100086C6A2C4A6C2CAC052DC56DA5AD85ED670
:10082000894955C9328989495DC6138B45002A8A91
:10083000AE8A334B0B08930530055A859700FB1F92
:10084000E780C0812A84CD4959C5EF505FADAA84A5
:100850005686D28593DA840013DA040193FBF40FF1
:100860001305440093FAFA0F137AFA0FE180970008
:10087000FB1FE78060C4A301740123015401A3009E
:10088000440104A0EF501FA9AA854146080897001B
:10089000FB1FE78060C2214734005A86A285080802
:1008A000EF20C03FAA891DE121462C0023007901D9
:1008B000A300590123014901A3019900130549002F
:1008C0009700FB1FE78040BFEF503FA622859700AF
:1008D000FB1FE780C085B640264496440649625A0D
:1008E000D25A425BB25B4E85F259616182804111FE
:1008F00026C2AA842E854AC006C622C42E89972005
:10090000FB1FE780802269C5405969C45C300947F4
:1009100093F6B70F6387E60011471305E00F639561
:10092000E7081E2009456391270913098400414601
:10093000A6854A859700FB1FE780C0A14146A68592
:10094000130584019700FB1FE780C0A0383085465F
:100950009307F7FE93F7F70F63EEF6049304C403CF
:100960009737FB1F83A70762C14526858DC79C4F1C
:100970009DC382979306C4022686CA852285EFF01E
:100980007F983C2081CF22852244B2409244024984
:1009900041016F10E00BEF502FE8E9BF3830C94735
:1009A000E303F7FE3CB00145B240224492440249C1
:1009B0004101828093071005E317F7FE3C20E5D73D
:1009C00022852244B2409244024941016F10800EB8
:1009D0000945D9BF4945C9BF797152CC2A8A3285A8
:1009E00022D44AD04ECE06D626D2AE89328997205E
:1009F000FB1FE7808013494405C9445949448DC40D
:100A00009E2063932703DC30A18B85EB0944B8302B
:100A10009307B005631AF7002685EF108006BC2007
:100A2000ADCB9307C005BCB0B2502285225492547E
:100A30000259F249624A456182801739FB1F130946
:100A40006954832709001304E00FF9DF9C47E9DFAD
:100A50001384840122854146D2859700FB1FE780DD
:100A6000608F8327090083A5040822869C4793850D
:100A700005042E850A87814682972A844146CE85C1
:100A80000A859700FB1FE780609E49D11374F40F1D
:100A9000BDBF9307E00541BF39C9011122CC26CA69
:100AA00006CEAA842E84094595CD0D468D052800D5
:100AB0009700FB1FE780008A1C8570002C0093F7CD
:100AC000F70393E7070426855C85EF10B07619E9F4
:100AD0000D46A28568009700FB1FE78020997D15D1
:100AE0003335A000F2406244D2440561828009455A
:100AF0008280011152C42A8A32854EC656C25AC01B
:100B000006CE22CC26CA4AC82E8BB28AB689972036
:100B1000FB1FE780800109ED8944F24062444249AD
:100B2000B249224A924A024B2685D244056182800C
:100B30005C592A89C544F5F34D45EF600F8B13745A
:100B4000F50F5145EF606F8AE38809FC03C78901FF
:100B5000E36487FC9377F50FE3E0E7FC930530054A
:100B60001305400897F0FA1FE780404F232AA90297
:100B70002A84CD445DD11306400881459700FB1FB0
:100B8000E780C083A3010400230144012302640120
:100B9000231054012326340723240402A302040053
:100BA00063070A002285EF00F064AA8419E18144FA
:100BB000ADB74A85EFF04FBA8DB7397122DC06DE4A
:100BC00026DA4AD84ED652D456D25AD05ECE62CC0D
:100BD00066CA0944630A0610BA840944630607100A
:100BE000AA8B2E89328B368C9720FB1FE780E0F38F
:100BF000AA8A514475C993053005414597F0FA1FFB
:100C0000E780C045AA894D4465C198309C2003CA3D
:100C1000340022075D8FBC20620AC207D98F336A75
:100C2000FA0083A78A0263E647017D570944639867
:100C3000E70A6307090083C74A000544898BC5C3D7
:100C4000214681450A8597F0FA1FE7802077930CAB
:100C50004C0093053005B3CC0C08668597F0FA1F5D
:100C6000E780C03F2A894D443DC96286DA85110577
:100C70009700FB1FE78040841146A6854A859700B0
:100C8000FB1FE7806083414693858A014E8597006C
:100C9000FB1FE780608221478A866686CA854E856B
:100CA000EF10D07F2A841DE521468A852800970011
:100CB000FB1FE7806080214693854400280097F061
:100CC000FA1FE780A07A8547631EF502D2855E850C
:100CD000EF608FAD4A8597F0FA1FE78040454E855B
:100CE00097F0FA1FE780A044F25022856254D25454
:100CF0004259B259225A925A025BF24B624CD24C80
:100D0000216182800544F9B7797122D406D626D2B2
:100D10004AD04ECE2E849397556063D607049734FD
:100D2000FB1F9384A461A83097F0FA1FE780C05896
:100D30002AC609CDEFF0DF93B24511E5A82093074D
:100D4000F00F631FF5002E85EF304FB91319F468CB
:100D5000B25022549254F2494A8502594561828028
:100D6000EF30EFBCE5B713F9150063070900EFF0AA
:100D70000FB113491400E9BFE1DD854421A08504CA
:100D800093F4F40FEFE0BFD6E3F4A4FCB31790287C
:100D9000B3C90708E18FE5D74E85EFE09FFFC16734
:100DA000FD176305F500DD45EFF0CFA233493401AF
:100DB00045B79737FB1F23A707169737FB1F23A1BC
:100DC00007169737FB1F23AB07149737FB1F938733
:100DD0002756170700001307675D98C31707000021
:100DE0001307472FD8C317F7FFFF1307070D98C73F
:100DF0009737FB1F93870753171700001307A74563
:100E000098C317170000130767FED8C31717000011
:100E10001307672998C782809737FB1F83C74752FC
:100E2000A18B014789C71737FB1F130767509737F7
:100E3000FB1F23A7E70E014582809737FB1F83C75F
:100E40002750918B014789C71737FB1F1307874D21
:100E50009737FB1F23A4E70C01458280011106CEC2
:100E60002AC6EFF01FF5324599459737FB1FA38837
:100E7000A74CEFD0AFE7F24017F5FFFF1305C51CF5
:100E800005616FE07FC71C5599C3214582804111E0
:100E900022C426C22A84AE841305000493053005BB
:100EA00006C64AC097F0FA1FE780401B08D469C9FC
:100EB00013060004A68597F0FA1FE780A049745432
:100EC000B82A93778700FDCB1C54BC23A18BFDC7A8
:100ED00083270408D5E7930530051305001097F024
:100EE000FA1FE780A017AA872320A4080D45D1CBBD
:100EF00074549C309832C1CF3337E0000E079367AB
:100F000007016C545CB0B829058B19CB1854854681
:100F100038230D8B6316D70078201367170078A04D
:100F20000327040809C778201367870078A00547BE
:100F3000639FE70C13098400414681454A8597F079
:100F4000FA1FE780A047814513058401414697F0C9
:100F5000FA1FE780A0469304C4039737FB1F83A7BB
:100F60006702C1452685B5CF9C4FA5CF82978327C1
:100F70000408BDCB2285EF00F0339307000549C17B
:100F80002145B24022449244024941018280A14756
:100F90002DFBBC20918B91E7BC2A918B99E385476F
:100FA0008DB79820942295473307F70297D7010011
:100FB0009387C7CEBA97B6979C23A1B79C3081C7B9
:100FC0009032E1471DFEBC205D8F118B69DB9820BC
:100FD000954794223307F70297D701009387C7CD2F
:100FE000D1BFEF506F8361B722859306C402268676
:100FF000CA85EFF02FB12285EF00902551F1C1474E
:101000000A203CB08145EF503FE401459DBF13F7F6
:10101000870151C7C18B930484004146B1CB890538
:10102000268597F0FA1FE780E03281451305840199
:10103000414697F0FA1FE78060387C201309C4030B
:10104000C14593E747007CA09737FB1F83A787F331
:101050004A8595C79C4F85C78297832704089DC3FF
:101060002285EF00302509FD930720053CB071BFB4
:101070008145268597F0FA1FE78040347DB7EF4021
:10108000BFF9E1BF9306C4024A86A6852285EFF028
:101090006FA72285EF00D01BCD4769D9D5B5094789
:1010A00085456388E70093F7D70F11476396E700FC
:1010B00089450A20EF505FD97C2093E747007CA048
:1010C0008327040881C7930710054DB7C54779BF2B
:1010D0003C21638E0724397122DC06DE26DA4AD8E9
:1010E0004ED652D43C31130750052A846397E70843
:1010F00003497500173AFB1F130ACAE89309C50391
:1011000093573900AA97842783270A00C1454E8543
:10111000B5C39C4FA5C3829783270A00A1C79C47EC
:10112000B1C30325040813797900B3D62441858A15
:1011300093050504180893E606084E86130505086E
:1011400082971375F50F19ED41460C081305C4027B
:1011500097F0FA1FE78000202285EF00700F9307B9
:1011600060053CB0F2506254D2544259B259225AEE
:1011700021618280EF405FEA45B713071002639256
:10118000E7021C5503270508DE2371E713F7071054
:1011900079C378555A2B1377071055CF93077002F0
:1011A0003CB03C3013077002639DE70C3C5885E36C
:1011B00093053005714597F0FA1FE78020EA28D89B
:1011C00019C57146814597F0FA1FE780201F245802
:1011D000B1C4BC2C89E72285EFF00F9EA8AC28583B
:1011E0008145414697F0FA1FE780401D28583D474A
:1011F0002C2D9387F5FF93F7F70F6364F700EF400B
:10120000BFE1EF205FFD3C58A1458AAB1385270164
:10121000EF409FE02C580A20EF00503393078002E4
:101220000A203CB09720FB1FE7802090414609C56B
:101230007E2513D617003E966254F250D25442597E
:10124000B259225A1735FB1F0345750F060685450F
:1012500021616F30EF9313F7072009CB78545A2B95
:101260001377072001C7930790021DBF93F707402C
:101270008DDB7C54DE2B93F7074085D79307B002B4
:1012800005B713078002639FE7023C5899C78E2B6E
:101290000A2013862701EF00D0301C54DE2313F7F9
:1012A000072011C778545A2B1377072035EF93F78F
:1012B0000740A5CB7C54DE2B93F70740BDC39307B3
:1012C000B002B9BF13079002639BE700EF50EF83B2
:1012D000AA850A20EF00F02B9307A00291B713070D
:1012E000A0026396E702EF50AF81AA8585470145CA
:1012F0006384F500814505452EC6EF40FFFD2A8633
:10130000B2450A20EF0090251C54DE234DB7130789
:10131000B0026398E700EF40FFFFAA850A20EF00C4
:10132000B02B9307F00235BD93079002D5BD8280A4
:10133000411122C4405926C206C67C54AA84DE2B21
:1013400013F7071011C718545A23137707100DE32A
:1013500013F7072011C718545A231377072009EBF6
:1013600093F707408DCB1C54DE2393F7074085C7C6
:10137000930710023CB02285EFF09FD538309307D9
:10138000F002631EF7002244AA20B2409244814535
:1013900041016FE03FC49307F0023CB0EDB7B240AB
:1013A0002244924441018280397122DC405926DA7C
:1013B0004AD84ED606DE2A89AE84B289630604383E
:1013C0002A211E206391A7123C20638A0738938745
:1013D000E5FF93F7F70F2D476363F73817D7010041
:1013E0001307478FB3C7E7209C43BA9782872285AC
:1013F0006254F250D2544259B259B28521616FF011
:101400009FA84146CE851305C40497F0FA1FE780D4
:1014100060F42285BD25383093074005631AF70034
:10142000930790053335A000931435003CB06DA8A8
:1014300093066005D147E317D7FE9307A005DDB7F4
:101440001309C4054A854146CE8597F0FA1FE78007
:1014500060F0032504085DC53C30130790056397D1
:10146000E7002285452D9307E005A5A81307A005F1
:101470006394E7087C3013D73700229714279D8B9D
:10148000B3D6F640858A9737FB1F83A7A7AF93E6AD
:101490000608B1CB9C47A1CB9305050818084A86DE
:1014A0001305050482971375F50F15ED41460C08D9
:1014B0001305C40497F0FA1FE78040FB7C304D47CA
:1014C000850793F7F70F7CB0E36DF7F8854517357F
:1014D000FB1F0345D5E69710FB1FE780404E93079F
:1014E00050053CB031A8A144F25062544259B2595F
:1014F0002685D254216182801307C005E383E7F675
:101500008144DDB7930984004A86CE85228514087C
:10151000EFE05FDF41469305C404080897F0FA1F27
:10152000E780C0F471D18A861306C403CA854E854C
:10153000EF10606DA1440DE12285EFE0FFE72A87FF
:101540000A209737FB1F83A727DF814601468A853C
:101550008297B334A0008E0493072002C1BD0C22F1
:10156000EFE05FA771BF3830930720026319F71EC1
:101570007C5889EB93053005714597F0FA1FE78099
:10158000E0AD68D86858630C051C4146CE8597F0DD
:10159000FA1FE78020DC64582285EFE0FFE1A8AC69
:1015A000930730023DBF3830930730026319F71AB2
:1015B0001E2268582146938529001EA9490597F0E7
:1015C000FA1FE78020D97C54DE2B13F727002DC7A4
:1015D00018545A23098B2DC39307400219B738308A
:1015E00093074002631DF7163C5C81EB85455D4522
:1015F00097F0FA1FE78080A628DC285CE30205F05C
:1016000083C709004146CE857CA997F0FA1FE78081
:1016100060D493075002F1B538309307500263103D
:10162000F714285C194693851900410597F0FA1FB5
:10163000E78040D27C54DE2B918B95CF1C54DE2367
:10164000918B95CB9307600269BD7C5C89EB930518
:101650003005514597F0FA1FE78040A068DC685CD0
:10166000E30305E84146CE8597F0FA1FE78080CE78
:101670007C5C7D5798CB4A85EFF09FCB51B5032515
:10168000040813060004CE851305050497F0FA1F1D
:10169000E78040CC2285EFE03FC33C3013070005D4
:1016A0006395E700930740052DBD13071005E38FF1
:1016B000E7E013072005E395E7E49737FB1F83A7CF
:1016C000678CE38207E29C47E38F07E083250408E9
:1016D00093048400180893850508814626862E8584
:1016E00082970A201008A685EF50EFFE9307B005F9
:1016F000CDBB38309307E0056313F7068325040854
:1017000041464E8597F0FA1FE78040D6AD44E30D81
:1017100005DC032504084146CE8597F0FA1FE780D3
:1017200060C32285EFE05FC92A872C580A209737CB
:10173000FB1F83A767C0814601468297B334A00090
:101740008E0493071002DDB1AD47E39BF5DA142256
:101750002E21130665000821EF409FF355B39D44E9
:1017600061B3AA87094541C6D9C11CA29C211CB2FC
:101770009C313CA2BC213CB2BC31A30206005CA25D
:10178000DE2193D787485CB2DA211377072001C79F
:1017900093E727005CB2DE2193F7074089C75C32EC
:1017A00093E747005CB2DE211317B028F98F89C791
:1017B0005C3293E787005CB223030600DE21858B51
:1017C0007CA2DA21098B01C793E727007CA2DE21E6
:1017D000918B89C77C2293E747007CA2DE21A18BF5
:1017E00089C77C2293E787007CA2014582808280A2
:1017F0002E86AA8505456FF0DFF62E86AA85094557
:101800006FF03FF68DC52A87094505C7411106C609
:10181000AE878D4694A1138517004146BA8597F08F
:10182000FA1FE78020B3B24001454101828009459B
:10183000828082808DC52A87094505C7411106C669
:10184000AE87914694A1138517004146BA8597F05B
:10185000FA1FE78020B0B24001454101828009456E
:10186000828082808DC52A87094505C7411106C639
:10187000AE87994694A1138517004146BA8597F023
:10188000FA1FE78020ADB240014541018280094541
:10189000828082809DC92A87094515CB411106C6E1
:1018A0009D4694A11623AE871385370094B1162365
:1018B0002146A182B4A19305270097F0FA1FE78083
:1018C00060A9B24001454101828009458280828041
:1018D0008DC52A87094505C7411106C6AE87A146B1
:1018E00094A1138517004146BA8597F0FA1FE78047
:1018F00060A6B24001454101828009458280828014
:1019000085C92A8709451DC7411106C6A54694A168
:101910001423AE871385270094B119469305170049
:1019200097F0FA1FE78000A3B24001454101828091
:101930000945828082808DC52A87094505C74111E6
:1019400006C6AE87A94694A1138517004146BA85FD
:1019500097F0FA1FE78000A0B24001454101828064
:1019600009458280828095C52A8709450DC74111A6
:1019700006C6AE87B14694A113851700130600046E
:10198000BA8597F0FA1FE780E09CB240014541011B
:1019900082800945828082808DC52A87094505C7D6
:1019A000411106C6AE87B54694A11385170041467E
:1019B000BA8597F0FA1FE780E099B24001454101EE
:1019C0008280094582808280AA87094581C999C79A
:1019D000154798A19C2301459CB182808280AA87EB
:1019E000094581C999C72D4798A19C2301459CB100
:1019F000828082800DC55D718A8586C6A2C42A84D4
:101A0000EFE09F880A200A8697060000938686DE0C
:101A10009D45EFE0CFFAB6402644616182800545DE
:101A200082800DC55D718A8586C6A2C42A84EFE0D6
:101A3000BF850A200A8697060000938646DC9D45EE
:101A4000EFE0EFF7B6402644616182800545828071
:101A50005D71A2C49305C5022A8441460A8586C6E3
:101A600097F0FA1FE780008F0A200A869706000089
:101A7000938686D9C545EFE08FF4B6402644616170
:101A800082805D71A2C49305C5032A8441460A85FC
:101A900086C697F0FA1FE780E08B0A200A86970631
:101AA0000000938666D9C545EFE06FF1B640264445
:101AB000616182809727FB1F83A7C74CA9CB9C43FA
:101AC0005D71A2C486C62A841305E00F8DCF03255D
:101AD00004089305050C130505088297832504085F
:101AE000130600040A859385050897F0FA1FE7801E
:101AF00060860A2097060000938626E70A869305EB
:101B00001004EFE0CFEBB6402644616182801305FC
:101B1000E00F8280317122DD2A840A2126DB06DF74
:101B20004AD94ED752D556D35AD15ECF62CD66CB65
:101B30009710FB1FE78060FF3C58AA8489EB930550
:101B40003005714597E0FA1FE780405128D82858A2
:101B5000CD4715C97146814597F0FA1FE780008689
:101B6000032904072285EFE03F85230DA9003C20CF
:101B70001729FB1F130909416382071283270900F4
:101B80008DE39307E00FFA506A54DA544A59BA5970
:101B90002A5A9A5A0A5BFA4B6A4CDA4C3E852961FA
:101BA000828003AC0701E30E0CFC032B0408EF401A
:101BB0002FF5AA8B0145EF402FF2DC303458130B80
:101BC0000B029309C403130AC405938A64002A878D
:101BD00036C0B337F000930801045688B33670015D
:101BE0005286CE855A85029C1C54B8232307E102F5
:101BF0009833A306E1029C232306F1028327090000
